:020000040800F2
:1000000000060020E1010008E3010008E301000808
:10001000E3010008E3010008E3010008E301000830
:10002000E3010008E3010008E3010008A92F00082C
:10003000E3010008E3010008E3010008E301000810
:10004000E3010008E3010008E3010008E301000800
:10005000E3010008E301000851320008793200088A
:10006000A1320008C9320008F1320008E30100089B
:10007000E3010008E3010008E3010008E3010008D0
:10008000E3010008E3010008E3010008E3010008C0
:10009000E3010008E3010008E30100081933000848
:1000A000E3010008E3010008E3010008E3010008A0
:1000B000ED330008E3010008E3010008E301000854
:1000C000E3010008E3010008E3010008E301000880
:1000D000E3010008E3010008E3010008E301000870
:1000E0007D330008E3010008E3010008E301000894
:1000F000E3010008E3010008E3010008E301000850
:10010000E3010008E3010008E3010008E30100083F
:10011000E3010008E3010008E3010008E30100082F
:10012000E3010008E3010008E3010008E30100081F
:10013000E3010008E3010008E3010008E30100080F
:10014000E3010008E3010008E30100085D2700085F
:10015000E3010008E3010008E3010008E3010008EF
:10016000E3010008E3010008E3010008E3010008DF
:10017000E3010008E3010008E3010008E3010008CF
:10018000E3010008E3010008E3010008E3010008BF
:10019000E3010008E3010008E3010008E3010008AF
:1001A000E3010008E3010008E3010008E30100089F
:1001B000E3010008E3010008E3010008E30100088F
:1001C000E3010008E3010008E3010008E30100087F
:1001D000E3010008E3010008E3010008E30100086F
:1001E00002E000F000F8FEE772B6374880F30888B6
:1001F000364880F3098836483649086040F20000E6
:10020000CCF200004EF63471CEF200010860BFF36C
:100210004F8FBFF36F8F40F20000C0F2F0004EF638
:100220008851CEF200010860BFF34F8FBFF36F8F8C
:100230004FF00000E1EE100A4EF63C71CEF20001E4
:100240000860062080F31488BFF36F8F01F04EFF23
:1002500002F048FE4FF055301F491B4A91423CBF07
:1002600041F8040BFAE71D49184A91423CBF41F896
:10027000040BFAE71A491B4A1B4B9A423EBF51F83E
:10028000040B42F8040BF8E700201849184A914281
:100290003CBF41F8040BFAE701F02CFF02F076FEB8
:1002A000144C154DAC4203DA54F8041B8847F9E7A7
:1002B00000F042F8114C124DAC4203DA54F8041B22
:1002C0008847F9E701F014BF000600200022002053
:1002D0000000000808ED00E00000002000060020FB
:1002E000B0370008002200204022002040220020D9
:1002F000602E0020E0010008E0010008E001000895
:10030000E00100082DE9F04F2DED108AC1F80CD066
:10031000C3689D46BDEC108ABDE8F08F002383F3CF
:1003200011882846A047002001F090FAFEE701F06E
:100330001FFA00DFFEE7000038B500F0BFFB01F058
:10034000A5FE054601F0C8FE0446C8B90E4B9D4205
:1003500018D001339D4218BF044641F2883504BFCE
:1003600001240025002001F09BFE0CB100F074F880
:1003700000F01EFD284600F0C3F800F06DF8F9E724
:100380000025EFE70546EDE7010007B008B500F0EE
:1003900067FBA0F120035842584108BD07B541F260
:1003A0001203022101A8ADF8043000F077FB03B07E
:1003B0005DF804FB38B5302383F3118817480368D0
:1003C0000BB101F00FFB164A144800234FF47A7169
:1003D00001F0FEFA002383F31188124C236813B155
:1003E0002368013B2360636813B16368013B63606A
:1003F0000D4D2B7833B963687BB9022000F038FCCF
:10040000322363602B78032B07D163682BB902205A
:1004100000F02EFC4FF47A73636038BD4022002058
:10042000B50300086023002058220020084B1870F4
:1004300003280CD8DFE800F008050208022000F0CD
:1004400005BC022000F0F0BB024B00225A6070474E
:100450005822002060230020244B254A10B51C465A
:100460001968013140D004339342F9D16268214BBD
:100470009A4239D9204B9B6803F1006303F580331E
:100480009A4231D2002000F033FB0220FFF7CEFF6A
:100490001A4B1A6C00221A64196E1A66196E596C7E
:1004A0005A64596E5A665A6E5A6942F080025A610D
:1004B0005A6922F080025A615A691A6942F0005260
:1004C0001A611A6922F000521A611B6972B64FF064
:1004D000E0233021C3F8084DD4E9003281F31188BC
:1004E0009D4683F30888104710BD00BF0000010837
:1004F00020000108FFFF0008002200200038024011
:100500002DE9F04F93B0AA4B00902022FF210AA8BA
:100510009D6800F0F7FBA74A1378A3B9A64801210C
:1005200003601170302383F3118803680BB101F06D
:1005300059FAA24AA04800234FF47A7101F048FA10
:10054000002383F31188009B13B19D4B009A1A601E
:100550009C4A009C1378032B1EBF00231370984AFB
:100560004FF0000A18BF5360D3465646D1460120CB
:1005700000F06CFB24B1924B1B68002B00F0118241
:10058000002000F06DFA0390039B002BF2DB0120AA
:1005900000F04AFB039B213B162BE8D801A252F83E
:1005A00023F000BF0106000829060008BD06000868
:1005B0006F0500086F0500086F0500084707000871
:1005C000170900083108000893080008BB08000854
:1005D000E10800086F050008F30800086F0500082F
:1005E00065090008A10600086F050008A9090008B0
:1005F0000D060008A10600086F0500089308000812
:100600000220FFF7C3FE002840F0F581009B022185
:10061000BAF1000F08BF1C4605A841F21233ADF82D
:10062000143000F03BFAA2E74FF47A7000F018FAA9
:10063000071EEBDB0220FFF7A9FE0028E6D0013FF2
:10064000052F00F2DA81DFE807F0030A0D101336F8
:1006500005230593042105A800F020FA17E054486B
:100660000421F9E758480421F6E758480421F3E744
:100670004FF01C08404600F03DFA08F104080590D0
:10068000042105A800F00AFAB8F12C0FF2D10120DC
:1006900000FA07F747EA0B0B5FFA8BFB4FF00009F4
:1006A00000F07CFB26B10BF00B030B2B08BF0024E2
:1006B000FFF774FE5BE746480421CDE7002EA5D086
:1006C0000BF00B030B2BA1D10220FFF75FFE0746B7
:1006D00000289BD0012000F00BFA0220FFF7A6FEB5
:1006E00000261FFA86F8404600F012FA044690B140
:1006F0000021404600F01CFA01360028F1D1BA462C
:10070000044641F21213022105A8ADF814303E460A
:1007100000F0C4F92BE70120FFF788FE2546244BA3
:100720009B68AB4207D9284600F0E4F9013040F05D
:1007300067810435F3E7234B00251D70204BBA4633
:100740005D603E46ACE7002E3FF460AF0BF00B035C
:100750000B2B7FF45BAF0220FFF768FE322000F026
:100760007FF9B0F10008FFF651AF18F003077FF4EE
:100770004DAF0F4A926808EB050393423FF646AF30
:10078000B8F5807F3FF742AF124B0193B84523DDA8
:100790004FF47A7000F064F90390039A002AFFF690
:1007A00035AF019B039A03F8012B0137EDE700BF3A
:1007B000002200205C23002040220020B503000816
:1007C000602300205822002004220020082200205C
:1007D0000C2200205C220020C820FFF7D7FD07462E
:1007E00000283FF413AF1F2D11D8C5F12002424558
:1007F0000AAB25F0030028BF424683490192184402
:1008000000F05AFA019A8048FF2100F07BFA4FEA83
:10081000A8037D490193C8F38702284600F07AFABD
:10082000064600283FF46DAF019B05EB830537E7D3
:100830000220FFF7ABFD00283FF4E8AE00F0A4F97A
:1008400000283FF4E3AE0027B846704B9B68BB42DC
:1008500018D91F2F11D80A9B01330ED027F003039C
:1008600012AA134453F8203C05934046042205A9DC
:1008700000F0C8FA04378046E7E7384600F03AF956
:100880000590F2E7CDF81480042105A800F006F9E0
:1008900006E70023642104A8049300F0F5F800287B
:1008A0007FF4B4AE0220FFF771FD00283FF4AEAE36
:1008B000049800F051F90590E6E70023642104A8AC
:1008C000049300F0E1F800287FF4A0AE0220FFF7C7
:1008D0005DFD00283FF49AAE049800F04DF9EAE778
:1008E0000220FFF753FD00283FF490AE00F05CF9C2
:1008F000E1E70220FFF74AFD00283FF487AE05A993
:10090000142000F057F904210746049004A800F0D1
:10091000C5F83946B9E7322000F0A2F8071EFFF605
:1009200075AEBB077FF472AE384A926807EB0903D5
:1009300093423FF66BAE0220FFF728FD00283FF4FC
:1009400065AE27F003074F44B9453FF4A9AE4846CA
:1009500000F0D0F80421059005A800F09FF809F1F7
:100960000409F1E74FF47A70FFF710FD00283FF417
:100970004DAE00F009F9002844D00A9B01330BD09A
:1009800008220AA9002000F0C5F900283AD0202248
:10099000FF210AA800F0B6F9FFF700FD1C4800F09F
:1009A0005BFF13B0BDE8F08F002E3FF42FAE0BF0CD
:1009B0000B030B2B7FF42AAE0023642105A80593BB
:1009C00000F062F8074600287FF420AE0220FFF70F
:1009D000DDFC804600283FF419AEFFF7DFFC41F252
:1009E000883000F039FF059800F00AFA464600F01A
:1009F000D5F93C46BBE5064652E64FF0000905E650
:100A0000BA467EE637467CE65C22002000220020C3
:100A1000A086010070B50F4B1B780133DBB2012BB0
:100A20000C4611D80C4D29684FF47A730E6AA2FB5C
:100A30000332014622462846B047844204D1074B80
:100A400000221A70012070BD4FF4FA7000F004FF0C
:100A50000020F8E710220020082600209423002020
:100A600007B50023024601210DF107008DF807307C
:100A7000FFF7D0FF20B19DF8070003B05DF804FB3D
:100A80004FF0FF30F9E700000A4608B50421FFF7F0
:100A9000C1FF80F00100C0B2404208BD30B4054C37
:100AA0002368DD69044B0A46AC460146204630BC4B
:100AB000604700BF08260020A086010070B501F045
:100AC000EBF9094E094D30800024286833888342B1
:100AD00008D901F0DBF92B6804440133B4F5803FF9
:100AE0002B60F2D370BD00BF962300206823002046
:100AF00001F080BA00F1006000F5803000687047B6
:100B000000F10060920000F5803001F00BBA0000A7
:100B1000054B1A68054B1B889B1A834202D9104467
:100B200001F0B4B90020704768230020962300200C
:100B300038B5084D044629B128682044BDE838403E
:100B400001F0C4B92868204401F0A8F90028F3D0C6
:100B500038BD00BF6823002010F003030AD1B0F5B0
:100B6000047F05D200F10050A0F51040D0F8003805
:100B7000184670470023FBE700F10050A0F5104035
:100B8000D0F8100A70470000064991F8243033B1BC
:100B90000023086A81F824300822FFF7B1BF012042
:100BA000704700BF6C230020014B1868704700BFDE
:100BB000002004E070B5194B1D68194B0138C5F3CE
:100BC0000B0408442D0C04221E88A6420BD15C683D
:100BD0000A46013C824213460FD214F9016F4EB10E
:100BE00002F8016BF6E7013A03F10803ECD1814208
:100BF0000B4602D22C2203F8012B0A4A0524168840
:100C0000AE4204D1984284BF967803F8016B013C50
:100C100002F10402F3D1581A70BD00BF002004E0B5
:100C2000D0340008BC340008022804D1054B4FF032
:100C300000729A6170470128FCD1034B4FF080424B
:100C4000F7E700BF0004024000000240022804D180
:100C5000054B4FF400729A6170470128FCD1034B99
:100C60004FF48042F7E700BF00040240000002405A
:100C7000022805D1064A536983F400735361704713
:100C80000128FCD1034A536983F48043F6E700BF8F
:100C9000000402400000024070B504464FF47A762A
:100CA0004CB1412C254628BF412506FB05F000F03C
:100CB000D3FD641BF4E770BD10B50023934203D04D
:100CC000CC5CC4540133F9E710BD000010B5013805
:100CD00010F9013F3BB191F900409C4203D11AB198
:100CE0000131013AF4E71AB191F90020981A10BDC8
:100CF0001046FCE703460246D01A12F9011B0029F0
:100D0000FAD1704702440346934202D003F8011B14
:100D1000FAE770472DE9F8431F4D144695F8242053
:100D20000746884652BBDFF870909CB395F8243094
:100D30002BB92022FF2148462F62FFF7E3FF95F8E9
:100D40002400C0F10802A24228BF2246D6B2414682
:100D5000920005EB8000FFF7AFFF95F82430A41B4D
:100D60001E44F6B2082E17449044E4B285F824607D
:100D7000DBD1FFF709FF0028D7D108E02B6A03EB8E
:100D800082038342CFD0FFF7FFFE0028CBD10020A3
:100D9000BDE8F8830120FBE76C230020024B1A78A2
:100DA000024B1A70704700BF9423002010220020CD
:100DB00010B5104C104800F0B5F821460E4800F070
:100DC000DDF82468626DD2F8043843F00203C2F8FB
:100DD00004384FF47A70FFF75FFF0849204600F0AF
:100DE000D3F9626DD2F8043823F00203C2F8043854
:100DF00010BD00BF9C35000808260020A43500085F
:100E00007047000030B5094D0A4491420DD011F8E9
:100E1000013B5840082340F30004013B2C4013F0F1
:100E2000FF0384EA5000F6D1EFE730BD2083B8ED30
:100E3000026843681143016003B11847704700001E
:100E400013B5446BD4F894341A681178042915D179
:100E5000217C022912D11979128901238B40134276
:100E60000CD101A904F14C0001F0F8FED4F894442F
:100E7000019B21790246206800F0D0F902B010BD34
:100E8000143001F07BBE00004FF0FF33143001F04E
:100E900075BE00004C3001F04DBF00004FF0FF3335
:100EA0004C3001F047BF0000143001F049BE000093
:100EB0004FF0FF31143001F043BE00004C3001F020
:100EC00019BF00004FF0FF324C3001F013BF00009B
:100ED0000020704710B5D0F894341A6811780429AE
:100EE000044617D1017C022914D159795289012372
:100EF0008B4013420ED1143001F0DCFD024648B1A4
:100F0000D4F894444FF4807361792068BDE81040B0
:100F100000F072B910BD0000406BFFF7DBBF0000AE
:100F2000704700007FB5124B036000234360C0E9A7
:100F30000233012502260F4B0574044602900193EB
:100F400000F18402294600964FF48073143001F0BA
:100F50008DFD094B0294CDE9006304F523724FF433
:100F60008073294604F14C0001F054FE04B070BDBA
:100F7000F0340008190F0008410E00080B683022F9
:100F800082F311880A7903EB820290614A7909326F
:100F900043F822008A7912B103EB8203986102239D
:100FA000C0F894140374002080F311887047000087
:100FB00038B5037F044613B190F85430ABB9201D07
:100FC00001250221FFF734FF04F1140025776FF0AB
:100FD000010100F069FC84F8545004F14C006FF0FA
:100FE0000101BDE8384000F05FBC38BD10B50121FB
:100FF00004460430FFF71CFF0023237784F85430A5
:1010000010BD000038B504460025143001F046FD3F
:1010100004F14C00257701F015FE201D84F8545092
:101020000121FFF705FF2046BDE83840FFF752BF1A
:1010300090F8443003F06003202B07D190F845204E
:10104000212A4FF0000303D81F2A06D8002070473A
:10105000222AFBD1C0E90E3303E0034A8263072250
:10106000C2630364012070471122002037B5D0F815
:1010700094341A681178042904461AD1017C022993
:1010800017D11979128901238B40134211D100F134
:101090004C05284601F096FE58B101A9284601F0FA
:1010A000DDFDD4F89444019B21790246206800F0CC
:1010B000B5F803B030BD0000F0B500EB810385B09A
:1010C0009E6904460D46FEB1302383F3118804EB7C
:1010D0008507301D0821FFF7ABFEFB685B691B68C5
:1010E00006F14C001BB1019001F0C6FD019803A967
:1010F00001F0B4FD024648B1039B2946204600F0AA
:101100008DF8002383F3118805B0F0BDFB685A69A0
:101110001268002AF5D01B8A013B1340F1D104F17B
:101120004402EAE7093138B550F82140DCB13023F8
:1011300083F31188D4F894241368527903EB820363
:10114000DB689B695D6845B104216018FFF770FE9C
:10115000294604F1140001F0B7FC2046FFF7BAFE5F
:10116000002383F3118838BD7047000001F016B8E2
:10117000012303700023C0E90133C361836203626A
:10118000C36243620363704738B50446302383F378
:1011900011880025C0E90355C0E90555416001F0FB
:1011A0000DF80223237085F31188284638BD00000E
:1011B00070B500EB810305465069DA600E461446AF
:1011C00018B110220021FFF79DFDA06918B110226F
:1011D0000021FFF797FD31462846BDE8704001F039
:1011E000B7B80000826802F0011282600022C0E9F4
:1011F0000422826101F038B9F0B400EB8104478920
:10120000E4680125A4698D403D43458123600023A6
:10121000A2606360F0BC01F053B90000F0B400EBD1
:1012200081040789E468012564698D403D43058197
:1012300023600023A2606360F0BC01F0CDB9000020
:1012400070B50223002504460370C0E90255C0E9C9
:101250000455C564856180F8345001F015F8636861
:101260001B6823B129462046BDE87040184770BD71
:101270000378052B10B504460AD080F850300523BA
:10128000037043681B680BB1042198470023A360D7
:1012900010BD00000178052906D190F85020436860
:1012A00002701B6803B118477047000070B590F8D2
:1012B0003430044613B1002380F8343004F1440282
:1012C000204601F0F3F863689B68B3B994F84430A2
:1012D00013F0600535D00021204601F093FB00217A
:1012E000204601F085FB63681B6813B10621204688
:1012F0009847062384F8343070BD2046984700286C
:10130000E4D0B4F84A30E26B9A4288BFE36394F9C0
:101310004430E56B002B4FF0300380F20381002D49
:1013200000F0F280092284F8342083F31188002130
:10133000D4E90E232046FFF771FF002383F31188C1
:10134000DAE794F8452003F07F0343EA022340F2F2
:101350000232934200F0C58021D8B3F5807F48D097
:101360000DD8012B3FD0022B00F09380002BB2D17F
:1013700004F14C02A2630222E2632364C1E7B3F5E5
:10138000817F00F09B80B3F5407FA4D194F8463074
:10139000012BA0D1B4F84C3043F0020332E0B3F596
:1013A000006F4DD017D8B3F5A06F31D0A3F5C0634F
:1013B000012B90D8636894F846205E6894F8471033
:1013C000B4F848302046B047002884D04368A3636F
:1013D0000368E3631AE0B3F5106F36D040F60242BB
:1013E00093427FF478AF5C4BA3630223E363002353
:1013F000C3E794F84630012B7FF46DAFB4F84C305E
:1014000023F00203C4E90E55A4F84C30256478E7B4
:10141000B4F84430B3F5A06F0ED194F8463084F898
:101420004E30204600F088FF63681B6813B101212D
:1014300020469847032323700023C4E90E339CE71A
:1014400004F14F03A3630123C3E72378042B10D1D6
:10145000302383F311882046FFF7C4FE85F31188FB
:101460000321636884F84F5021701B680BB120463C
:10147000984794F84630002BDED084F84F30042390
:10148000237063681B68002BD6D002212046984742
:10149000D2E794F848301D0603F00F0120460AD524
:1014A00000F0F6FF012804D002287FF414AF2B4B84
:1014B0009AE72B4B98E700F0DDFFF3E794F846300E
:1014C000002B7FF408AF94F8483013F00F01B3D02D
:1014D0001A06204602D501F0A9FAADE701F09CFA00
:1014E000AAE794F84630002B7FF4F5AE94F8483024
:1014F00013F00F01A0D01B06204602D501F082FA9E
:101500009AE701F075FA97E7142284F8342083F300
:1015100011882B462A4629462046FFF76DFE85F3A3
:101520001188E9E65DB1152284F8342083F311882F
:101530000021D4E90E232046FFF75EFEFDE60B22D4
:1015400084F8342083F311882B462A462946204606
:10155000FFF764FEE3E700BF2035000818350008F8
:101560001C35000838B590F834300446002B3ED0C6
:10157000063BDAB20F2A34D80F2B32D8DFE803F05B
:101580003731310822323131313131313131373770
:10159000C56BB0F84A309D4214D2C3681B8AB5FBB4
:1015A000F3F203FB12556DB9302383F311882B46F8
:1015B0002A462946FFF732FE85F311880A2384F86C
:1015C00034300EE0142384F83430302383F3118850
:1015D00000231A4619462046FFF70EFE002383F328
:1015E000118838BD036C03B198470023E7E7002159
:1015F000204601F007FA0021204601F0F9F963685E
:101600001B6813B10621204698470623D7E7000040
:1016100010B590F83430142B044629D017D8062B77
:1016200005D001D81BB110BD093B022BFBD800210E
:10163000204601F0E7F90021204601F0D9F963685E
:101640001B6813B1062120469847062319E0152B85
:10165000E9D10B2380F83430302383F31188002341
:101660001A461946FFF7DAFD002383F31188DAE7FB
:10167000C3689B695B68002BD5D1036C03B19847A5
:10168000002384F83430CEE70023037582680369B1
:101690001B6899689142FBD25A68036042601060EF
:1016A0005860704700230375826803691B68996856
:1016B0009142FBD85A6803604260106058607047DE
:1016C00008B50846302383F311880B7D032B05D022
:1016D000042B0DD02BB983F3118808BD8B69002230
:1016E0001A604FF0FF338361FFF7CEFF0023F2E76C
:1016F000D1E9003213605A60F3E70000FFF7C4BF7E
:10170000054BD9680875186802681A605360012291
:101710000275D860FEF7F6BD9823002030B50C4B5B
:10172000DD684B1C87B004460FD02B46094A68463B
:1017300000F04EF92046FFF7E3FF009B13B1684627
:1017400000F050F9A86907B030BDFFF7D9FFF9E7FD
:1017500098230020C1160008044B1A68DB689068C3
:101760009B68984294BF0020012070479823002076
:10177000084B10B51C68D86822681A6053600122B3
:101780002275DC60FFF78EFF01462046BDE8104061
:10179000FEF7B8BD9823002038B5074C0749084824
:1017A000012300252370656001F044FB02232370B0
:1017B00085F3118838BD00BF0026002028350008B9
:1017C0009823002000F044B9034A516853685B1A1B
:1017D0009842FBD8704700BF001000E08B600223E6
:1017E00008618B82084670478368A3F1840243F83E
:1017F000142C026943F8442C426943F8402C094AEE
:1018000043F8242CC26843F8182C022203F80C2C4D
:10181000002203F80B2C044A43F8102CA3F12000FB
:10182000704700BF1D0300089823002008B5FFF78C
:10183000DBFFBDE80840FFF761BF0000024BDB683B
:1018400098610F20FFF75CBF98230020302383F3BB
:101850001188FFF7F3BF000008B50146302383F37A
:1018600011880820FFF75AFF002383F3118808BD71
:10187000064BDB6839B1426818605A6013604360F8
:101880000420FFF74BBF4FF0FF3070479823002034
:101890000368984206D01A68026050609961184641
:1018A000FFF72CBF7047000038B504460D4620688E
:1018B000844200D138BD036823605C608561FFF716
:1018C0001DFFF4E710B503689C68A2420CD85C6861
:1018D0008A600B604C602160596099688A1A9A602E
:1018E0004FF0FF33836010BD1B68121BECE7000054
:1018F0000A2938BF0A2170B504460D460A26601928
:1019000001F092FA01F07EFA041BA54203D8751C7F
:101910002E460446F3E70A2E04D9BDE870400120A4
:1019200001F0C8BA70BD0000F8B5144B0D46D9617E
:1019300003F1100141600A2A1969826038BF0A2246
:10194000016048601861A818144601F05FFA0A2780
:1019500001F058FA431BA342064606D37C1C281903
:1019600001F062FA27463546F2E70A2F04D9BDE8AE
:10197000F840012001F09EBAF8BD00BF9823002076
:10198000F8B506460D4601F03DFA0F4A134653F8E6
:10199000107F9F4206D12A4601463046BDE8F840F6
:1019A000FFF7C2BFD169BB68441A2C1928BF2C4667
:1019B000A34202D92946FFF79BFF2246314603483E
:1019C000BDE8F840FFF77EBF98230020A823002041
:1019D00010B4C0E9032300235DF8044B4361FFF713
:1019E000CFBF000010B5194C236998420DD0D0E943
:1019F0000032816813605A609A680A449A60002332
:101A000003604FF0FF33A36110BD2346026843F823
:101A1000102F53600022026022699A4203D1BDE870
:101A2000104001F0FBB9936881680B44936001F0AA
:101A3000E9F92269E1699268441AA242E4D91144A1
:101A4000BDE81040091AFFF753BF00BF98230020DC
:101A50002DE9F047DFF8BC8008F110072C4ED8F8CC
:101A6000105001F0CFF9D8F81C40AA68031B9A4225
:101A70003ED81444D5E900324FF00009C8F81C40A4
:101A800013605A60C5F80090D8F81030B34201D105
:101A900001F0C4F989F31188D5E903312846984744
:101AA000302383F311886B69002BD8D001F0AAF999
:101AB0006A69A0EB04094A4582460DD2022001F072
:101AC000F9F90022D8F81030B34208D1514628461F
:101AD000BDE8F047FFF728BF121A2244F2E712EBE5
:101AE000090938BF4A4629463846FFF7EBFEB5E7F5
:101AF000D8F81030B34208D01444211AC8F81C009A
:101B0000A960BDE8F047FFF7F3BEBDE8F08700BF6E
:101B1000A82300209823002000207047FEE7000043
:101B2000704700004FF0FF307047000002290CD0D2
:101B3000032904D00129074818BF00207047032A51
:101B400005D8054800EBC2007047044870470020E4
:101B5000704700BF0036000820220020B43500087E
:101B600070B59AB00546084601A9144600F0C2F8BF
:101B700001A8FFF7BFF8431C5B00C5E90034002251
:101B8000237003236370C6B201AB02341046D1B296
:101B90008E4204F1020401D81AB070BD13F8011B83
:101BA00004F8021C04F8010C0132F0E708B53023F8
:101BB00083F311880348FFF759FA002383F3118850
:101BC00008BD00BF0826002090F8443003F01F0233
:101BD000012A07D190F845200B2A03D10023C0E940
:101BE0000E3315E003F06003202B08D1B0F8483025
:101BF0002BB990F84520212A03D81F2A04D8FFF7D3
:101C000017BA222AEBD0FAE7034A82630722C2639B
:101C100003640120704700BF1822002007B5052982
:101C200017D8DFE801F0191603191920302383F3C0
:101C30001188104A01900121FFF7BAFA01980E4A63
:101C40000221FFF7B5FA0D48FFF7DCF9002383F313
:101C5000118803B05DF804FB302383F31188074833
:101C6000FFF7A6F9F2E7302383F311880348FFF763
:101C7000BDF9EBE754350008783500080826002048
:101C800038B50C4D0C4C0D492A4604F10800FFF7FD
:101C900067FF05F1CA0204F110000949FFF760FF70
:101CA00005F5CA7204F118000649BDE83840FFF78F
:101CB00057BF00BFD02A0020202200203435000862
:101CC0003E3500084935000870B5044608460D4603
:101CD000FFF710F8C6B22046013403780BB9184656
:101CE00070BD32462946FEF7F1FF0028F3D10120EE
:101CF000F6E700002DE9F04705460C46FEF7FAFF2F
:101D00002B49C6B22846FFF7DFFF08B10636F6B208
:101D100028492846FFF7D8FF08B11036F6B2632EDF
:101D20000BD8DFF88C80DFF88C90234FDFF894A07D
:101D30002E7846B92670BDE8F08729462046BDE8D2
:101D4000F04701F09DBB252E2ED1072241462846A3
:101D5000FEF7BCFF70B9194B224603F10C0153F892
:101D6000040B42F8040B8B42F9D11B781370073532
:101D70000D34DDE7082249462846FEF7A7FF98B94B
:101D80000F4BA21C197809090232C95D02F8041C24
:101D900013F8011B01F00F015345C95D02F8031C44
:101DA000F0D118340835C3E704F8016B0135BFE7FB
:101DB0002036000849350008363600082836000865
:101DC000107AFF1F1C7AFF1FBFF34F8F024AD368A0
:101DD000DB03FCD4704700BF003C024008B5094B50
:101DE0001B7873B9FFF7F0FF074B1A69002ABFBFD2
:101DF000064A5A6002F188325A601A6822F48062F8
:101E00001A6008BD2E2D0020003C024023016745CA
:101E100008B50B4B1B7893B9FFF7D6FF094B1A692E
:101E200042F000421A611A6842F480521A601A683D
:101E300022F480521A601A6842F480621A6008BD67
:101E40002E2D0020003C02400B28F0B516D80C4C7B
:101E50000C4923787BB90C4D0E460C234FF00062E1
:101E600055F8047B46F8042B013B13F0FF033A447A
:101E7000F6D10123237051F82000F0BD0020FCE7CB
:101E8000602D0020302D002048360008014B53F80B
:101E900020007047483600080C2070470B2810B50A
:101EA000044601D9002010BDFFF7CEFF064B53F8C2
:101EB00024301844C21A0BB90120F4E71268013229
:101EC000F0D1043BF6E700BF483600080B2810B5F8
:101ED000044621D8FFF778FFFFF780FF0F4AF3236E
:101EE000D360C300DBB243F4007343F00203136119
:101EF000136943F480331361FFF766FFFFF7A4FF14
:101F0000074B53F8241000F0D9F8FFF781FF204663
:101F1000BDE81040FFF7C2BF002010BD003C0240EA
:101F200048360008F8B512F00103144642D1821871
:101F3000B2F1016F57D82D4B1B6813F0010352D03B
:101F40002B4DFFF74BFFF323EB60FFF73DFF40F214
:101F50000127032C15D824F001046618244C401ADC
:101F600040F20117B142236900EB010524D123F0AF
:101F700001032361FFF74CFF0120F8BD043C04304E
:101F8000E7E78307E7D12B6923F440732B612B69C3
:101F90003B432B6151F8046B0660BFF34F8FFFF793
:101FA00013FF03689E42E9D02B6923F001032B61E4
:101FB000FFF72EFF0020E0E723F44073236123693D
:101FC0003B4323610B882B80BFF34F8FFFF7FCFE51
:101FD0002D8831F8023BADB2AB42C3D0236923F068
:101FE00001032361E4E71846C7E700BF0038024059
:101FF000003C0240084908B50B7828B11BB9FFF72F
:10200000EDFE01230B7008BD002BFCD0BDE808409D
:102010000870FFF7FDBE00BF2E2D002010B5024452
:10202000064BD2B2904200D110BD441C00B253F80E
:10203000200041F8040BE0B2F4E700BF5028004054
:102040000F4B30B51C6F240407D41C6F44F400748C
:102050001C671C6F44F400441C670A4C236843F45B
:10206000807323600244084BD2B2904200D130BD4D
:10207000441C00B251F8045B43F82050E0B2F4E78E
:1020800000380240007000405028004007B501228F
:1020900001A90020FFF7C2FF019803B05DF804FB1F
:1020A00013B50446FFF7F2FFA04205D0012201A9B3
:1020B00000200194FFF7C4FF02B010BD704700007C
:1020C000034B1A681AB9034AD2F874281A60704789
:1020D000642D00200030024008B5FFF7F1FF024BED
:1020E0001868C0F3407008BD642D002070470000E0
:1020F000FEE700000A4B0B480B4A90420BD30B4BF8
:10210000DA1C121AC11E22F003028B4238BF0022D1
:102110000021FEF7F7BD53F8041B40F8041BECE761
:10212000F0370008602E0020602E0020602E002076
:1021300070B5D0E915439E6800224FF0FF3504EBDF
:1021400042135101D3F800090028BEBFD3F800099B
:1021500040F08040C3F80009D3F8000B0028BEBF50
:10216000D3F8000B40F08040C3F8000B0132631835
:102170009642C3F80859C3F8085BE0D24FF0011348
:10218000C4F81C3870BD0000890141F020010161D4
:1021900003699B06FCD41220FFF716BB10B5054C53
:1021A0002046FEF7E5FF4FF0A0436365024BA365B1
:1021B00010BD00BF682D00209C36000870B5037864
:1021C000012B054650D12A4B446D98421BD1294B17
:1021D0005A6B42F080025A635A6D42F080025A658F
:1021E0005A6D5A6942F080025A615A6922F080029F
:1021F0005A610E2143205B6900F022FC1E4BE36014
:102200001E4BC4F800380023C4F8003EC0232360EE
:102210006E6D4FF40413A3633369002BFCDA0123C2
:1022200033610C20FFF7D0FA3369DB07FCD41220AE
:10223000FFF7CAFA3369002BFCDA0026A6602846AD
:10224000FFF776FF6B68C4F81068DB68C4F81468A1
:10225000C4F81C684BB90A4BA3614FF0FF336361AC
:10226000A36843F00103A36070BD064BF4E700BF11
:10227000682D002000380240401400400300200276
:10228000003C30C0083C30C0F8B5446D0546002124
:102290002046FFF779FFA96D00234FF001128F68E8
:1022A000C4F834384FF00066C4F81C284FF0FF30F3
:1022B00004EB431201339F42C2F80069C2F8006B7D
:1022C000C2F80809C2F8080BF2D20B686A6DEB6518
:1022D000636210231361166916F01006FBD11220F9
:1022E000FFF772FAD4F8003823F4FE63C4F800381C
:1022F000A36943F4402343F01003A3610923C4F806
:102300001038C4F814380A4BEB604FF0C043C4F8DF
:10231000103B084BC4F8003BC4F81069C4F80039FE
:10232000EB6D03F1100243F48013EA65A362F8BD7C
:102330007836000840800010426D90F84E10D2F8B8
:10234000003823F4FE6343EA0113C2F800387047F3
:102350002DE9F84300EB8103456DDA68166806F055
:102360000306731E022B05EB41130C4680460FFA41
:1023700081F94FEA41104FF00001C3F8101B4FF0F4
:10238000010104F1100398BFB60401FA03F3916947
:102390008EBF334E06F1805606F5004600293AD02E
:1023A000578A04F15801490137436F50D5F81C187A
:1023B0000B43C5F81C382B180021C3F810195369BA
:1023C0000127611EA7409BB3138A928B9B08012AA9
:1023D00088BF5343D8F85C20981842EA034301F1C0
:1023E000400205EB8202C8F85C0021465360284693
:1023F000FFF7CAFE08EB8900C3681B8A43EA8453CF
:10240000483464011E432E51D5F81C381F43C5F8CB
:102410001C78BDE8F88305EB4917D7F8001B21F4B9
:102420000041C7F8001BD5F81C1821EA0303C0E7D8
:1024300004F13F0305EB83030A4A5A60284621460C
:10244000FFF7A2FE05EB4910D0F8003923F4004352
:10245000C0F80039D5F81C3823EA0707D7E700BFD2
:102460000080001000040002826D1268C265FFF750
:102470005FBE00005831436D49015B5813F40040C2
:1024800004D013F4001F0CBF02200120704700008D
:102490004831436D49015B5813F4004004D013F4F4
:1024A000001F0CBF022001207047000000EB8101DB
:1024B000CB68196A0B6813604B6853607047000063
:1024C00000EB810330B5DD68AA691368D36019B9E0
:1024D000402B84BF402313606B8A1468426D1C44F8
:1024E000013CB4FBF3F46343033323F0030302EB37
:1024F000411043EAC44343F0C043C0F8103B2B688B
:1025000003F00303012B09B20ED1D2F8083802EB15
:10251000411013F4807FD0F8003B14BF43F0805388
:1025200043F00053C0F8003B02EB4112D2F8003BED
:1025300043F00443C2F8003B30BD00002DE9F041F8
:10254000244D6E6D06EB40130446D3F8087BC3F8A8
:10255000087B38070AD5D6F81438190706D505EBD5
:1025600084032146DB6828465B689847FA071FD535
:10257000D6F81438DB071BD505EB8403D968CCB932
:102580008B69488A5A68B2FBF0F600FB16228AB9BA
:102590001868DA6890420DD2121AC3E90024302379
:1025A00083F311880B482146FFF78AFF84F31188D3
:1025B000BDE8F081012303FA04F26B8923EA0203E8
:1025C0006B81CB68002BF3D021460248BDE8F04177
:1025D000184700BF682D002000EB810370B5DD684F
:1025E000436D6C692668E6604A0156BB1A444FF495
:1025F0000020C2F810092A6802F00302012A0AB278
:102600000ED1D3F8080803EB421410F4807FD4F8FD
:10261000000914BF40F0805040F00050C4F8000999
:1026200003EB4212D2F8000940F00440C2F800095E
:10263000D3F83408012202FA01F10143C3F8341837
:1026400070BD19B9402E84BF4020206020682E8ABA
:102650008419013CB4FBF6F440EAC44040F0005059
:102660001A44C6E72DE9F8433B4D6E6D06EB401367
:102670000446D3F80889C3F8088918F0010F4FEA17
:1026800040171AD0D6F81038DB0716D505EB8003B3
:10269000D9684B691868DA68904230D2121A4FF044
:1026A00000091A60C3F80490302383F3118821468F
:1026B0002846FFF791FF89F3118818F0800F1CD08E
:1026C000D6F834380126A640334216D005EB8403F1
:1026D0006D6DD3F80CC0DCF814200134E4B2D2F8EC
:1026E00000E005EB04342F445168714515D3D5F84B
:1026F000343823EA0606C5F83468BDE8F8830123B8
:1027000003FA04F22B8923EA02032B818B68002B46
:10271000D3D0214628469847CFE7BCF81000AEEB4F
:102720000103834228BF0346D7F8180980B2B3EBF0
:10273000800FE2D89068A0F1040959F8048FC4F81A
:102740000080A0EB09089844B8F1040FF5D81844AC
:102750000B4490605360C7E7682D00202DE9F74FC8
:10276000A24C656D6E69AB691E4016F480586E61AF
:1027700007D02046FEF764FD03B0BDE8F04F00F03F
:1027800047BC002E12DAD5F8003E98489B071EBFC2
:10279000D5F8003E23F00303C5F8003ED5F8043811
:1027A00023F00103C5F80438FEF774FD370505D59D
:1027B0008E48FFF7BDFC8D48FEF75AFDB0040CD5DE
:1027C000D5F8083813F0060FEB6823F470530CBFEC
:1027D00043F4105343F4A053EB6031071BD56368F7
:1027E000DB681BB9AB6923F00803AB612378052BC9
:1027F0000CD1D5F8003E7D489A071EBFD5F8003EA3
:1028000023F00303C5F8003EFEF744FD6368DB6870
:102810000BB176489847F30274D4B70227D5D4F8A1
:102820005490DFF8C8B100274FF0010A09EB4712B6
:10283000D2F8003B03F44023B3F5802F11D1D2F836
:10284000003B002B0DDA62890AFA07F322EA030340
:10285000638104EB8703DB68DB6813B139465846B4
:102860009847A36D01379B68FFB29F42DED9F006FF
:1028700017D5676D3A6AC2F30A1002F00F0302F42B
:10288000F012B2F5802F00F08580B2F5402F08D10C
:1028900004EB83030022DB681B6A07F58057904234
:1028A0006AD13003D5F8184813D5E10302D50020CA
:1028B000FFF744FEA20302D50120FFF73FFE6303AA
:1028C00002D50220FFF73AFE270302D50320FFF7C7
:1028D00035FE75037FF550AFE00702D50020FFF706
:1028E000C1FEA10702D50120FFF7BCFE620702D599
:1028F0000220FFF7B7FE23077FF53EAF0320FFF767
:10290000B1FE39E7636DDFF8E4A0019300274FF0D3
:102910000109A36D9B685FFA87FB9B453FF67DAF7E
:10292000019B03EB4B13D3F8001901F44021B1F5DF
:10293000802F1FD1D3F8001900291BDAD3F8001912
:1029400041F09041C3F80019D3F800190029FBDBCE
:102950005946606DFFF718FC218909FA0BF321EA4B
:102960000303238104EB8B03DB689B6813B1594697
:10297000504698470137CCE7910708BFD7F8008049
:10298000072A98BF03F8018B02F1010298BF4FEAB2
:10299000182884E7023304EB830207F58057526856
:1029A000D2F818C0DCF80820DCE9001CA1EB0C0C04
:1029B000002188420AD104EB830463689B699A680A
:1029C00002449A605A6802445A606AE711F0030FA1
:1029D00008BFD7F800808C4588BF02F8018B01F151
:1029E000010188BF4FEA1828E3E700BF682D0020E7
:1029F000436D03EB4111D1F8003B43F40013C1F8E0
:102A0000003B7047436D03EB4111D1F8003943F4AB
:102A10000013C1F800397047436D03EB4111D1F841
:102A2000003B23F40013C1F8003B7047436D03EBF8
:102A30004111D1F8003923F40013C1F8003970476F
:102A400000F1604303F561430901C9B283F8001343
:102A5000012200F01F039A4043099B0003F16043E9
:102A600003F56143C3F880211A60704730B5039CB9
:102A70000172043304FB0325C0E90653049B03637E
:102A80000021059BC160C0E90000C0E90422C0E943
:102A90000842C0E90A11436330BD0000416A0022C8
:102AA000C0E90411C0E90A22C2606FF00101FEF71B
:102AB000FBBE0000D0E90432934201D1C2680AB9DA
:102AC000181D70470020704703691960C268013201
:102AD000C260C269134482690361934224BF436A9E
:102AE00003610021FEF7D4BE38B504460D46E36805
:102AF0003BB16269131D1268A3621344E3620020B4
:102B000007E0237A33B929462046FEF7B1FE0028B4
:102B1000EDDA38BD6FF00100FBE70000C368C26961
:102B2000013BC3604369134482694361934224BFFC
:102B3000436A436100238362036B03B11847704704
:102B400070B53023044683F31188866A3EB9FFF7D7
:102B5000CBFF054618B186F31188284670BDA36ADD
:102B6000E26A13F8015BA362934202D32046FFF7A7
:102B7000D5FF002383F31188EFE700002DE9F84F1C
:102B800004460E46174698464FF0300989F31188DF
:102B90000025AA46D4F828B0BBF1000F09D1414660
:102BA0002046FFF7A1FF20B18BF311882846BDE82E
:102BB000F88FD4E90A12A7EB050B521A934528BFE8
:102BC0009346BBF1400F1BD9334601F1400251F847
:102BD000040B43F8040B9142F9D1A36A4033403609
:102BE000A3624035D4E90A239A4202D32046FFF774
:102BF00095FF8AF31188BD42D8D289F31188C9E7BD
:102C000030465A46FEF758F8A36A5B445E44A36216
:102C10005D44E7E710B5029C0172043303FB042115
:102C2000C0E906130023C0E90A33039B0363049B36
:102C3000C460C0E90000C0E90422C0E9084243635F
:102C400010BD0000026AC260426AC0E9042200228C
:102C5000C0E90A226FF00101FEF726BED0E9042385
:102C60009A4201D1C26822B9184650F8043B0B6061
:102C7000704700231846FAE7C368C2690133C3608E
:102C80004369134482694361934224BF436A4361A9
:102C90000021FEF7FDBD000038B504460D46E3688F
:102CA0003BB123691A1DA262E2691344E36200206A
:102CB00007E0237A33B929462046FEF7D9FD0028DC
:102CC000EDDA38BD6FF00100FBE700000369196021
:102CD000C268013AC260C2691344826903619342C7
:102CE00024BF436A036100238362036B03B1184767
:102CF0007047000070B530230D460446114683F33B
:102D00001188866A2EB9FFF7C7FF10B186F31188C4
:102D100070BDA36A1D70A36AE26A01339342A36285
:102D200004D3E16920460439FFF7D0FF002080F387
:102D30001188EDE72DE9F84F04460D469046994677
:102D40004FF0300A8AF311880026B346A76A4FB9BC
:102D500049462046FFF7A0FF20B187F3118830468F
:102D6000BDE8F88FD4E90A073A1AA8EB060797429C
:102D700028BF1746402F1BD905F1400355F8042BF7
:102D800040F8042B9D42F9D1A36A4033A362403638
:102D9000D4E90A239A4204D3E16920460439FFF7B3
:102DA00095FF8BF311884645D9D28AF31188CDE778
:102DB00029463A46FDF780FFA36A3B443D44A3629F
:102DC0003E44E5E7D0E904239A4217D1C3689BB19A
:102DD000836A8BB1043B9B1A0ED01360C368013B1E
:102DE000C360C3691A44836902619A4224BF436A7B
:102DF0000361002383620123184670470023FBE729
:102E000000F030B94FF08043586A70474FF080436C
:102E1000002258631A610222DA6070474FF0804343
:102E20000022DA60704700004FF08043586370471B
:102E3000FEE7000070B51B4B01630025044686B019
:102E4000586085620E4600F0BFF804F11003C4E933
:102E500004334FF0FF33C4E90635C4E90044A560EC
:102E6000E562FFF7CFFF2B460246C4E9082304F1D1
:102E700034010D4A256580232046FEF7AFFC01236F
:102E8000E0600A4A0375009272680192B268CDE967
:102E90000223074B6846CDE90435FEF7C7FC06B0B0
:102EA00070BD00BF00260020A8360008AD3600081F
:102EB000312E0008024AD36A1843D062704700BF1F
:102EC000982300204B6843608B688360CB68C360A5
:102ED0000B6943614B6903628B6943620B68036052
:102EE0007047000008B5264B26481A6940F2FF11CA
:102EF0000A431A611A6922F4FF7222F001021A6170
:102F00001A691A6B0A431A631A6D0A431A651E4A34
:102F10001B6D1146FFF7D6FF02F11C0100F5806022
:102F2000FFF7D0FF02F1380100F58060FFF7CAFF1C
:102F300002F1540100F58060FFF7C4FF02F1700157
:102F400000F58060FFF7BEFF02F18C0100F58060A4
:102F5000FFF7B8FF02F1A80100F58060FFF7B2FFAC
:102F600002F1C40100F58060FFF7ACFF02F1E0015F
:102F700000F58060FFF7A6FFBDE8084000F0EEB85E
:102F80000038024000000240B436000808B500F0E6
:102F900059FAFEF701FCFFF793F8BDE80840FEF789
:102FA0006FBE000070470000EFF3098305494A6BCC
:102FB00022F001024A63683383F30988002383F314
:102FC0001188704700EF00E0302080F3118862B66E
:102FD0000C4B0D4AD96821F4E0610904090C0A433D
:102FE000DA60D3F8FC20094942F08072C3F8FC2073
:102FF0000A6842F001020A602022DA7783F8220090
:10300000704700BF00ED00E00003FA05001000E08B
:1030100010B5302383F311880E4B5B6813F4006303
:1030200014D0F1EE103AEFF30984683C4FF080734E
:10303000E361094BDB6B236684F30988FEF78CFBA5
:1030400010B1064BA36110BD054BFBE783F311885C
:10305000F9E700BF00ED00E000EF00E02F030008FB
:10306000320300080F4B1A6C42F001021A641A6E08
:1030700042F001021A660C4A1B6E936843F001038A
:1030800093604FF0804353229A624FF0FF32DA622E
:1030900000229A615A63DA605A6001225A611A600A
:1030A000704700BF00380240002004E04FF080422B
:1030B00008B51169D3680B40D9B2C9439B071161A8
:1030C00007D5302383F31188FEF77CFB002383F3BD
:1030D000118808BD1F4B1A696FEAC2526FEAD252BB
:1030E0001A611A69C2F308021A614FF0FF301A69B7
:1030F0005A69586100215A6959615A691A6A62F01D
:1031000080521A621A6A02F080521A621A6A5A6A65
:1031100058625A6A59625A6A1A6C42F080521A64AA
:103120001A6E42F080521A661A6E0B4A106840F40A
:1031300080701060186F00F44070B0F5007F1EBF03
:103140004FF4803018671967536823F40073536095
:1031500000F054B90038024000700040334B4FF08B
:1031600080521A64324A4FF4404111601A6842F0AA
:1031700001021A601A689107FCD59A6822F00302CE
:103180009A602A4B9A6812F00C02FBD1196801F080
:10319000F90119609A601A6842F480321A601A685C
:1031A0009203FCD55A6F42F001025A671F4B5A6FC7
:1031B0009007FCD51F4A5A601A6842F080721A6064
:1031C0001B4A53685904FCD5184B1A689201FCD568
:1031D000194A9A60194B1A68194B9A42194B21D116
:1031E000194A1168194A91421CD140F205121A601D
:1031F000144A136803F00F03052BFAD10B4B9A689E
:1032000042F002029A609A6802F00C02082AFAD18F
:103210005A6C42F480425A645A6E42F480425A66B2
:103220005B6E704740F20572E1E700BF0038024074
:10323000007000400854400700948838002004E0E3
:1032400011640020003C024000ED00E041C20F414B
:10325000074A08B5536903F00103536123B1054AD6
:1032600013680BB150689847BDE80840FFF7D0BE1F
:10327000003C0140E02D0020074A08B5536903F0E7
:103280000203536123B1054A93680BB1D068984794
:10329000BDE80840FFF7BCBE003C0140E02D002027
:1032A000074A08B5536903F00403536123B1054A83
:1032B00013690BB150699847BDE80840FFF7A8BEF5
:1032C000003C0140E02D0020074A08B5536903F097
:1032D0000803536123B1054A93690BB1D06998473C
:1032E000BDE80840FFF794BE003C0140E02D0020FF
:1032F000074A08B5536903F01003536123B1054A27
:10330000136A0BB1506A9847BDE80840FFF780BECA
:10331000003C0140E02D0020164B10B55C6904F420
:1033200078725A61A30604D5134A936A0BB1D06A26
:103330009847600604D5104A136B0BB1506B984741
:10334000210604D50C4A936B0BB1D06B9847E2056C
:1033500004D5094A136C0BB1506C9847A30504D5EA
:10336000054A936C0BB1D06C9847BDE81040FFF74D
:103370004FBE00BF003C0140E02D0020194B10B5AE
:103380005C6904F47C425A61620504D5164A136DE7
:103390000BB1506D9847230504D5134A936D0BB1BB
:1033A000D06D9847E00404D50F4A136E0BB1506EF0
:1033B0009847A10404D50C4A936E0BB1D06E984780
:1033C000620404D5084A136F0BB1506F9847230469
:1033D00004D5054A936F0BB1D06F9847BDE81040F4
:1033E000FFF716BE003C0140E02D002008B5FFF7B6
:1033F0005DFEBDE80840FFF70BBE0000062108B5E2
:103400000846FFF71DFB06210720FFF719FB0621E1
:103410000820FFF715FB06210920FFF711FB062105
:103420000A20FFF70DFB06211720FFF709FB0621F5
:103430002820FFF705FBBDE8084007211C20FFF707
:10344000FFBA000008B5FFF745FE00F00BF8FDF7E6
:103450008DFEFDF765FDFFF7A5FDBDE80840FFF710
:10346000CFBC00000023054A19460133102BC2E9E6
:10347000001102F10802F8D1704700BFE02D0020D2
:10348000034611F8012B03F8012B002AF9D17047EC
:1034900053544D3332463F3F3F0053544D33324631
:1034A0003430780053544D3332463432780053541C
:1034B0004D33324634343658580000000120330072
:1034C0000010410001105A0003105900071031008C
:1034D0000000000090340008130400009A34000833
:1034E00019040000A434000821040000AE340008D0
:1034F000000000009D0E0008890E0008C50E00089F
:10350000B10E0008BD0E0008A90E0008950E0008B7
:10351000810E0008D10E000800000000010000002C
:10352000000000006330000024350008F023002074
:10353000002600204172647550696C6F740025424A
:103540004F415244252D424C002553455249414C90
:10355000250000000200000000000000B910000873
:103560002511000840004000A02A0020B02A0020B9
:103570000200000000000000030000000000000046
:10358000691100080000000010000000C02A00209F
:10359000000000000100000000000000682D002075
:1035A000010102001D1C00082D1B0008C91B00089A
:1035B000AD1B000843000000BC35000809024300B1
:1035C000020100C0320904000001020201000524CA
:1035D0000010010524010001042402020524060054
:1035E00001070582030800FF09040100020A000028
:1035F00000070501024000000705810240000000AD
:1036000012000000083600081201100102000040FC
:1036100009124157000201020301000004030904DA
:1036200025424F41524425004D6174656B4634304C
:10363000352D535444003031323334353637383930
:103640004142434445460000004000000040000065
:1036500000400000004000000000010000000200E7
:103660000000020000000200000002000000020052
:10367000000002000000020000000000AD1200087F
:10368000651500081116000840004000C82D0020F4
:10369000C82D002001000000D82D0020800000006F
:1036A00040010000030000006D61696E0069646CF8
:1036B000650000000000801200000000AAAAAAAA6B
:1036C00000000000FFBF00000000000000A00A0092
:1036D0000000140000000000AAAAAAAA000010001E
:1036E000FFFD0000000000000000000015000000C9
:1036F00000000000AAAAAAAA15000000FFFF00000F
:1037000000000000000000000000000000000000B9
:10371000AAAAAAAA00000000FFFF00000000000003
:10372000000000000000000000000000AAAAAAAAF1
:1037300000000000FFFF000000000000000000008B
:103740000000000000000000AAAAAAAA00000000D1
:10375000FFFF00000000000000000000000000006B
:1037600000000000AAAAAAAA00000000FFFF0000B3
:103770000000000000000000000000000000000049
:103780000A0000000000000003000000000000002C
:103790000000000000000000000000000000000029
:1037A0000000000000000000000000000000000019
:1037B0007D0000000000000000000F00000000007D
:1037C000FF009600000000080096000000000800BE
:1037D000040000001C36000800000000000000008B
:1037E00000000000000000000000000000000000D9
:1037F000FFFFFFFFFFFFFFFFFFFFFFFFFFFFFFFFD9
:10380000FFFFFFFFFFFFFFFFFFFFFFFFFFFFFFFFC8
:10381000FFFFFFFFFFFFFFFFFFFFFFFFFFFFFFFFB8
:020000040801F1
:10000000000600209912010815E4080871E30808A9
:10001000DDE3080871E30808A9E308089B1201085A
:100020009B1201089B1201089B120108897D0B0895
:100030009B1201089B1201089B1201089B120108E8
:100040009B1201089B1201089B1201089B120108D8
:100050009B1201089B12010821890B0849890B0892
:1000600071890B0899890B08C1890B08792D0B0838
:10007000A12D0B08CD2D0B08F92D0B08252E0B08F3
:100080004D2E0B08792E0B08FD2C0B089B12010836
:100090009B1201089B1201089B120108E9890B08B9
:1000A000218B0B08358B0B08498B0B084D8B0B08EC
:1000B000518B0B08658B0B08798B0B0805340B08EB
:1000C000AD350B089B1201089B1201089B12010819
:1000D0009B120108BD8A0B08D18A0B08E58A0B0820
:1000E0004D8A0B089B1201089B1201089D8B0B087F
:1000F000A18B0B08B58B0B08B98B0B08A52E0B0831
:100100009B1201089B1201088D8B0B089B120108A2
:10011000F98A0B080D8B0B089B1201089B12010832
:10012000D12E0B08F92E0B08252F0B08512F0B0889
:100130007D2F0B089B1201089B1201089B120108DE
:100140009B1201089B1201089B120108B5840B0841
:10015000A52F0B08D12F0B08FD2F0B089B120108B0
:100160009B1201089B1201089B1201089B120108B7
:100170009B1201089B1201089B1201089B120108A7
:100180009B1201089B1201089B1201089B12010897
:100190009B1201089B1201089B1201089B12010887
:1001A0009B1201089B1201089B1201089B12010877
:1001B0009B1201089B1201089B1201089B12010867
:1001C0009B1201089B1201089B1201089B12010857
:1001D0009B1201089B1201089B1201089B12010847
:1001E000213F01080D890108DD270208C991030894
:1001F0009553050811590508ADC805088D2C06084A
:100200005134060889370608BD9C060899BB0608C4
:1002100029720708599D0708B1AA0708BDD5080823
:10022000A1DA0808D9110A08416B0A0899910A084D
:10023000CD9C0A0831CC0A085DD20A0800000000F3
:1002400081F0004102E000BF83F0004330B54FEA87
:1002500041044FEA430594EA050F08BF90EA020FF4
:100260001FBF54EA000C55EA020C7FEA645C7FEA87
:10027000655C00F0E2804FEA5454D4EB5555B8BFAA
:100280006D420CDD2C4480EA020281EA030382EA1B
:10029000000083EA010180EA020281EA0303362DAD
:1002A00088BF30BD11F0004F4FEA01314FF4801C80
:1002B0004CEA113102D0404261EB410113F0004F92
:1002C0004FEA03334CEA133302D0524263EB430349
:1002D00094EA050F00F0A780A4F10104D5F1200EE7
:1002E0000DDB02FA0EFC22FA05F2801841F1000142
:1002F00003FA0EF2801843FA05F359410EE0A5F116
:1003000020050EF1200E012A03FA0EFC28BF4CF046
:10031000020C43FA05F3C01851EBE37101F00045FC
:1003200007D54FF0000EDCF1000C7EEB00006EEB09
:100330000101B1F5801F1BD3B1F5001F0CD3490893
:100340005FEA30004FEA3C0C04F101044FEA4452EA
:1003500012F5800F80F09A80BCF1004F08BF5FEA71
:10036000500C50F1000041EB045141EA050130BD51
:100370005FEA4C0C404141EB0101013C28BFB1F563
:10038000801FE9D291F0000F04BF01460020B1FAAE
:1003900081F308BF2033A3F10B03B3F120020CDA81
:1003A0000C3208DD02F1140CC2F10C0201FA0CF05F
:1003B00021FA02F10CE002F11402D8BFC2F1200CC4
:1003C00001FA02F120FA0CFCDCBF41EA0C0190407A
:1003D000E41AA2BF01EB0451294330BD6FEA0404C3
:1003E0001F3C1CDA0C340EDC04F11404C4F12002AE
:1003F00020FA04F001FA02F340EA030021FA04F3C0
:1004000045EA030130BDC4F10C04C4F1200220FA16
:1004100002F001FA04F340EA0300294630BD21FA54
:1004200004F0294630BD94F0000F83F4801306BF1A
:1004300081F480110134013D4EE77FEA645C18BF0E
:100440007FEA655C29D094EA050F08BF90EA020FA5
:1004500005D054EA000C04BF1946104630BD91EA9D
:10046000030F1EBF0021002030BD5FEA545C05D1A0
:100470004000494128BF41F0004130BD14F58004DF
:100480003CBF01F5801130BD01F0004545F0FE4153
:1004900041F470014FF0000030BD7FEA645C1ABF88
:1004A000194610467FEA655C1CBF0B46024650EABF
:1004B000013406BF52EA033591EA030F41F40021EB
:1004C00030BD00BF90F0000F04BF0021704730B571
:1004D0004FF4806404F132044FF000054FF0000146
:1004E00050E700BF90F0000F04BF0021704730B507
:1004F0004FF4806404F1320410F0004548BF4042DC
:100500004FF000013EE700BF42004FEAE2014FEA30
:1005100031014FEA02701FBF12F07F4393F07F4F0B
:1005200081F06051704732F07F4208BF704793F00E
:100530007F4F04BF41F40021704730B54FF4607421
:1005400001F0004521F000411CE700BF50EA010224
:1005500008BF704730B54FF000050AE050EA0102CD
:1005600008BF704730B511F0004502D5404261EB3D
:1005700041014FF4806404F132045FEA915C3FF47E
:10058000D8AE4FF003025FEADC0C18BF03325FEA1B
:10059000DC0C18BF033202EBDC02C2F1200300FACC
:1005A00003FC20FA02F001FA03FE40EA0E0021FAF1
:1005B00002F11444BDE600BF70B54FF0FF0C4CF4DF
:1005C000E06C1CEA11541DBF1CEA135594EA0C0F91
:1005D00095EA0C0F00F0DEF82C4481EA030621EACC
:1005E0004C5123EA4C5350EA013518BF52EA033507
:1005F00041F4801143F4801338D0A0FB02CE4FF0B9
:100600000005E1FB02E506F00042E0FB03E54FF0E8
:100610000006E1FB03569CF0000F18BF4EF0010EE0
:10062000A4F1FF04B6F5007F64F5407404D25FEADC
:100630004E0E6D4146EB060642EAC62141EA55518F
:100640004FEAC52040EA5E504FEACE2EB4F1FD0CD1
:1006500088BFBCF5E06F1ED8BEF1004F08BF5FEA4F
:10066000500E50F1000041EB045170BD06F0004601
:1006700046EA010140EA020081EA0301B4EB5C04AE
:10068000C2BFD4EB0C0541EA045170BD41F48011A6
:100690004FF0000E013C00F3AB8014F1360FDEBFCB
:1006A000002001F0004170BDC4F10004203C35DAA7
:1006B0000C341BDC04F11404C4F1200500FA05F32A
:1006C00020FA04F001FA05F240EA020001F00042CB
:1006D00021F0004110EBD37021FA04F642EB060141
:1006E0005EEA430E08BF20EAD37070BDC4F10C046B
:1006F000C4F1200500FA04F320FA05F001FA04F22F
:1007000040EA020001F0004110EBD37041F100011A
:100710005EEA430E08BF20EAD37070BDC4F1200525
:1007200000FA05F24EEA020E20FA04F301FA05F28D
:1007300043EA020321FA04F001F0004121FA04F235
:1007400020EA020000EBD3705EEA430E08BF20EA05
:10075000D37070BD94F0000F0FD101F0004640003F
:1007600041EB010111F4801F08BF013CF7D041EAC1
:10077000060195F0000F18BF704703F000465200C5
:1007800043EB030313F4801F08BF013DF7D043EA96
:100790000603704794EA0C0F0CEA135518BF95EA4C
:1007A0000C0F0CD050EA410618BF52EA4306D1D1D3
:1007B00081EA030101F000414FF0000070BD50EAF2
:1007C000410606BF1046194652EA430619D094EA7C
:1007D0000C0F02D150EA013613D195EA0C0F05D166
:1007E00052EA03361CBF104619460AD181EA0301BA
:1007F00001F0004141F0FE4141F470014FF0000072
:1008000070BD41F0FE4141F4780170BD70B54FF00C
:10081000FF0C4CF4E06C1CEA11541DBF1CEA13558C
:1008200094EA0C0F95EA0C0F00F0A7F8A4EB05046E
:1008300081EA030E52EA03354FEA013100F0888065
:100840004FEA03334FF0805545EA131343EA12632E
:100850004FEA022245EA111545EA10654FEA0026E3
:100860000EF000419D4208BF964244F1FD0404F59C
:10087000407402D25B084FEA3202B61A65EB0305F8
:100880005B084FEA32024FF480104FF4002CB6EBB5
:10089000020E75EB030E22BFB61A754640EA0C0035
:1008A0005B084FEA3202B6EB020E75EB030E22BF75
:1008B000B61A754640EA5C005B084FEA3202B6EBB6
:1008C000020E75EB030E22BFB61A754640EA9C0075
:1008D0005B084FEA3202B6EB020E75EB030E22BF45
:1008E000B61A754640EADC0055EA060E18D04FEA03
:1008F000051545EA16754FEA06164FEAC30343EAA3
:1009000052734FEAC2025FEA1C1CC0D111F4801F6F
:100910000BD141EA00014FF000004FF0004CB6E768
:1009200011F4801F04BF01430020B4F1FD0C88BF07
:10093000BCF5E06F3FF6AFAEB5EB030C04BFB6EB12
:10094000020C5FEA500C50F1000041EB045170BD05
:100950000EF0004E4EEA113114EB5C04C2BFD4EB32
:100960000C0541EA045170BD41F480114FF0000EB6
:10097000013C90E645EA060E8DE60CEA135594EA32
:100980000C0F08BF95EA0C0F3FF43BAF94EA0C0F35
:100990000AD150EA01347FF434AF95EA0C0F7FF4AA
:1009A00025AF104619462CE795EA0C0F06D152EAFE
:1009B00003353FF4FDAE1046194622E750EA4106E2
:1009C00018BF52EA43067FF4C5AE50EA41047FF4F3
:1009D0000DAF52EA43057FF4EBAE12E74FF0FF3C58
:1009E00006E000BF4FF0010C02E000BF4FF0010C29
:1009F0004DF804CD4FEA410C7FEA6C5C4FEA430CA2
:100A000018BF7FEA6C5C1BD001B050EA410C0CBFF0
:100A100052EA430C91EA030F02BF90EA020F002052
:100A2000704710F1000F91EA030F58BF994208BFB9
:100A300090422CBFD8176FEAE37040F00100704776
:100A40004FEA410C7FEA6C5C02D150EA013C07D1CD
:100A50004FEA430C7FEA6C5CD6D152EA033CD3D018
:100A60005DF8040B704700BF8446104662468C4612
:100A70001946634600E000BF01B5FFF7B7FF002845
:100A800048BF10F1000F01BD4DF808EDFFF7F4FF6E
:100A90000CBF012000205DF808FB00BF4DF808EDF9
:100AA000FFF7EAFF34BF012000205DF808FB00BF1C
:100AB0004DF808EDFFF7E0FF94BF012000205DF83E
:100AC00008FB00BF4DF808EDFFF7CEFF94BF0120F3
:100AD00000205DF808FB00BF4DF808EDFFF7C4FFEC
:100AE00034BF012000205DF808FB00BF4FEA410C35
:100AF0007FEA6C5C02D150EA013C0AD14FEA430C18
:100B00007FEA6C5C02D152EA033C02D14FF0000054
:100B100070474FF0010070474FEA410212F5001292
:100B200015D211D56FF47873B3EB625212D94FEA34
:100B3000C12343F0004343EA505311F0004F23FA1E
:100B400002F018BF404270474FF00000704750EA73
:100B5000013005D111F0004008BF6FF00040704730
:100B60004FF00000704700BF4A0011D212F500128A
:100B700011D20DD56FF47873B3EB62520ED44FEAF5
:100B8000C12343F0004343EA505323FA02F0704775
:100B90004FF00000704750EA013002D14FF0FF30B3
:100BA00070474FF0000070474FEA4102B2F1E04356
:100BB00024BFB3F5001CDCF1FE5C0DD901F0004C44
:100BC0004FEAC0024CEA5070B2F1004F40EB830094
:100BD00008BF20F00100704711F0804F21D113F1C0
:100BE0003872BCBF01F00040704741F480114FEAF9
:100BF0005252C2F11802C2F1200C10FA0CF320FA82
:100C000002F018BF40F001004FEAC1234FEAD3239E
:100C100003FA0CFC40EA0C0023FA02F34FEA430308
:100C2000CCE77FEA625307D150EA01331EBF4FF091
:100C3000FE4040F44000704701F0004040F0FE40AC
:100C400040F40000704700BF80F0004002E000BFA9
:100C500081F0004142001FBF5FEA410392EA030FA7
:100C60007FEA226C7FEA236C6AD04FEA1262D2EBF1
:100C70001363C1BFD218414048404140B8BF5B42F6
:100C8000192B88BF704710F0004F40F4000020F08F
:100C90007F4018BF404211F0004F41F4000121F0A5
:100CA0007F4118BF494292EA030F3FD0A2F10102EF
:100CB00041FA03FC10EB0C00C3F1200301FA03F12D
:100CC00000F0004302D5494260EB4000B0F5000F50
:100CD00013D3B0F1807F06D340084FEA310102F10F
:100CE0000102FE2A51D2B1F1004F40EBC25008BFC1
:100CF00020F0010040EA03007047490040EB00008B
:100D0000013A28BFB0F5000FEDD2B0FA80FCACF18B
:100D1000080CB2EB0C0200FA0CF0AABF00EBC250B8
:100D200052421843BCBFD0401843704792F0000FA6
:100D300081F4000106BF80F400000132013BB5E7F9
:100D40004FEA41037FEA226C18BF7FEA236C21D06F
:100D500092EA030F04D092F0000F08BF08467047D4
:100D600090EA010F1CBF0020704712F07F4F04D1A2
:100D7000400028BF40F00040704712F100723CBFB5
:100D800000F50000704700F0004343F0FE4040F4DF
:100D9000000070477FEA226216BF08467FEA23639D
:100DA0000146420206BF5FEA412390EA010F40F488
:100DB000800070474FF0000304E000BF10F00043D4
:100DC00048BF40425FEA000C08BF704743F09643BB
:100DD00001464FF000001CE050EA010208BF7047D6
:100DE0004FF000030AE000BF50EA010208BF70475D
:100DF00011F0004302D5404261EB41015FEA010C72
:100E000002BF84460146002043F0B64308BFA3F169
:100E10008053A3F50003BCFA8CF2083AA3EBC2534B
:100E200010DB01FA02FC634400FA02FCC2F120026A
:100E3000BCF1004F20FA02F243EB020008BF20F0A1
:100E40000100704702F1200201FA02FCC2F1200207
:100E500050EA4C0021FA02F243EB020008BF20EAFC
:100E6000DC7070477BB972B90029BEBF00204FF01B
:100E7000004106E008BF00281CBF6FF000414FF0A2
:100E8000FF3000F007BAADF1080C6DE904CE00297F
:100E900009DB002B1ADB00F095F8DDF804E0DDE952
:100EA000022304B07047404261EB4101002B1BDB81
:100EB00000F088F8DDF804E0DDE9022304B04042E8
:100EC00061EB4101524263EB43037047524263EBD3
:100ED000430300F077F8DDF804E0DDE9022304B015
:100EE000404261EB41017047524263EB430300F023
:100EF00069F8DDF804E0DDE9022304B0524263EB57
:100F00004303704753B94AB9002908BF00281CBFE2
:100F10004FF0FF314FF0FF3000F0BCB9ADF1080CDD
:100F20006DE904CE00F04EF8DDF804E0DDE90223BF
:100F300004B07047430803F05533C01A830803F028
:100F4000333300F03330184400EB101000F00F3052
:100F500000EB002000EB0040000E704707EE900A07
:100F6000F5EEC07AF1EE10FA01D400F00BB8F1EE14
:100F7000677A08B517EE900A00F004F8404261EB7A
:100F8000410108BDD0B5FFF7BFFA0C4B0022064661
:100F90000F46FFF711FBFFF7E7FD0446FFF792FA54
:100FA000074B0022FFF708FB02460B463046394646
:100FB000FFF74AF9FFF7D8FD2146D0BD0000F03D0C
:100FC0000000F0412DE9F047089D04468E46002BB5
:100FD0004DD18A42944669D9B2FA82F252B101FAED
:100FE00002F3C2F1200120FA01F10CFA02FC41EAFD
:100FF000030E94404FEA1C48210CBEFBF8F61FFA82
:101000008CF708FB16E341EA034306FB07F199421C
:101010000AD91CEB030306F1FF3080F01F819942CF
:1010200040F21C81023E63445B1AA4B2B3FBF8F0A9
:1010300008FB103344EA034400FB07F7A7420AD930
:101040001CEB040400F1FF3380F00A81A74240F258
:1010500007816444023840EA0640E41B00261DB1C3
:10106000D4400023C5E900433146BDE8F0878B42F8
:1010700009D9002D00F0EF800026C5E900013046B7
:101080003146BDE8F087B3FA83F6002E4AD18B4291
:1010900002D3824200F2F980841A61EB030301203B
:1010A0009E46002DE0D0C5E9004EDDE702B9FFDE27
:1010B000B2FA82F2002A40F09280A1EB0C014FEAD2
:1010C0001C471FFA8CFE0126200CB1FBF7F307FB2F
:1010D000131140EA01410EFB03F0884208D91CEBD2
:1010E000010103F1FF3802D2884200F2CB8043466F
:1010F000091AA4B2B1FBF7F007FB101144EA01444E
:101100000EFB00FEA64508D91CEB040400F1FF31DC
:1011100002D2A64500F2BB800846A4EB0E0440EACA
:1011200003409CE7C6F12007B34022FA07FC4CEAD3
:10113000030C20FA07F401FA06F31C43F9404FEAC6
:101140001C4900FA06F3B1FBF9F8200C1FFA8CFEDB
:1011500009FB181140EA014108FB0EF0884202FA2F
:1011600006F20BD91CEB010108F1FF3A80F08880F0
:10117000884240F28580A8F102086144091AA4B2AD
:10118000B1FBF9F009FB101144EA014100FB0EFE2E
:101190008E4508D91CEB010100F1FF346CD28E455D
:1011A0006AD90238614440EA0840A0FB0294A1EBEE
:1011B0000E01A142C846A64656D353D05DB1B3EB4B
:1011C000080261EB0E0101FA07F722FA06F3F1407B
:1011D0001F43C5E9007100263146BDE8F087C2F122
:1011E0002003D8400CFA02FC21FA03F3914001439A
:1011F0004FEA1C471FFA8CFEB3FBF7F007FB1036D3
:101200000B0C43EA064300FB0EF69E4204FA02F47E
:1012100008D91CEB030300F1FF382FD29E422DD9D1
:10122000023863449B1B89B2B3FBF7F607FB163306
:1012300041EA034106FB0EF38B4208D91CEB010186
:1012400006F1FF3816D28B4214D9023E6144C91A06
:1012500046EA004638E72E46284605E70646E3E616
:101260001846F8E64B45A9D2B9EB020864EB0C0E20
:101270000138A3E74646EAE7204694E74046D1E72F
:10128000D0467BE7023B614432E7304609E76444DD
:10129000023842E7704700BF02E000F000F8FEE7C6
:1012A00072B6374880F30888364880F30988364894
:1012B0003649086040F20000CCF200004EF634716E
:1012C000CEF200010860BFF34F8FBFF36F8F40F283
:1012D0000000C0F2F0004EF68851CEF20001086026
:1012E000BFF34F8FBFF36F8F4FF00000E1EE100A96
:1012F0004EF63C71CEF200010860062080F314889F
:10130000BFF36F8FA6F09EFDA5F006FE4FF055309F
:101310001F491B4A91423CBF41F8040BFAE71D49A3
:10132000184A91423CBF41F8040BFAE71A491B4A9C
:101330001B4B9A423EBF51F8040B42F8040BF8E7EE
:1013400000201849184A91423CBF41F8040BFAE7C3
:10135000A6F07CFDA5F034FE144C154DAC4203DA2A
:1013600054F8041B8847F9E700F06AFC114C124D51
:10137000AC4203DA54F8041B8847F9E7A6F064BDD1
:1013800000060020002200200000010808ED00E017
:101390000000002000060020B8E40D080022002014
:1013A000F8260020F826002090470120E0010108DF
:1013B0003C0201083C0201083C0201082DE9F04F03
:1013C0002DED108AC1F80CD0C3689D46BDEC108A83
:1013D000BDE8F08F002383F311882846A047002042
:1013E000A5F020FBFEE7A5F07DF900DFFEE7000099
:1013F00001F0FF01102A2BDB10F0070F08D010F8C6
:10140000013B013A8B422DD010F0070F42B3F6D1C9
:10141000F0B441EA012141EA014122F007047FF0E2
:1014200000070023F0E80256083C85EA010586EA39
:10143000010685FA47F5A3FA87F586FA47F6A5FA75
:1014400087F68EB9EED1F0BC01F0FF0102F0070281
:1014500032B110F8013B013A83EA010313B1F8D12C
:101460000020704701387047002D06BF354603380D
:10147000073815F0010F07D1013015F4807F02BF46
:10148000013015F4C03F0130F0BC0138704700BF97
:1014900010F8012B11F8013B012A28BF9A42F7D01E
:1014A000D01A7047034613F8012B002AFBD1181AF3
:1014B0000138704738B50022002304460D46FFF777
:1014C000EDFA28B920462946BDE8384000F00AB8B0
:1014D000204605F1004100F005F8404261EB410172
:1014E00038BD00BFD0B50C4B002206460F46FFF7B3
:1014F00063F8FFF739FB0446FEF7E4FF074B0022D1
:10150000FFF75AF802460B4630463946FEF79CFE76
:10151000FFF72AFB2146D0BD0000F03D0000F0415E
:10152000036800221B6818471FB5094BD3F88C2AA3
:101530000092D3F8902A0192D3F8942A0292D3F819
:10154000983A03936A4672F0EDFD05B05DF804FB2E
:101550001047002070B50024144E2546E1B23046F5
:1015600003F0EAFE002178F033FF02281CD00428A3
:101570001AD0012804F1010408BF0125102CEDD177
:101580000DB9002070BD094D0024E1B2284603F0DA
:10159000D3FE012178F01CFF022805D0042803D0D7
:1015A0000134102CF1D1ECE70120EBE710270020EB
:1015B00037B5C47F0191054644B9FFF7CBFF0199C8
:1015C000044630B9064A284671F068FF204603B049
:1015D00030BD284603B0BDE8304072F009BE00BF00
:1015E0003C010C08F0B591B005460E4671F0E8FFDD
:1015F0000446D8B11021284671F066FDB0B1002133
:101600002E2204A803AF0391AAF068FB0BF020FF81
:1016100032233A4600210BF075FA044630B9054BE7
:10162000009732461021284671F056FD204611B031
:10163000F0BD00BF68010C08F8B5394F3B7806468D
:10164000002B6AD101253D7072F08CFE044630B942
:10165000344A387013782B4313702046F8BD4DF090
:1016600099F829464CF082F82F4803F0E1F92F4B06
:101670001D710B253FF080FA013D3FF033FA15F064
:10168000FF05F7D10BF0E4FE294BD0F80022C3F898
:10169000202290F87C22D10706D5920704D429464F
:1016A000A3F5405002F086FC224B234D1B68D86AFC
:1016B000036801211B6898471B4808F081FB012142
:1016C0001E4879F009FF4DF065F895F81C2295F851
:1016D000B41E4CF027FAA5F5005003F09BF949F031
:1016E000FBF848F03BFC0023A5F500503B7000F0F0
:1016F00039FA0028B1D157F00DF80421104A50F002
:1017000055F92021304671F0DFFC0028A5D00D4BA3
:1017100001222021304671F0DFFC00249DE700BF4C
:10172000F8260020DC7F002010270020BD7F00204D
:10173000105700200827002010470020EC550020FB
:1017400074010C0891010C08F0B5234B93F8A73FE6
:1017500087B01BB90024204607B0F0BD72F0B8FE78
:1017600004460028F6D00BF073FE06460AF0C8FCCB
:10177000D0B111F0B1FD90F92430022B14D1002525
:101780000027E9B203AA3046039704970597019111
:101790000BF054F828B111F09FFD019903AA11F044
:1017A000A7FA0135032DECD100210C4879F094FE05
:1017B0000B4827F0A9FA4CF0EDFF00214BF0D6FFC3
:1017C000084B1B68D86A036800211B6898470648C5
:1017D00003F044FFBFE700BF10470020EC55002096
:1017E0005C520020082700201027002009F08CB848
:1017F0005AF0A2BC48F0BABF20F03AB84CF038B961
:101800000FF07EBB5AF0E2BF58F0E8B856F01EBAAF
:1018100009F09EB808F00ABD40F0E0BB1AF082BAA9
:101820005AF0E4BF08F006BE02F0B2BB04F05EBEA0
:1018300000F0E6BB03F03CBD08F0C2BB20F036BBB5
:10184000034808601F21117008221A60704700BF0A
:1018500084040C0810B5044603F04EFB204603F048
:1018600025FC204603F0A8FA204603F051FA58F070
:1018700025FCBDE8104058F001BB0000FFF7EABFAF
:1018800038B5044600F5485034300EF097FE11F09C
:1018900023FD90F92130F3B190F84033DBB104F52A
:1018A0003C5020304FF030FC034693ED000ADFED52
:1018B0000A0A9F20B7EE001A22F040F894F9B835D2
:1018C00004F28455012B08BF85ED0E0A2846BDE8B9
:1018D000384011F011BC38BD00000000FFF7D0BF48
:1018E00037B50121044608F0F3FF90B304F56455C1
:1018F0002046083501F010FE284672F00FFE04F570
:1019000075511031284672F06FFE4FF48051204619
:1019100008F0DEFFE8B104F56C5204F57F60203278
:10192000692101904BF002FE04F5705201980832D3
:101930006A214BF0FBFD04F57352019830326B21A4
:101940004BF0F4FD04F57F52019838326C214BF0D6
:10195000EDFD8021204608F0BBFF60B14FF400216F
:10196000204608F0B5FF30B921F0E2FA03B0BDE837
:1019700030401FF00BBC03B030BD0000FFF7B0BF1C
:1019800010B5044600F52A50243078F079FD204641
:1019900003F0E6F8204603F051F8204603F096F8ED
:1019A000204603F0F7FA204603F02CFC204603F013
:1019B00061FC04F58F501030BDE810405FF02CBA88
:1019C000FFF7DEBF10B5044600F59250103001213C
:1019D0000BF0B0FC04F561500C30BDE8104009F08C
:1019E0004FBF0000FFF7EEBF10B5044608F0D2FB72
:1019F0001021204608F06CFF40B1204601F0DCFCCD
:101A000021F096FABDE810401FF0B2BC10BD0000F6
:101A1000FFF7EABF10B500F5005292F8B13E13F09F
:101A2000010408D1084A00F53250083004214FF073
:101A3000BDFF002010BD92F8D53EDB0701D5034A5B
:101A4000F1E70120F6E700BF00020C081F020C08B6
:101A500000230B600120704710B5044604F50054C4
:101A60006BF0DCFC94F8A71FBDE810406BF0B2BC33
:101A7000FFF7F2BF13B500F50053044693F8B13EEB
:101A8000DA072BD500F5925001A910300AF010FCAE
:101A9000C8B104F5805494F8CC34DB070DD504F5B7
:101AA000986393ED007ADFED0F6ADDED017AB8EE11
:101AB000C77AE7EE667ACDED017A9DED010AB1EEC7
:101AC000400A02B010BD0EF005F8437C242202FB50
:101AD0000300D0ED0B7AF1EE677AECE79FED020A96
:101AE000EFE700BF0AD7233C0000000010B500F567
:101AF000005386B093F8B13EDB07044603D49FED54
:101B0000170A06B010BD04F5925402A8103410F064
:101B10001DFB02A920460BF08DFA0028EFD001A989
:101B200020460AF0C5FB58B90DF0D4FF437C2422AF
:101B300002FB0300D0ED0B7AF1EE677ACDED017A6E
:101B4000DDED037A9FED067A9DED010AF8EEE77A66
:101B5000A7EEC70AB1EE400AD3E700BF00000000BD
:101B60000AD7233C70B505468AB005F5925602A8FF
:101B7000103610F0EBFA02A930460BF05BFA04467F
:101B800088BB05F5907018F01FFE60BB254ADFED9D
:101B9000267AD2ED006A12ED017A9FED246A66EE94
:101BA000A76A52ED027A009427EE067A67EE867AEB
:101BB000FDEEE66ABDEEC77AFDEEE77A16EE903AE4
:101BC00017EE102A17EE901A06A810F0DFFA089800
:101BD00005F53255083508B1099939B9144A042177
:101BE00028464FF0E3FE20460AB070BD22F00CF903
:101BF000044608B90F4AF2E706A930460BF03EF852
:101C0000044608B90C4AEAE70C4A062128464FF078
:101C1000CDFE30460BF0FEFD4521284657F098FBDF
:101C2000E1E700BF985100200000C8428096184BA1
:101C300034020C0863020C088C020C08BB020C086E
:101C400038B5054B1C6823680A461D68034B0146DE
:101C50002046A847002038BD082700201027002074
:101C600010B5044648F038FE04F5005101F6DC6377
:101C7000426FDA6004F5405303F6081003F555632C
:101C80008266C3F8FC2291F8B43E133B012B06D9BF
:101C900004F564500830BDE8104073F08DB810BDF5
:101CA000FFF7DEBF37B50221044608F011FEB8B3D6
:101CB0000121204608F00CFE90BB04F56455204637
:101CC000083501F029FC284672F028FC04F575510E
:101CD0001031284672F088FC4FF48051204608F0FD
:101CE000F7FDE8B104F56C5204F57F6020326921FC
:101CF00001904BF01BFC04F57052019808326A21E8
:101D00004BF014FC04F57352019830326B214BF008
:101D10000DFC04F57F52019838326C214BF006FC23
:101D20004FF40031204608F0D3FD20B104F53B50BC
:101D30001C307AF0C5FB4021204608F0C9FD18B1DF
:101D400004F57F604BF090F84FF48061204608F076
:101D5000BFFD18B104F57F604BF020F9202120462B
:101D600008F0B6FD58B1234DD5F8C80403689B6848
:101D7000984728B304F57550103075F0DBFE8021CC
:101D8000204608F0A5FD18B321F0D2F81FF022FA82
:101D90001021204608F09CFD20B104F56450083065
:101DA00073F00CF94FF40041204608F091FDF0B1BA
:101DB00004F59640503003B0BDE830405AF03EBEC6
:101DC000D5F8C8040368DB6898470028D2D0D6E766
:101DD0004FF48021204608F07BFD0028D4D14FF439
:101DE0000021204608F074FD0028CDD1D0E703B0D3
:101DF00030BD00BF10770020FFF754BF70B500F56D
:101E000000552C4BB5F862221A70044600F55E505E
:101E100000212830FFF7CCFB95F8B03E264E60F34A
:101E2000000385F8B03EB071204608F03FFD95F8FC
:101E3000A73FF0714FF6FF712046737108F048FD1F
:101E400028B1D5F8B02E0721204601F083FB95F884
:101E5000A73F23B904F53B501C307AF03BFD59F005
:101E600095FE59F063FB204608F064FD134B1B6898
:101E7000DB6A93F89C6036B195F81E321BB97CF092
:101E8000FFFAC5F8200285F81E6248F025FD48F0EB
:101E90008DF904F56450083072F0FCFC48F01CFD2C
:101EA00048F084F904F57D502430BDE870406AF0B4
:101EB0001FBB00BF7C230020BD7F0020082700201F
:101EC000FFF79CBF10B506480C4677F0BDF8DFED74
:101ED000057A20EE270A012084ED000A10BD00BF1C
:101EE000746800200AD7233C10B508480C4677F0E8
:101EF000BFF807EE900A9FED067AF8EEE77A012028
:101F000067EE877AC4ED007A10BD00BF74680020C8
:101F10000AD7233C70B52DED048B00F5005482B038
:101F20000E4615464FF47A714FF4FA52B4F95C023A
:101F30008DED011AF0EE408AB0EE608A21F03CFD92
:101F4000034607EE903ADFED240AA4F85C02B8EEEF
:101F5000E71A0B209DED010ADFED209A21F0EEFC3F
:101F6000B4F95C32DFED1E6A07EE103AB8EEC77ABC
:101F7000B0EE409AC7EE267A67EEA88A27EE888AE6
:101F800028EEA80AA8EE080AA7F0F8FDB4EEC09A59
:101F9000F1EE10FA42BFC9EE007A28EE278A68EE09
:101FA000A78A28EE290AA7F07DFAB0EE409A28EE1B
:101FB000A90AA7F007FC29EE000AA7F053F9DFED04
:101FC000097A20EE270A86ED000A85ED008A02B024
:101FD000BDEC048B70BD00BF00007A44D4023739D9
:101FE00000A08C459F0CB34507EE901A00F50050F9
:101FF000F8EEE77A90EDC00A27EE800A70470000FD
:1020000073B5044600F5925001A9103004F500564E
:102010000AF0D6FDD6F8843C8342054606D004F586
:102020006450083074F09CF8C6F8845C02B070BD4F
:1020300038B5104A13780133DBB2032B044600F5A0
:10204000405505D8137005F6140595ED000A38BD06
:1020500000F5605000233030137078F0A1F904F5DA
:102060006051083121F04EFE05F6140383ED000A9D
:10207000E9E700BFF926002038B5044600F56050B6
:102080002DED028B303078F091F9054623F054FDA8
:102090002046B0EE408A08F009FC04F54054C0B177
:1020A000DFED0F7AB4EEE78AF1EE10FA11DDD5ED2F
:1020B000000A95ED010AA7F017FCDFED0A7A20EE81
:1020C000270ADFED097A20EE270A04F6240383EDC0
:1020D000000ABDEC028B04F6240494ED000A38BD1E
:1020E00000401C46E02E65420000C84200F5A553A2
:1020F000D3ED005AD2ED007AD3ED036A91ED006A78
:1021000026EEE77A67EEA57AA6EE257AE6EE267A3F
:1021100081ED007AC2ED007A7047000000F50050B2
:10212000B0F98E3233B9B0F98C020028B8BF404202
:1021300080B2704783EAE370A0EBE370F8E7000039
:1021400070B52DED068B00F5005482B094F8D41EC6
:102150008DED010A11F001010546009162D1D4F81C
:10216000940A9FED329A58F003F8B4F99232DFEDF9
:10217000300A9DED010A07EE900A08EE103A05F5C7
:10218000405606F2EC73F8EEE79AB8EEC88AD3ED43
:10219000007A6720B0EE491A28EE278A21F0CEFB9C
:1021A00039EEC8AA0099B4F992024FF4C872F0EE61
:1021B000408A21F001FCB4EEE8AAF1EE10FAA4F88E
:1021C000920216DD2846FFF7A9FF07EE900A78EE87
:1021D000CA8AB8EEE70A60EE288A88EE8A0AFDEE1F
:1021E000C07A17EE903AA6F8243202B0BDEC068B06
:1021F00070BD78EE297AF4EEE87AF1EE10FA49BF74
:10220000B4F98C329FED0A0A00EE103A78EEE78AB4
:1022100041BFB8EEC00A79EE677A60EE288A88EE90
:10222000A70ADCE79FED020ADFE700BF00007A445F
:102230000000000000207047704700007047000059
:102240007047000000207047002070470020704752
:102250000120704700207047704700007047000061
:1022600070470000002070470C4991F8B43E102BD5
:102270000FD801229A400A4B1340002B0CBF1020AC
:10228000182091F8A73F33B940F0400040F001001A
:1022900070471020F5E740F0C000F7E71047002036
:1022A00098000100014B93F864027047104700202A
:1022B0007047000010B5044652F06AFE054879F0F8
:1022C000F1F9054A034606212046BDE8104052F0C8
:1022D00047BE00BFEC550020F8060C0800B513EE11
:1022E000103A8DB06222CDF8253013EE903ACDF839
:1022F00029302123CDE900328DF82410192303AAB7
:10230000C2218DED030ACDED040A8DED051ACDED48
:10231000061A8DED072ACDED082A50F07BFB0DB093
:102320005DF804FB08B50B484EF0EEFE0346DFED0A
:102330000A0A93ED000A9F20B7EE001A21F0FEFA78
:10234000DFED067A20EE270ABDEEC00A10EE103A45
:1023500018B208BD30560020000000000000C8423E
:102360000148FFF7C3BB00BF1027002008B506488F
:10237000FFF7BCFBDFED057A20EE270AFDEEC07A01
:1023800017EE900A08BD00BF1027002000007A4415
:10239000F8B5704E04460BF05BF8B6F8A03205466F
:1023A000D80737D506F5DA5306F5D952DFED6A7A44
:1023B00053ED032A13ED042A53ED051A13ED021A07
:1023C00092ED000A9FED657AD5EDC50AD3ED003A8E
:1023D00093ED013A207C62EEA72A22EE272A61EED5
:1023E000A71A21EE271A60EE870A20EE270A01219C
:1023F000FFF774FF207C50F0A3FA0746207C51F0D1
:10240000A3F900F121039F4204D2207CBDE8F840EB
:102410004FF0ECBCB6F8A03299072FD5504BDFED4A
:102420004E7A53ED032A13ED042A53ED051A13EDEA
:10243000021A13ED080A9FED497AD5EDC60AD3EDCD
:10244000003A93ED013A207C62EEA72A22EE272A79
:1024500061EEA71A21EE271A60EE870A20EE270AFE
:102460000221FFF73BFF207C50F06AFA0746207CF0
:1024700051F06AF900F121039F42C6D3B6F8A032A9
:102480005A072FD5374BDFED347A53ED032A13ED7E
:10249000042A53ED051A13ED021A13ED080A9FEDF5
:1024A0002F7AD5EDC70AD3ED003A93ED013A207C9F
:1024B00062EEA72A22EE272A61EEA71A21EE271A3A
:1024C00060EE870A20EE270A0321FFF707FF207C32
:1024D00050F036FA0746207C51F036F900F121031E
:1024E0009F4292D3B6F8A0321B0732D51E4B9FED08
:1024F0001F7AD5EDD60ADFED187AD3ED032A93EDD6
:10250000022AD3ED011A93ED041A13ED020AD3ED5A
:10251000063A93ED073A207C70EE870A62EEA72A0E
:1025200022EE272A61EEA71A21EE271A20EE270AAB
:10253000F1EE600A0421FFF7D1FE207C50F000FA92
:102540000546207C51F000F900F121039D42FFF483
:102550005CAFF8BD104700200AD7233CE02E65424F
:102560003863002020640020106700200AE81C4126
:10257000014802F093B800BF1027002007B50846B5
:1025800001910FF0EBFE38B10448019904F064FEAC
:10259000002003B05DF804FB0420FAE7CC7C0020A7
:1025A00038B5C5780B46352D044628BF352535226C
:1025B00000211846A9F092FB2A4604F10C01BDE85F
:1025C0003840A9F041BB00002DE9F0472DED028B0A
:1025D0008A7A4B7A43EA0223CA7A43EA0243522BAD
:1025E000A2B005460C4600F0568111D8452B00F0EC
:1025F000E680462B00F03C81012B00F062822146F0
:10260000284622B0BDEC028BBDE8F04756F0A2B8D8
:10261000562B00F0DA8100F2C080542BEFD114A9C0
:102620002046FFF7BDFFAE4B93F8B42E042A09D025
:10263000032A40F0188103F5405393F86C37032BBD
:1026400040F011819DF884200C2A00F20C8141F2A7
:102650008234D440E44314F0010440F00481BDF816
:102660008030002613F0070703F0380A03F4E079FE
:1026700003F4806803F400650D960E960F962CD136
:102680009FED986A9DED167ADDED177ADDED156AFE
:1026900027EE067A67EEC67A66EE866AA2F108032E
:1026A000012BCDED0D6A8DED0E7ACDED0F7A01D9AE
:1026B0000C2A04D18C480EAA0DA9FFF717FD9DF82E
:1026C0008430DA1F022A01D90C2B06D1874877F013
:1026D00065FE01460DA823F00DFD10961196129689
:1026E000BAF1000F20D19FED7F6A9DED197ADDEDE3
:1026F0001A7ADDED186A9DF8843027EE067A67EEC7
:10270000C67A66EE866AA3F10802012ACDED106A48
:102710008DED117ACDED127A01D90C2B04D17248CE
:1027200011AA10A9FFF7E2FCB8F1000F40F02381D5
:10273000DFED6F7A9DED1E0A9DF8844020EE270A9A
:10274000DFED687AA4F10906744220EE270A74418D
:10275000002D40F01381DFED667ADDED1F0A60EE9B
:10276000A70ADFED607A60EEA70A002F40F009812A
:10277000BAF1000F40F01981B9F1000F73D0B5FA2A
:1027800085F56D09B8FA88F3019400955B0910AAE4
:102790000DA9584805F090FC65E003F18073863B75
:1027A00023F07F43012B3FF62AAF0A46017C5248B3
:1027B00022B0BDEC028BBDE8F04748F0CFBD484DDC
:1027C000CA79B5F964329A424DD1CE781E2E28BF0F
:1027D0001E261E22002114A8A9F080FA324604F118
:1027E0000C0114A8A9F030FA9DF85A20B5F962320C
:1027F0009A4238D1BDF96C300B93BDF96A300A9317
:10280000BDF968300993BDF966300893BDF96430AD
:102810000793BDF962300693BDF960300593BDF9A9
:102820005E3004939DF85D300393BDF85B300293F6
:10283000BDF858300193BDF95630BDF95220BDF9AD
:1028400050100093A5F50050BDF9543003F0EEFB95
:102850007BF016FEC5F8C00E55F05CFF04467BF019
:102860000FFEC4F8B80122B0BDEC028BBDE8F087C2
:102870001B4ECA79B6F964329A42F4D17BF000FE5D
:102880002146C6F8C00E284622B0BDEC028BBDE83A
:10289000F04754F0C9B9CD78272D28BF2725272226
:1028A000002114A8A9F01AFA2A4604F10C0114A870
:1028B000A9F0CAF99DF876305F0623D57BF0E0FDDC
:1028C0000E4D14ACC5F884040FCC05F591650FC509
:1028D0000FCC0FC594E8030085E80300C3E700BFF1
:1028E000104700200000C84210270020405F002051
:1028F000E02E6542087D0020F8720020107700204D
:102900000000000013F0C00FADD15FED030A9DED94
:102910001C0A40F2C120B7EE001A21F00FF8F6EEC3
:10292000000AB0EE408A20F007FF08BBB6EE007A3E
:10293000834BB4EEC78AF1EE10FA78EE477AD4BF33
:1029400093ED610A93ED600A77EEA77AD8BFB0EEF7
:10295000C00A20EE270A159B1093169B1193179B14
:1029600012937848189B139310A905F06BFC7AE733
:102970009FED750AEFE79FED740AE9E6DFED720A55
:10298000F3E6BAF1000F7FF46EAFB9F1000F3FF438
:102990006AAFB5FA85F3B8FA88F26A4800945B0921
:1029A000520910A905F0BAFA5DE7B9F1000F3FF43A
:1029B0005AAFB5FA85F3B8FA88F200945B09520968
:1029C0000DA9604806F080F84DE714A92046FFF7EE
:1029D000E7FD5E4A92F8B43E042B08D0032B1CD1CD
:1029E00002F5405292F86C27032A7FF43CAFBDF801
:1029F0008020500702F0070102F0380602F4E0746C
:102A00000DD4022B0BD1DDED177A9FED517A4C4B93
:102A100067EE877AC3ED297A25E7022BE5E70023E5
:102A20000D930E930F9300296AD1DDE9150121F072
:102A3000EBF900283FF417AF9DF884100CAA284644
:102A400055F0E6F900283FF40EAFDDED177A9FED63
:102A5000408A0C9B009367EE887ADDE91512FDEE43
:102A6000E77A10A817EE903A0FF090FB0DA910A886
:102A70000FF02EFD00283FF4F6AED6B9002C3FF43F
:102A8000F2AEDDED186A9DED197ADDED1A7A2D486A
:102A900066EE886A27EE087A27EEC88A10AA0DA982
:102AA000CDED106A8DED117A8DED128A05F098FA50
:102AB000D9E6002C3FF4D7AE0DA9224805F0CCFF93
:102AC000D1E6CD781F2D28BF1F251F22002114A875
:102AD000A9F004F92A4604F10C0114A8A9F0B4F8ED
:102AE000159B9A007FF5BFAE169B9B003FF5BBAED2
:102AF000184822B0BDEC028BBDE8F04777F0DEBC91
:102B0000002E7FF4B0AE002C3FF4ADAE9FED106A06
:102B1000DDED186A9DED197ADDED1A7A094866EE49
:102B2000866A27EE067A67EEC67A10A9CDED106A9E
:102B30008DED117ACDED127A05F0D6F993E600BF4E
:102B400010670020087D00200000000010470020D2
:102B50000000C842B451002010B5074B93F9E82B90
:102B600040F6C53440F6C513002A08BF1C4651F094
:102B700089FA204310BD00BF1067002008B5064841
:102B8000FEF778FFDFED057A20EE270AFDEEC07A2A
:102B900017EE900A08BD00BF1027002000007A44FD
:102BA00010B504460FF028FE204610BD08B54B694D
:102BB000012B03D0BDE8084051F0C8BA55F0AAFD7A
:102BC000024A06214EF0F2FE032008BD04070C085D
:102BD00010B50C4890F8A74F3CB155F09BFD0A4A40
:102BE00006214EF0E3FE04200BE0A0F50050FEF7B6
:102BF00011FF0028F7D00CF06DFF01210CF01EFE34
:102C0000204610BD104700202C070C080E4B93F8EF
:102C1000D42ED20714D403F5805292F8A5277AB99E
:102C2000B3F8D42E02F4FF7252B993F8A72F4AB921
:102C300093F8B03E13F0100F14BF0320012070472B
:102C400005207047042070471047002010B588B059
:102C500004460022134803A970F0F6F8F8B1247C6A
:102C60007BF00EFCDDED037A9FED0F7A049067EEAA
:102C7000877A0023FDEEE77A0593069317EE903AE4
:102C8000ADF81C3000238322ADF81E301023CDE9AF
:102C900000328F210E2304AA20464FF0BBFE08B05D
:102CA00010BD00BFD44800200000C8420C2070476F
:102CB000014B93F8B40E70471047002038B512212D
:102CC0002DED028B04464FF0A3F820B90025BDEC92
:102CD000028B284638BD072058F0D2FCB6EE008A99
:102CE000F0EE487AE0EE087A4B49F7EE008A20468B
:102CF00038EEE70A53F040FA122120464FF088F8E8
:102D00000028E3D0062058F0BBFCF0EE487AE0EE55
:102D1000087A4249204638EEE70A53F02DFA12218C
:102D200020464FF075F80028D0D03D4D3D49D5F8EC
:102D3000E437002BB8BF03339B1000EE103A204657
:102D4000B8EEC00A53F018FA122120464FF060F88E
:102D50000028BBD03B2058F093FCF0EE487AE0EE20
:102D6000087A31492046B0EE670A53F005FA12217D
:102D700020464FF04DF80028A8D03C2058F080FCA9
:102D8000A0EE088A29492046B0EE480A53F0F4F92B
:102D9000122120464FF03CF8002897D005F2EC7342
:102DA000234993ED000A204653F0E6F9122120460C
:102DB0004FF02EF8002889D095F8F0371D4900EE25
:102DC000103A2046B8EE400A53F0D6F912212046B8
:102DD0004FF01EF800283FF479AF95F8F137164907
:102DE00000EE103A2046B8EE400A53F0C5F9122121
:102DF00020464FF00DF8054600283FF467AF0F4B13
:102E0000DFED0F7A93ED000A0E4980EE270A204687
:102E100053F0B2F95BE700BF48070C0850070C08F5
:102E20001057002057070C0861070C0869070C08A9
:102E300071070C087B070C0885070C08707E0020C2
:102E40000000C8428F070C08282938B5054614D061
:102E5000472908D027291BD112214EF0D9FF04465B
:102E600030B9002402E0FFF729FF0124204638BDD5
:102E7000297C094848F0D0F8F8E716214EF0C8FF41
:102E800004460028EDD0297C034848F09FF9EDE77F
:102E9000BDE8384055F090B9F8720020024B93F825
:102EA000B00EC0F3001070471047002070B5254EDB
:102EB0002DED028B0546D6F8C80491ED018A036812
:102EC00084B09B690C46984750B9BDEEC88A18EE8D
:102ED000103ADB0704D4022004B0BDEC028B70BDB5
:102EE000D4E9040120F090FF0028F4D068460FF0E8
:102EF0002DF96A462146284654F0A0FF0028EAD062
:102F0000114968460FF036FA0028E4D10F486946A7
:102F100005F058FD98B1D6F8C80403689B69984736
:102F200008B10020D8E70A480222042103F004FB7C
:102F300028B10648694605F045FD0028F1D1042076
:102F4000CAE700BF10770020045F0020087D002042
:102F50001027002008B502221021044803F0ECFAE3
:102F600000280CBF0420002008BD00BF102700204F
:102F700008B502220921044803F0DEFA00280CBF3C
:102F80000420002008BD00BF1027002013B5D1ED9C
:102F9000007AF5EEC07AF1EE10FA0C4602DA022061
:102FA00002B010BD9FED187AF4EEC77AF1EE10FA78
:102FB000F5D891ED030ADFED157AB0EEC07AB4EEE4
:102FC000E77AF1EE10FA18D5D4ED037A1048D4ED73
:102FD000010A94ED000AFCEEE77ACDED007AD4ED1B
:102FE000027A9DF80020FDEEE77ACDED017A9DF999
:102FF000041004F0BDF80020D2E7F7EE000A20F03C
:103000009BFB0028CBD0DFE70000B4430000003476
:10301000CC7C002008B5D1ED017AF5EEC07AF1EE56
:1030200010FA08DD9FED050A054827EE800A76F0C4
:1030300051F9002008BD0420FCE700BF0000C84291
:103040007468002008B5084890F8A73F0BB9042021
:1030500008BD02220321A0F5005003F06DFA0028FC
:10306000F5D00020F4E700BF1047002070B501F153
:103070000C050E460FCD86B06C460FC495E80300D4
:1030800084E8030096E80E00044806F0E3FE0028FA
:103090000CBF0420002006B070BD00BF1027002028
:1030A00030B48B8BB22B05460C4618D00AD8152BA2
:1030B00035D0732B10D0112B2ED02146284630BC92
:1030C00056F06EB9D12B0DD0B3F5967F0DD0C02B35
:1030D000F3D130BCFFF7EABE30BCFFF757BF30BCBE
:1030E000FFF798BF30BCFFF7C1BFD1ED007A9FED6D
:1030F0000F7AF0EEE77AF4EEC77AF1EE10FA11D516
:10310000D1ED017AF0EEE77AF4EEC77AF1EE10FA3B
:1031100008D530BCFFF796BF30BCFFF71BBF30BCF3
:10312000FFF726BF022030BC704700BF000000340C
:1031300070B52DED048B9FED2B0A9FED2B8A8CB083
:1031400004462A4822F0B6FF21EE081A2848267CB9
:10315000BDEEC11A60EE888A11EE103A20EE089A90
:103160001DB275F085FF07EE900AF8EEE77A204869
:1031700067EE887AFDEEE77A17EE903A1CB275F0AA
:1031800063FFDFED1C7A1C4B8DED059A20EE080ADB
:10319000B722B4EEE70AF1EE10FA58BFB0EE670AB4
:1031A000BCEEC00AD3ED007ACDED068A0023089369
:1031B000099310EE103A27EE888AADF82C301A23C6
:1031C000CDE900323E2105AA30468DED078AADF8E3
:1031D0002850ADF82A404FF01DFC0CB0BDEC048B1C
:1031E00070BD00BF9F0CB3450AD7233C846000200C
:1031F0007468002000FF7F479C64002008B591EDB3
:10320000007AF6EE007AB4EEE77AF1EE10FA06DD17
:10321000044801220521FEF797FA002008BD04208A
:10322000FCE700BFB85E0020002070470020704718
:10323000002070470120704790F89C308B4286BF79
:10324000283150F8210000207047000090F89C3091
:103250008B4286BF283150F82100002070470000C3
:10326000FA207047014B93F8620270471047002024
:1032700038B50446D0E90B30616B40F4E05222636C
:1032800041F4E052626343F4F842E2622B4A92F85E
:10329000B45E023D0E2D0FD8DFE805F00808080ED9
:1032A0000E080E080E0E0E0E0E0E080040F4F8402A
:1032B00041F4F8412063616392F8B11EC80708D554
:1032C00043F4F84343F00803E362236B43F008033D
:1032D0002363636B23F00803636392F8D81EC90766
:1032E00044BF43F008036363154B93F88034013BFC
:1032F000012B0BD8E36A43F48003E362236B43F4AE
:1033000080032363636B43F48003636392F8C83ADA
:10331000DB0712D50B4B1868E36A43F48073E36252
:10332000236B43F48073236338B1192142F03EFDCF
:1033300018B1636B43F48073636338BD104700209A
:10334000107700206880002013B54FF44470CDE959
:1033500000210FF049FA044628B1DDE9002155F0BB
:103360001BFC024B2360204602B010BD14090C0860
:103370007047000000207047002070470020704711
:1033800000207047002070470020704700207047E1
:10339000704700000120704700F50A501430704754
:1033A00000487047BC2D0C0800F5005090F8B40E92
:1033B000704700009C207047F0B52DED028B8FB058
:1033C0000023009300F580439FED508A93F9E83B7A
:1033D000044600F50056002B00F08F8000F5974062
:1033E00001226946683048F02FFD3322002101A8F0
:1033F000A8F074FCA3238DF8043095238DF80530D4
:103400007BF046F804F5405505F60813CDF80700A3
:1034100004F53C50D3F8DC20D3F8E030CDF80B10A5
:103420002030CDF80F20CDF813304DF06DFE03465F
:10343000DFED370A93ED000A9F20B7EE001A20F067
:103440007DFA10EE103ACDF8173006F6FC73B6EEA2
:10345000061AF4EE000A05F5556793ED000A3020D0
:1034600020F06CFA97EDD87ADFED2A7AC7EE277A4A
:1034700004F56050303010EE103ACDF81B3017EEE6
:10348000903ACDF81F3076F08DFF20EE080A94F8C0
:10349000712410EE103A2421CDF8233004F58C630A
:1034A00001FB023304F57F60DB6ACDF8273004F5B9
:1034B000AE430B44D3ED0F7AFDEEE77A332217EEDD
:1034C000903AD7EDDE7AADF82B30FDEEE77AB6F81C
:1034D000CA3AADF82D30009BCDF82F3017EE903A58
:1034E00001A9ADF83330B5F8E037ADF835304AF022
:1034F00059F90FB0BDEC028BF0BD06F6D823D3ED21
:10350000007A67EE887ACDED007A6EE70AD7233C21
:10351000000000000000C8421FB5044600F56550D9
:103520009FED0B0A343022F0C5FD04F5925001A93D
:1035300010308DED010ACDED020A8DED031A08F071
:10354000B1F809F085FF04B0BDE8104009F00EBDE8
:10355000E02E65427FB50E464FF6FF7104461546D4
:1035600007F0B6F9E0B1102200216846A8F0B6FBDA
:10357000A3238DF8003095238DF8013004238DF8B6
:1035800002307AF085FF1022CDF80300CDF8071045
:1035900004F57F6069468DF80B6003954AF082F967
:1035A00004B070BDF0B58BB0154606460F46242218
:1035B000002101A81C46A8F091FBA3238DF804303C
:1035C00095238DF8053006238DF806307AF060FFDC
:1035D0002B6804936B680593AB6806932368079385
:1035E0006368CDF80700CDF80B1008932422A36878
:1035F0008DF80F7001A906F57F6009934AF0D2F8A3
:103600000BB0F0BD10B500F50053044693F81C2232
:1036100093F8B41E00F57F604AF084FA04F59250E6
:1036200010300AF0F7F804F59070BDE8104017F07C
:1036300021BC00007047000070B504460B4E56F0E8
:10364000E3FB0B4B23605025601956F06BFD665170
:103650003035B5F5547FF7D104F5547058F06EF954
:103660002046044941F0ACF8204670BDB0410C083A
:103670003C4D0C08C4420C0830B50A4D0FCD8DB03E
:103680006C460FC40FCD0FC495E80F0084E80F00FF
:1036900000220321684640F075FC57F0D1FE0DB0C2
:1036A00030BD00BF18FF0B0837B500F509510122E6
:1036B0002031044648F0ACFD05212A48002240F0A4
:1036C00061FC41F083FA284A1388204643F008033E
:1036D0001380FFF7D1FF1721244841F057FCB6EEC5
:1036E000000A234841F068FC012504F50451002339
:1036F000083139201F4A009540F048FC1E490B68EC
:10370000D8070DD41D4B0D6004F5F95218321A601C
:1037100004F502521832DA6004F5885204329A61D4
:1037200004F50C50154903221C30012540F080FCA3
:10373000134A0095002304F57F61162040F026FC13
:10374000104B1A68D20705D40F4A1D6004F58B543C
:10375000183414600C48012103B0BDE8304040F03B
:1037600083BC00BF74420C084C800020BC410C0894
:1037700098410C0828770D08FC2600200022002024
:1037800090F00C0800270020242200200020704721
:10379000002070470069C0F3401070470F299DBF9B
:1037A000302303FB01005030002070470020704799
:1037B0000120704700F0CCBF01F014B900F04EBCFE
:1037C00001F07CBB70B51F4B036000F5005304464D
:1037D000D3F8440E1C4AC3F8882C08B10FF010F837
:1037E0001A4B236004F5805393F8D42E42B9D3F8D2
:1037F000D05E2DB128461CF043FE28460EF0FCFF9B
:1038000004F58A501C306EF013FF04F5895058F00F
:10381000C7FE04F6F44504F69446B54204D0183DBC
:1038200028461CF083FAF8E7094BC4F8C83804F6B8
:10383000C4104DF045F904F513604DF041F92046F0
:1038400070BD00BFC83B0C08980B0D086CE90C0854
:10385000C0AA0C0838B54C4B044640F8043B5BF05A
:1038600047FE04F110000CF0CFFF04F1680046F0B1
:103870000BFD04F5907016F0B7FE04F58C600BF0AC
:10388000C1FD04F284500EF0BDFF04F6C8001DF027
:1038900093FE04F547605BF0B3FD04F5546042F01D
:1038A0005DF904F57F6049F0B1FE04F588500430FD
:1038B00061F0B8FA04F5895058F05AFE04F58A50C0
:1038C0001C306EF0A1FE04F58B50183047F09EF8C6
:1038D00004F58E500C305CF0E9FF04F580530025B0
:1038E0002A4A83F8F05104F58F53103304F59050B1
:1038F00013603CF06BFF04F592502946103008F03D
:10390000E7F804F5C55069F027F804F5EB500430EA
:103910006BF0B2FE04F5F3501C306DF0CFFF04F5F0
:10392000F7506EF005FC04F5F950183007F060F818
:1039300004F50250183069F06DFC04F50350144989
:10394000303040F03DFF04F50450083061F0DCFDFC
:1039500004F5075004306FF06FF904F5005304F5D7
:10396000085083F81C520B4D34306FF0B3FA2B68BB
:1039700013B109487AF052FD2046084940F020FF73
:103980002C60204638BD00BF6CE90C08708900200F
:10399000447C0D08A0800020584D0C0884E80C08D9
:1039A00010B504465A3076F009FD04F15C0076F05B
:1039B00005FD04F15E0076F001FD04F1600076F093
:1039C000FDFC04F1620076F0F9FC04F1640076F08D
:1039D000F5FC04F1660076F0F1FC04F1680076F085
:1039E000EDFC04F16A0076F0E9FC04F16C0076F07D
:1039F000E5FC04F16E0076F0E1FC04F1700076F075
:103A0000DDFC04F1720076F0D9FC04F1740076F06C
:103A1000D5FC04F1760076F0D1FC04F1780076F064
:103A2000CDFC04F17A0076F0C9FC04F17C0076F05C
:103A3000C5FC04F17E0076F0C1FC04F1800076F054
:103A4000BDFC04F1820076F0B9FC04F1840076F04C
:103A5000B5FC04F1860076F0B1FC04F1880076F044
:103A6000ADFC04F18A0076F0A9FC04F18C0076F03C
:103A7000A5FC04F18E0076F0A1FC04F1900076F034
:103A80009DFC04F1920076F099FC04F1940076F02C
:103A900095FC04F1960076F091FC04F1980076F024
:103AA0008DFC204610BD00002DE9F04F044685B086
:103AB000FFF7D0FEBE4B236004F509502030FFF71E
:103AC0006FFF04F50C501C3004F50055FFF7B4FDF2
:103AD00004F52A50243076F093FC95F8C83A23F088
:103AE000030385F8C83A05F6D4234FF000080026F2
:103AF000A5F8CA8AC5F8CC8AC5F8D08A1E6005F632
:103B0000D82304F52B501E601C304DF0F9FA04F553
:103B10002B50283058F03EF9A64BC5F86C3BA64B0D
:103B2000C5F8743B04F52E50A44BC5F87C3BC5F892
:103B3000684BC5F8704BC5F8784B10300EF006FB9B
:103B400004F52E502C300EF001FB04F52F500830F8
:103B50000EF0FCFA4FF6FF79994BC5F8DC3B04F503
:103B60002D57A5F8E09B07F1A4000EF0EFFA0C37F3
:103B7000944B95491F604FF0FF3A3846C5F840AC6A
:103B800040F01EFE04F53150A5F8A49BA5F888ABC3
:103B9000043004F532573EF0DFF908378B4BC5F897
:103BA000848CC5F8883C07F1140079F095FB04F586
:103BB000095B04F534590BF11C0B04F5335809F17A
:103BC0002409404608F1140852F0E0F8C845F8D13D
:103BD0000723C5F8483E0023A5F84C3E4FF4CB70B0
:103BE0000EF008FEC5F8440E04F53950103079F097
:103BF00073FB04F53A50143079F06EFB744B1A687D
:103C000002B91F60734BC5F8883C04F53B59132378
:103C100009F11C0985F8B43E4FF4C871484678F0A4
:103C20002FFD6D4BC5F8DC3E6C4B04F54058C8E9E0
:103C300067336B4B1F6817B16A487AF0EFFBC3F824
:103C40000090694BC5F8DC3E05F6DC634FF07E5210
:103C5000C3F83823C3F83C636449484640F0B0FDDC
:103C6000634B0393634B0093029404AB04F54850F9
:103C700013E90C004FF4007134300CF0E5F804F552
:103C80005E5028306FF0D4F95B4BC8F8A83704F5C4
:103C90005F5088F8F17734300EF058FA012388F835
:103CA000043808F6080304F592511E605E609E60B9
:103CB00008F5036310311E605E609E6008F63C03E9
:103CC0009FED4E0A1E605E609E6004F561560C36E4
:103CD000C8F848183A46304604F5645807F084FEA0
:103CE00008F108085A4604F5605A04F5755B0AF1B4
:103CF000300A0BF1100B31464B46404670F0ACFEDB
:103D000031464B465246CDF80080584673F004F9D0
:103D100004F5824032465B465146CDF8008064305F
:103D200075F0CAF904F5944032465B465146CDF829
:103D30000080283076F044F804F594405B46324623
:103D40005146783074F050FE04F595404FF4004130
:103D500050300CF05BFE04F59640503058F020FDDA
:103D600004F59740543041F0C5FC04F597406830A5
:103D700004F5A04647F01AFF2C22394606F284408B
:103D8000A7F0ACFF1E4A1F49116004F5A943303368
:103D90004FF0140CB8B20CFB00120137127C002A51
:103DA000F8D1194A1080194A17689FB3184844E798
:103DB000C83B0C08B5370108B9370108BD37010801
:103DC0000000FFFF907F00201CB80C08980B0D0826
:103DD000E4830020F0090C08F8A00D0864230D0806
:103DE000289100206C4D0C08909F0D08989E0D089E
:103DF000C1370108F0060C08C8010C0800000000DB
:103E00005C80002024430C085A8000201880002089
:103E10008E4D0C0804F5A9404C30C6F8C074C6F8A5
:103E2000C474C6F8C804136002F0F0FA304BC6F848
:103E3000CC3404F5AA40083002F0E8FA2D4BC6F85D
:103E4000083504F5AA40443002F0E0FA2A4BC6F8DF
:103E5000443504F5AB4002F0D9FA284BC6F880355A
:103E600004F5AB403C3002F0D1FA254BC6F8BC3526
:103E700004F5AB40783002F0C9FA224BC6F8F835A9
:103E800004F5AC40343002F0C1FA1F4BC6F83436AA
:103E900004F5AC40703002F0B9FA1C4BC6F870362D
:103EA00004F5AD402C3002F0B1FA194BC6F8AC362F
:103EB00004F5AD40683002F0A9FA164BC6F8E836B2
:103EC00004F5AE40243005F0A7FCA6F86C7795F811
:103ED000D43E43F0010385F8D43E0F4B1A680AB173
:103EE0000E48AAE620461C6005B0BDE8F08F00BF72
:103EF00068530C0824550C0810510C0864510C0828
:103F000078520C0818530C08D0540C08C8520C08EE
:103F100074550C0880540C0804270020A94D0C0887
:103F200010B579F0B9FD064C064B18602046FFF736
:103F3000BBFD2046044A0549BDE81040A5F08CB9F8
:103F40001027002008270020F0DF0020C5370108D7
:103F500030B5044689B0684604F592550EF0F6F87F
:103F6000103504A80EF0F2F86946284609F01EF84C
:103F700060B104A9284609F05DF838B1059B0193AA
:103F800023680022DB6C69462046984709B030BDA3
:103F900000F5805292F8CC24D20709D400F50052E3
:103FA00092F8A71F09B1FFF7D3BF03689B6C1847AE
:103FB0007047000010B586B0044602A801910EF0CB
:103FC000C5F804F5925002A9103008F0EFFFD0B107
:103FD00094F87114DDED037A9FED0C7A019A242098
:103FE00004F58C6300FB0133D3ED0B6A2368F8EE14
:103FF000E77ADB6CE6EEC77A02A92046FDEEE77AA7
:10400000CDED037A984706B010BD00BF0000C8424E
:10401000F0B5044685B004F59256684610360F4652
:1040200015460EF093F86946304609F003F810B9CA
:10403000002005B0F0BD3946304608F09BFE002850
:10404000F6D0002DF5D004F58054284694F8CC34F1
:1040500043F0020384F8CC34EBE7000010B50A4AC1
:104060001378044600F5AB4043F080033C301370F6
:1040700003F07AFA30B920460822BDE81040022148
:1040800002F05ABA10BD00BFDC7F00202DE9F041DC
:1040900001F1080305460F460FCB88B004AC84E855
:1040A0000F0005F54056134301BFD6F8FC370693C1
:1040B000D6F800380793059BB3B920460EF076F882
:1040C00005F55F5808F13408014603AA40460EF092
:1040D00079F8C0B10399019120460EF067F8019973
:1040E000024620460EF038F80023C6F82832BB8876
:1040F000A6F8263205F5AB4021463C3002F014FF0D
:1041000008B0BDE8F081D6F8F81701914046E4E721
:1041100070B58CB00D4604AC064620460EF016F87D
:104120002B691F490BB96B693BB300230B7005F179
:1041300008010FC984E80F0006F55F5003AA0321A8
:1041400034300EF03FF890B108AA032120460EF05B
:1041500039F860B10399032220460DF0FDFF06F502
:10416000AB4021463C3002F0DFFE0CB070BD06F5DE
:1041700040530122D3F8F817EEE701220A7006F542
:104180004051009208ADD1F80028D1F8FC1728461C
:104190000DF0FCFF95E80F0084E80F00DFE700BF9B
:1041A000807E002000F5A55100F5AB401C313C306D
:1041B00002F0BABE70B5083105460FC98EB006AC24
:1041C00084E80F00134312D105F58240002303A9B0
:1041D000643003930493059374F0E8FF022203A96B
:1041E0000AA80EF0A7FA0C9B08930D9B0993079B56
:1041F000ABB920460DF0DAFF05F55F5634360146BF
:104200000AAA30460DF0DEFF88B10A9901912046D6
:104210000DF0CCFF0199024620460DF09DFF05F5FB
:10422000AB4021463C3002F07FFE0EB070BD05F57C
:1042300040533046D3F8F8170191E9E7F0B501F1A2
:10424000080305460E460FCB89B004AC84E80F0086
:10425000134307D105F54053D3F8FC27D3F80038B2
:1042600006920793059BABB920460DF09FFF05F51D
:104270005F573437014603AA38460DF0A3FF08B351
:104280000399019120460DF091FF019902462046C5
:104290000DF062FF327EB388D2074FEA132344BF8A
:1042A00003EB83035B00327A07EE903A05F5AB40EF
:1042B000B8EE670AC2F3400221463C3002F078FEB5
:1042C00009B0F0BD05F540533846D3F8F817019111
:1042D0000DF06CFF0199024620460DF03DFF4AF0BB
:1042E00059FA022215214AF00DF8D3E738B50446F1
:1042F0000D46FFF75FFF04F540500023C0F8283259
:10430000AB88A0F8263238BD10B58B8853B100F5C4
:10431000AB443C34204604F08FFA2046BDE8104000
:1043200003F090BA10BD000073B505460C467AF054
:10433000A7F805F54056C6F83002D4ED027AF5EE3E
:10434000C07AF1EE10FA17DD9FED137A67EE877AE7
:10435000FCEEE77AC6ED8B7AD6F82C2205F53250C2
:104360004FF47A73B2FBF3F30C4A0621083002B023
:10437000BDE870404DF01ABB61F070F80023009367
:1043800094F90D2094F90E3094F90C1061F002F8B4
:10439000C6F82C02E0E700BF00007A444C4E0C083F
:1043A000DFED0B7A91ED041AD1ED030A91ED020ACB
:1043B0008B8800F5AB404FF47A7121EE271A60EE3E
:1043C000A70A20EE270A5943783004F029BA00BF23
:1043D0000000C842F8B500F58043054693F86841EF
:1043E00014F001040F4602D100242046F8BD124A01
:1043F000537800F5405643F001035370D6F8283245
:104400001BB97AF03DF8C6F828027AF039F8D6F8E8
:104410002832C01A4FF47A73B0FBF3F0B6F82632A4
:104420009842E1D305F532503B88044A0621083012
:104430004DF0BCFAD9E700BFDC7F00205C4E0C08D1
:10444000F0B5144E357887B0044625B1012D1AD049
:10445000012007B0F0BD00F5804393F8682112F009
:104460000100F6D001270097D1E904122B4602A8DB
:104470000DF08CFE04F5AB403C3002A902F054FD77
:1044800037702846E5E700F5804494F8680100F0AD
:104490000100DEE7807E002010B500F58043044671
:1044A00093F8683113F0010017D004F54054D4F8A4
:1044B00028321BB979F0E4FFC4F8280279F0E0FF54
:1044C000D4F82832C01A4FF47A73B0FBF3F0B4F882
:1044D0002632984234BF0020012010BD7FB500F580
:1044E000A043054693F86C37012B0C4636D100F5F6
:1044F000804393F8680110F001002DD001AE002335
:10450000314604F108000193029303930DF0E0FF9C
:10451000DDED037A9FED207AF0EEE77AF4EEC77ACC
:10452000F1EE10FA06D505F56050303075F03AFF1F
:104530008DED030A23694BB963693BB905F56050FA
:10454000303075F02DFF03C886E8030005F5AB4059
:104550003C3002F017FD002004B070BD0B79DFED98
:104560000F6A07EE903A0B7E9B070D4B48BF9FEDFD
:104570000D7A93ED006AF8EE677A48BF67EE877AA6
:1045800086EE267AB0EEC77AB4EEE77AF1EE10FA4C
:10459000ACBF01200020DFE700000034DB0FC94082
:1045A000C07100200000803B8B8823B100F5AB4038
:1045B0003C3004F053B901207047000010B50446A8
:1045C00079F05EFF04F54053D3F83022801AD3F817
:1045D0002C2290424FF0000084BFC3F82C0201202F
:1045E00010BD000038B504460D4679F049FF04F5CA
:1045F00040539FED077AC3F82C08D5ED027A67EE99
:10460000877AFDEEE77A17EE902AC3F8282838BD9E
:1046100000007A440B464A7CD3ED030A91F910104E
:1046200093ED020A014802F0A3BD00BFCC7C00203C
:1046300010B5044679F024FF04F54053D3F82C2834
:10464000801AD3F8282822EAE27290424FF0000044
:1046500084BFC3F82808012010BD000038B500F55C
:104660004055044695F80438032B03D00A4803212B
:1046700003F06CFB04F58054D5F81C38D4F85004D2
:10468000C01A1FF025F90028B8BF4042C828CCBF87
:104690000020012038BD00BFCC7C002008B500F50B
:1046A000005393F8B43E042B07D0032B0AD100F536
:1046B000A04393F86C37032B04D14B88102B03D005
:1046C000732B07D0002008E0BDE8084003480831FC
:1046D00004F078B9FFF79EFF012008BD087D002097
:1046E000D1F8093007EE903AF5EEC07AF1EE10FA03
:1046F00008DD9FED050A00F5824027EE800A643050
:1047000074F0E8BD704700BF0000C8428B88012BE1
:10471000036805D00A6932B94A6922B9CA6812B970
:104720009B6C00211847DB6C002208311847000001
:1047300000F5804300F5964091ED041AD1ED020A90
:1047400091ED030A93F8C91B0022503058F094B839
:1047500037B501F108050446284601910DF026FD04
:10476000012801990BD1CB68002B11DD514A04F5CA
:104770003250042108304DF019F900206BE0032875
:1047800004D1CB68002B03DA4B4AF0E74B4AEEE743
:104790004B88702B74D01CD8152B12D80F2B07D830
:1047A00004F53250464A042108304DF0FFF8E4E7A2
:1047B000113B2046042B4BD8DFE803F055585B52E1
:1047C0004F005C2B58D05D2BEAD12046FFF7ACFDA3
:1047D00040E0B32B60D014D8732B55D0B22B57D0F8
:1047E000722BDDD1D1ED027A9FED367A67EE877AB2
:1047F00004F54054FDEEE77A17EE903AC4F82838F5
:1048000028E0CD2B1ED8C22BCAD9A3F1C3020A2A95
:10481000C6D801A050F822F0A1480108A14701081C
:10482000A1480108A1470108A1470108A1470108C3
:10483000A1480108A1470108A1470108A1470108B3
:10484000AB480108DE2BABD12046FFF7A9FD01E004
:10485000FFF71CFC012003B030BDFFF759FCF9E75E
:10486000FFF7A0FCF6E7FFF7A5FCF3E7FFF7E6FC90
:10487000F0E7FFF73BFDEDE72046FFF745FDE9E7F1
:104880002046FFF7AFFEE5E72046FFF7C3FEE1E76E
:104890002046FFF725FFDDE72046FFF737FFD9E782
:1048A0000948294602F0D8FCD4E72046FFF740FF2C
:1048B000D0E700BF704E0C08904E0C08B34E0C08A9
:1048C000C14E0C080000C842CC7C002010B5044644
:1048D00004F5405400F58240643074F0B5FBD4F820
:1048E000283823EAE37307EE903AF8EEE77A0020DF
:1048F000B4EEE70AF1EE10FA44BFC4F8280801202C
:1049000010BD000010B54B88152B04460A4615D87B
:104910000F2B1AD9113B042B35D8DFE803F05E4585
:104920004A3E3900A3F1C3020B2A0ED8DFE802F099
:10493000260D260D0D0D260D0D0D2626702B44D0AF
:104940000BD85C2B39D05D2B3BD004F53250244A78
:10495000042108304DF02AF810E0732B39D005D827
:10496000722BF2D1BDE81040FFF7B0BFCE2B07D8B5
:10497000C22BD7D8A3F1B202012AE6D8012012E057
:10498000DE2BFBD0E1E7BDE810401146FFF722BD6A
:10499000BDE810401146FFF753BD00F5804494F880
:1049A000680100F0010010BDBDE810401146FFF79E
:1049B00095BDBDE81040FFF76FBDBDE81040FFF7A3
:1049C000F3BDBDE81040FFF7F9BDBDE81040FFF7AB
:1049D0002FBEBDE81040FFF741BE0020E3E700BF57
:1049E000D84E0C0870B500F50053054693F8B43E58
:1049F000032B0E4602D00024204670BDFFF782FF35
:104A000004460028F7D005F532503188083051F0BF
:104A10009FF9F1E708B5044B01221A7079F024FDE3
:104A2000024B186008BD00BF827E0020887E0020F7
:104A3000014B00221A707047827E002038B500F5C5
:104A40000054054694F97632C3B179F019FDD4EDDE
:104A50009E7A05F58C6393ED097A194BF8EEE77AA7
:104A6000F4EEC77AF1EE10FA09DD1860154B186004
:104A700094F8D43E6FF3451384F8D43E38BD1B68D8
:104A800003F5FA6383423EBF94F8D43E43F020031B
:104A900084F8D43E94F8D43E9B06EFD5094A1368B7
:104AA00003F5EA4330338342E8D2106005F5325013
:104AB000054ABDE83840042108304CF077BF00BFFC
:104AC000947E0020987E0020F44E0C0838B500F546
:104AD0000054054694F97732D3B179F0D1FC94F9BA
:104AE0007C3207EE903A05F58C6393ED0A7A194B08
:104AF000F8EEE77AF4EEC77AF1EE10FA09DD186005
:104B0000154B186094F8D43E6FF3861384F8D43EA6
:104B100038BD1B6803F5FA6383423EBF94F8D43E68
:104B200043F0400384F8D43E94F8D43E5B06EFD5BE
:104B3000094A136803F5EA4330338342E8D2106030
:104B400005F53250054ABDE83840042108304CF0E4
:104B50002DBF00BF9C7E0020A07E0020104F0C08BF
:104B600070B500F50054284E94F8B63A054613B1D6
:104B700094F9743293B994F8D43ED90605D549F026
:104B800009FE00221B2149F0BDFB94F8D43E00220F
:104B900062F30413F27484F8D43E70BD0123F374FD
:104BA00079F06EFCD4F8B83E03F59C432033834281
:104BB00008D2C4F8B80E05F53250144A0221083064
:104BC0004CF0F4FE94F8D43EDA06E6D443F0100339
:104BD00084F8D43E49F0DEFD01221B2149F092FB0E
:104BE00094F8D43EDB06D8D594F97432022BD4D194
:104BF00094F8A73F002BD0D028461D22BDE8704076
:104C0000092101F099BC00BFBD7F0020304F0C0886
:104C100038B504460D4679F033FC04F500533DB930
:104C2000D3F8C42EC3F8C80E0AB9C3F8C40E38BDF1
:104C3000D3F8C82E801A642882BF0022C3F8C82E79
:104C4000C3F8C42EF3E70000F8B5044679F00CFC75
:104C5000294BB4F8BE201988284E914205460ED043
:104C60001A80274B18603378A3B10024347049F0C0
:104C700091FD22461321BDE8F84049F043BB33784B
:104C8000204FD3B93B782BB11D4B1F4A1B68C31A69
:104C9000934200D8F8BD0123337004F5005393F814
:104CA000A73F23B104F53B501C3075F0B5FC49F02B
:104CB00071FD0122132149F025FB3B78002BE9D03F
:104CC0003378002BE6D00E4A10491368EB1A8B425A
:104CD000E0D904F50053156093F8A73F002BD9D015
:104CE00004F53B541C342046002176F0F5FB2046A9
:104CF000BDE8F84077F0C6BF847E0020817E0020AA
:104D0000887E0020827E002080841E0040420F00AA
:104D100038B500F50054054694F8B13ED80714D5CF
:104D200094F8D81E94F8D53EC90703F001020DD5BA
:104D30005AB149F02FFD00221A2149F0E3FA94F804
:104D4000D53E6FF3000384F8D53E38BD002AFCD170
:104D500043F0010305F5325084F8D53E144A022190
:104D600008304CF023FE49F015FD03221A2149F0CA
:104D7000C9FA94F8B43E022B0FD11C221321284605
:104D800001F0DAFB0028E0D105F55E500122BDE814
:104D9000384017212830FCF7D7BC092BEDD0054B44
:104DA000D3F8C80403689B6898470028E5D1CCE78E
:104DB000404F0C0810770020F0B500F500543C4E31
:104DC00094F998728BB0054667B979F059FB94F85D
:104DD000D43E306067F3820384F8D43E354BDF73F2
:104DE0000BB0F0BD002307930893099307AF05AB01
:104DF00000F59250019303AA04AB06A90097103066
:104E000008F03EF8384621F053FDD4EDA77AF4EED1
:104E1000C07AF1EE10FA13DD9DED067AF4EEC77A52
:104E2000F1EE10FA0CDD79F02BFB94F8D43E3060F3
:104E30006FF3820384F8D43E1E4B0022DA73CFE76F
:104E400079F01EFB336803F5FA63984294F8D43E78
:104E5000EED35A07C4D443F0040384F8D43E154B70
:104E60000122DA7349F096FC0222102149F04AFA35
:104E700079F006FBD4F8D03E03F59C4320339842EA
:104E80000AD979F0FDFAC4F8D00E05F532500A4A75
:104E9000042108304CF08AFD94F99832022B9FD1FE
:104EA00005F55E50012218212830FCF74DFC97E7EC
:104EB0008C7E0020BD7F0020544F0C0838B515466D
:104EC000044649F067FC0122062149F01BFA022D35
:104ED00008D0032D0FD120460422BDE83840092117
:104EE00001F02ABB04F55E500122BDE838400721DD
:104EF0002830FCF729BC38BD38B500F5005405460C
:104F000094F97E3233B994F8D43E6FF3000384F8F9
:104F1000D43E38BD79F0B4FAD4F8C03E9FED1B7A88
:104F2000D4EDA06A07EE903AF8EE677AE6EE877A5B
:104F300007EE100AB8EE477AB4EEE77AF1EE10FA0F
:104F4000E1D494F8D43EDA07E3D443F0010384F8C3
:104F5000D43E49F01FFC01221C2149F0D3F905F58C
:104F600032500B4A022108304CF020FD284600F058
:104F70005DFB94F97E32022BCBD105F55E50012208
:104F8000BDE838401D212830FCF7DEBB00007A4424
:104F90005C4F0C08F8B500F50054054694F97532DD
:104FA00053B3D4F8407E3FB379F06AFA94EDA10A86
:104FB000DFED3A7A9FED3A1ADFED3A0A064620EE27
:104FC000270A4FF4A2701EF0B9FCBCEEC00AF71B12
:104FD00010EE103A9F4210D294F8D43E990705D5AE
:104FE00049F0D8FB0022082149F08CF994F8D43E0E
:104FF0006FF3410384F8D43EF8BDD4F8BC3E47F2C9
:105000003052F31A93420AD905F53250B4F964329A
:10501000254AC4F8BC6E042108304CF0C7FC94F853
:10502000D43E9A07E8D494F8A72F002AE4D043F09E
:10503000020384F8D43E49F0ADFB0122082149F077
:1050400061F994F97532022B08D10122122105F57C
:105050005E502830BDE8F840FCF776BB032B0DD13D
:1050600094F8A73F002BC7D005220221284601F063
:1050700063FA0028C0D101221A21E8E7042BBBD132
:1050800094F8A73F002BB7D005220921284601F04C
:1050900053FA0028B0D101221921D8E700007A4440
:1050A0000000804F00000000704F0C0838B5054626
:1050B00005F5005479F0E4F994F8A72F294B12B1C3
:1050C00094F999223AB9186094F8D43E6FF3C71353
:1050D00084F8D43E38BD94F8B42E012AF3D0132AB4
:1050E000F1D005F564529FED207AD2ED387A67EE63
:1050F000877AB3EE0E7AF4EEC77AF1EE10FAE2D9BF
:105100001B6803F5FA638342E4D8D4F8CC3E03F578
:105110009C432033834208D2C4F8CC0E05F53250AC
:10512000124A042108304CF041FC94F9D43E002B83
:10513000D0DB94F8D43E43F0800384F8D43E49F0A9
:1051400029FB01220C2149F0DDF894F99932022B58
:10515000C0D105F55E500122BDE838400C21283051
:10516000FCF7F2BA907E0020E02E65428C4F0C08CE
:1051700010B500F50053044693F97D32012B0AD097
:10518000022B18D000F55E50BDE810400122152119
:105190002830FCF7D9BA0B22102101F0CDF920B943
:1051A0000B220221204601F0C7F9044A137843F08C
:1051B0000803137010BD0B220921F4E7DC7F0020E7
:1051C00038B500F50055044695F8D43E43F0080381
:1051D00085F8D43E49F0DEFA0122172149F092F811
:1051E00095F8C83ADB0704D42046BDE83840FFF7FD
:1051F000BFBF034802F066F80028F5D038BD00BFF5
:10520000CC7C002070B500F50055064695F8B43EFC
:10521000D5F8C84ED5F8C42E033B012B18D8A41AD4
:10522000B4F57A7F94BF0024012495F8D43EC3F3EB
:10523000C003A3421AD06CB106F5325008300C4AB4
:1052400002214CF0B3FB3046BDE87040FFF7B8BF19
:105250000024EAE749F09EFA2246172149F052F865
:1052600095F8D43E64F3C30385F8D43E70BD00BF07
:105270009C4F0C0813B500F5005090F8A73F9BB168
:1052800090F844410948002160F0B2FD024648B15F
:10529000019249F07FFA019A092102B0BDE810405D
:1052A00049F030B8002CF3D102B010BD18480020EE
:1052B00030B500F56055303587B0044600212846EA
:1052C00075F010F802A80CF041FF04F5925002A905
:1052D00004F54054103007F069FE049BC4F8FC3715
:1052E000059BC4F80038284675F04EF8830611D5A2
:1052F000284675F057F8BDEEC00A284610EE103A61
:10530000C4F8F83775F056F8BDEEC00A10EE103A42
:10531000A4F8E03707B030BD024B014618680268B8
:1053200012681047EC83002001225BF085BC00006E
:1053300000225BF081BC00001F2900F28D80DFE8B5
:1053400001F08B1014181B1F23272B2F33373B3FE3
:1053500043474B4F53575B5F63676B6F73777B7F3D
:10536000838700F50A503C30704700F50A503E3004
:10537000704700F50B50704700F50B500230704736
:1053800000F50B500430704700F50B5006307047A5
:1053900000F50B500830704700F50B500A3070478D
:1053A00000F50B500C30704700F50B500E30704775
:1053B00000F50B501030704700F50B50123070475D
:1053C00000F50B501430704700F50B501630704745
:1053D00000F50B501830704700F50B501A3070472D
:1053E00000F50B501C30704700F50B501E30704715
:1053F00000F50B502030704700F50B5022307047FD
:1054000000F50B502430704700F50B5026307047E4
:1054100000F50B502830704700F50B502A307047CC
:1054200000F50B502C30704700F50B502E307047B4
:1054300000F50B503030704700F50B50323070479C
:1054400000F50B503430704700F50B503630704784
:1054500000F50B503830704700F50A503A3070476D
:1054600010B50446FFF768FF114674F0B1FF6B28D2
:105470000AD8672809D8512812D84F2831D8A0F166
:105480004C03DBB2012B20D910BDA0F1690304F558
:105490008E500C30022B0ED8DFE803F011131500EC
:1054A000A0F15403DBB2012BEED8114B1B680B218A
:1054B000B3F8CC200EE00021FFF73AFFE4E701212A
:1054C000FAE70221F8E70321F6E7094B1B68B3F876
:1054D000A420092104F58F501030BDE810405BF086
:1054E0001BBC034B1B680A21B3F8B820F2E700BFCE
:1054F00048840020F0B50F4B89B06A46064603F198
:105500002007144618685968154603C50833BB427E
:105510002A46F7D10025E9B23046FFF70DFF0135E5
:10552000627814F8021B74F059FF102DF3D109B002
:10553000F0BD00BF48FF0B0837B50446FFF7DAFFA0
:105540000820FFF7E9FE354B42891A800920FFF752
:10555000E3FE334B42891A8004F5005501221321E2
:10556000204600F0E9FF95F9B032002B09DC04F584
:105570000A5001230DF1070130308DF807303FF05C
:10558000B1FF95F9B02295EDA90A95EDAA1AD5EDCE
:10559000AB0A012A04F540540FD0DFED227A31EE38
:1055A000277AB4EEC07AF1EE10FA1CDD70EEE77ADD
:1055B000F4EEC07AF1EE10FA15D52D201EF0BEF9EA
:1055C00004F2EC7383ED000A04F2EC74DFED160ACA
:1055D00094ED000A3320B7EE001A1EF0AFF984ED07
:1055E000000A03B030BD02EBD2735B10013B5BB22B
:1055F00007EE903A013A31EE601AF8EEE77A07EEDC
:10560000102A67EE817AB8EEC77A04F2EC71C7EE21
:10561000876A76EEA00AC1ED000AD5E7382200209D
:105620003A2200200AD7233CCDCCCC3D38B578F0C7
:1056300027FF00240546E0B22A4640F2DC5101343F
:1056400054F086FC062CF6D1024A00231380024A4D
:10565000138038BDB67E0020B47E0020054A0023AA
:105660001380054A00F540501380044A80F8F03753
:1056700013807047A87E0020AA7E0020AC7E002008
:10568000F0B585B01D460446FFF756FE114674F08E
:105690009FFE0238692800F2CB80DFE810F06A0034
:1056A00079008300890091009400A30097009D0079
:1056B0009A00A000A600C900C900C900C900C9001D
:1056C000C900C900A900C300C600C900CB00E6009C
:1056D000E800C900C900C900EA0026014F017901AC
:1056E000A501BE01C900C900C900C900D701210236
:1056F0009602EC02F90202030B031403AB04C90087
:105700007A0364036B038B038103830397038D0385
:105710008F03C900A503BC03C703E203EF03F4032F
:105720002F043A0451045E0463047704820499044C
:10573000A604C703E203CC03E7033A0451043F0481
:1057400056048204990487049E04C900C900C90054
:10575000C900C900C900C900C900C900C900C90001
:10576000C900C900A30399039B037703880394032B
:10577000A00304F55E5004F50054012294F8A73FFD
:10578000283011464BB105B0BDE8F040FBF7DCBF57
:10579000012204F55E501146283005B0BDE8F04006
:1057A000FBF74ABF012204F55E5011462830EAE7B4
:1057B00001221321204605B0BDE8F04000F0BCBE38
:1057C00001220021F6E701220221F3E70122032151
:1057D000F0E701220421EDE701220721EAE7012297
:1057E0001146E7E701221021E4E701221521E1E754
:1057F0009FEDA91A04F5964504F58044503594F8B8
:10580000C91B28460022F0EE410AB0EE410A57F0CB
:1058100033F894F8C91B0322284605B0BDE8F040D0
:1058200057F016B89D4B9E4A01E09C4B9D4A1A606A
:1058300005B0F0BD002DFBD19B4A137804F5325022
:1058400083F0010313700830984A4BB140F26C7337
:105850001380974A062105B0BDE8F0404CF0A6B889
:1058600040F24C431380934AF4E7934BDBE7924BAF
:10587000DCE7002DDCD10820FFF74EFDC789468903
:105880008E4D07EE907A04F50050B8EE671AB0F925
:10589000B8228B4C07EE906ABB1B93FBF2F32A787D
:1058A000F8EE670A9BB2CAB1B4F90020D31800EE33
:1058B000103AF120B8EEC00A1EF040F8BDEEC00A62
:1058C00010EE103A2380B4F900309F4201DD9E4271
:1058D000AEDB2B7883F001032B70A9E7B4F900202D
:1058E000D31A00EE103AF320E4E7002DA0D10820EF
:1058F000FFF712FD4289C18904F50050704CB0F9E0
:10590000B8028B1A93FBF0F3B4F9000010FA83F39A
:1059100000EE103A4FF4807007EE901AB8EE671A56
:1059200007EE902AF8EE670AB8EEC00A1EF006F8F5
:10593000BDEEC00A10EE103A238079E7002D7FF407
:1059400077AF0820FFF7E8FC5D4D4189C689B5F9BE
:10595000002004F50050731AB0F9B80293FBF0F37D
:105960009BB2D31A00EE103A40F2091007EE906A8B
:10597000B8EE671A07EE901AB8EEC00AF8EE670A9A
:105980001DF0DCFFBDEEC00A10EE103A2B804FE791
:10599000002D7FF44DAF0920FFF7BEFCC789468973
:1059A000484D07EE907A04F50050B8EE671AB0F94A
:1059B000B822454C07EE906ABB1B93FBF2F32A78A2
:1059C000F8EE670A9BB23AB1B4F90020D31800EEA2
:1059D000103A4FF48A706DE7B4F90020D31A00EE44
:1059E000103A4FF48B7065E7002D7FF421AF09204A
:1059F000FFF792FC4289C18904F50050324CB0F99E
:105A0000B8028B1A93FBF0F3B4F9000010FA83F399
:105A100000EE103A40F223107EE7002D7FF408AF2D
:105A20000920FFF779FC284D4189C689B5F9002086
:105A300004F50050731AB0F9B80293FBF0F39BB26F
:105A4000D31A00EE103A4FF496708FE7002D7FF4D2
:105A5000EFAE1E4A137883F00103002BF6EE007AB6
:105A6000B7EE007A0CBF17EE100A17EE900A13700B
:105A700004F55F5304F53254D862FAF745FD00226D
:105A8000134BFAF799FDCDE90001124A08340621BB
:105A900020464BF08BFFCBE6000000003C220020AC
:105AA0000080ED4400808944B87E00203022002030
:105AB000B84F0C08CF4F0C083422002040220020A1
:105AC00038220020412200203A220020B97E002006
:105AD00000005940E64F0C08CDCC4C3FCDCCCC3D1E
:105AE000002D7FF4A5AE04F500551FED051A5FEDFE
:105AF000050A95EDAB0A4FF49F701DF01FFF04F5EA
:105B00000A5003A92C308DED030A3FF081FCD5ED3E
:105B1000AB0A95EDAA0AB7EE001A40F23F101DF04D
:105B20000DFF04F50A5003A928308DED030A3FF05C
:105B30006FFC0A22012195F9B0021DF03DFF8DF89E
:105B40000C0004F50A5003A930303FF0CBFC95F966
:105B5000B032012B04F540560ED140F2431095EDC2
:105B6000AA1AD5EDAB0A95EDA90A1DF0E7FE06F2DB
:105B7000EC7383ED000A18E0013B95EDAA1AD5ED10
:105B8000AB0A07EE903A31EE607AF8EEE77A06F269
:105B9000EC7587EE270A40F24510D5ED007A30EE1D
:105BA000270A1DF0CBFE85ED000A06F2EC7604F51F
:105BB00032543068FAF7A8FC0022BD4BFAF7FCFC1F
:105BC0000834CDE90001BB4A61E7002D7FF430AE17
:105BD00004F500559FEDB81ADFEDB80A95EDAB0A54
:105BE0004FF4A7701DF0AAFE04F50A5003A92C304B
:105BF0008DED030A3FF00CFCD5EDAB0A95EDAA0A3A
:105C0000B7EE001A40F24F101DF098FE04F50A504E
:105C100003A928308DED030A3FF0FAFB0A22012187
:105C200095F9B0021DF0C8FE8DF80C0004F50A507D
:105C300003A930303FF056FC95F9B032012B04F542
:105C4000405602D140F2531089E7013B95EDAA1A64
:105C5000D5EDAB0A07EE903A71EE606AF8EEE77A9E
:105C600006F2EC7586EEA77A40F2551095ED000A23
:105C700030EE470A95E7924CB4F900300A3300EE53
:105C8000103A4FF4AE709FED8F1ADFED8F0A4BE69E
:105C90008B4CB4F900300A3B00EE103A40F25F1032
:105CA000F1E78A4CB4F900300A3300EE103A4FF4B1
:105CB000B170E8E7854CB4F900300A3B00EE103AC9
:105CC00040F26510DFE704F5005393F8A73F002B7F
:105CD0003FF4AEAD002D7FF4ABAD7D4BB3F900309A
:105CE000A3F5FA7383EAE372A2EBE372322AC8BF28
:105CF0001DB2784B1D80784BB3F9002082EAE27325
:105D0000A3EBE2739BB2322B744B98BF00221A8034
:105D1000734BB3F9003083EAE371A1EBE37189B20D
:105D2000322998BF00236F4915431D430B8004F5AA
:105D3000405610D001236C4A86F8F03704F53250F3
:105D4000062108304BF032FE96F8F037674A83F0B0
:105D5000010313706CE596F8F03786F8F057002BC6
:105D6000F2D0634AEAE7002104F58E500C30FFF7C9
:105D7000DFFA5DE5002D7FF45BAD294604F58E501A
:105D80000C3005B0BDE8F0405AF064BF002D7FF440
:105D90004FAD002104F58E500C30FFF7C5FA47E5F2
:105DA0000121E1E7002D7FF443AD0121E6E7002D5D
:105DB0007FF43EAD0121EDE70221D5E7002D7FF410
:105DC00037AD0221DAE7002D7FF432AD0221E1E7A1
:105DD0000321C9E7002D7FF42BAD0321CEE7002D71
:105DE0007FF426AD0321D5E7424B1D68424B1B686B
:105DF000586A036808219B6B98473230B5F9A22096
:105E0000B5F9A01000B21DF0D7FD82B2092104F54A
:105E10008F50103020E0374B1D68374B1B68586A95
:105E2000036808219B6B98473238E7E7314B1B68C2
:105E3000B3F8A020EAE7002D7FF4FAAC2D4B1B68E5
:105E4000B3F8A020B3F8AA10914204F58F5008BF10
:105E5000B3F8A4201030092105B0BDE8F0405AF095
:105E60005BBF244B1B68B3F8A220CFE7002D7FF463
:105E7000DFAC204B1B68B3F8A220E3E71D4B1B6887
:105E8000B3F8A420C2E71B4B1D681B4B1B68586A64
:105E9000036809219B6B98473230B5F9B620B5F9F4
:105EA000B41000B21DF088FD82B20A21AFE700BF36
:105EB00000005940F54F0C08CDCC4C3FCDCCCC3D2B
:105EC000B47E002000004843000048C3B67E002096
:105ED000B27E0020AC7E0020AE7E0020A87E002096
:105EE000B07E0020AA7E002006500C08322200203E
:105EF00016500C084884002008270020474B1D68D6
:105F0000474B1B68586A036809219B6B98473238D6
:105F1000C3E7424B1B68B3F8B420C6E7002D7FF4FB
:105F200087AC3E4B1B68B3F8B420B3F8BE1004F541
:105F30008F50914208BFB3F8B82010300A218BE788
:105F4000364B1B68B3F8B620AFE7002D7FF470AC7A
:105F5000324B1B68B3F8B620E7E7304B1B68B3F849
:105F6000B820A2E72D4B1D682D4B1B68586A0368AB
:105F70000A219B6B98473230B5F9CA20B5F9C81091
:105F800000B21DF019FD82B20B2140E7234B1D68C2
:105F9000234B1B68586A03680A219B6B9847323869
:105FA000EAE71E4B1B68B3F8C820EDE7002D7FF42D
:105FB0003FAC1A4B1B68B3F8C820B3F8D21004F5F5
:105FC0008F50914208BFB3F8CC2010300B2143E72B
:105FD000124B1B68B3F8CA20D6E7002D7FF428AC1B
:105FE0000E4B1B68B3F8CA20E7E70C4B1B68B3F8ED
:105FF000CC20C9E7002D7FF41BAC04F5405204F51A
:10600000325092F8F13783F0010382F8F13708300B
:106010000BB1044A1EE4044A1CE400BF488400207B
:10602000082700202B500C083D500C082DE9F84F94
:106030002DED068B994600F55F53D3ED0BAADFEDEE
:10604000D67A9FEDD69A9FEDD68ABDF8447000F5BA
:1060500000532AEE899A6AEEA7AAD3EDAD7A6AEECA
:10606000A7AADFEDD07AF0EE488AEAEEE78A4FF091
:10607000000804460E46FDEEE88A154618EE903AF2
:106080001BB208EE903AC84B83ED008AC74B83EDF4
:10609000008ABDF84830C34647EA03474FF0010A7B
:1060A0000AFA08F33B425FFA88F109D02046FFF76D
:1060B00043F9002174F08CF9012808BF4FF0010B5F
:1060C00008F10108B8F1200FEAD1DFF80CA34FF076
:1060D0000008012303FA08F0DAF8003038425FFACA
:1060E00088F103EA000300F01E81003B18BF012382
:1060F0005A462046FFF7C4FA08F10108B8F1200F0C
:10610000E7D104F54053CAF8007093F8F127A84B83
:10611000BAB1724207EE902AF8EEE77A67EE897A12
:10612000FDEEE77A17EE902A07EE905AF8EEE77A3E
:106130001A8067EE897A9F4AFDEEE77A17EE901A89
:10614000118078F09DF99C4ADFF890821278DFF890
:1061500090A2974B07461FFA89F19848002A40F011
:10616000EA800088B8F900B000F5FA7000B20AEED3
:10617000100ABAF9000009EE900A6FF4E1700144C8
:1061800062290FD885EAE570A0EBE57080B231286E
:1061900008D886EAE672A2EBE67292B2312A8CBF88
:1061A00000220122844802701888BDF9503000F2A4
:1061B000DC50184440F26C7240F24C4100B21DF0C9
:1061C000FBFB3A460146002053F0C2FE794B18888B
:1061D000BDF9543000F2DC50184440F26C7240F2C9
:1061E0004C4100B21DF0E8FB3A460146012053F055
:1061F000AFFEB8EECAAAF8EEE88A40F26C72EAEE98
:106200002A8A40F24C4104F54054FDEEE88A18EE2B
:10621000903A18B21DF0D0FB3A460146022053F0E6
:1062200097FEBDF9403007EE103AB8EEC77AF0EEAF
:10623000487AE7EE097A40F26C7240F24C41FDEE8A
:10624000E77A17EE903A18B21DF0B6FB3A460146CF
:10625000032053F07DFE94F8F137002B7CD1F8EE4B
:10626000E99AF0EE487AE9EE897A40F26C7240F2EF
:106270004C41FDEEE77A17EE903A18B21DF09CFB08
:106280003A460146042053F063FE07EE90BAF8EE5A
:10629000E77A40F26C72A7EE898A40F24C41BDEE7B
:1062A000C88A18EE103A18B21DF086FB3A4601462D
:1062B000052053F04DFE3D4BD3ED007AFDEEE77A1D
:1062C0003A4617EE903A062019B253F041FE364B8B
:1062D000D3ED007AFDEEE77A3A4617EE903A0720C2
:1062E00019B253F035FE364B3A46B3F90010082088
:1062F00053F02EFE334B3A46B3F90010092053F009
:1063000027FE314B3A46B3F900100A2053F020FE25
:106310002E4B1E802E4B1D802E4BA3F80090BDEC03
:10632000068BBDE8F88F002B3FF4E6AE5A462046B8
:10633000FFF796F8E0E60288B8F800B011440AB218
:106340000AEE102ABAF800203244AB4412B209EE29
:10635000902A0FFA8BFB27E7BAF9003007EE103AC4
:10636000B8EEC77AF0EE487AE7EE097A40F26C723E
:1063700040F24C41FDEEE77A17EE903A18B21DF06C
:106380001BFB3A460146042053F0E2FDB8F9003009
:1063900007EE903A7BE700BFCDCC4C3FCDCCCC3E56
:1063A0000080BB440000FA433C220020342200203D
:1063B000B67E0020B47E002032220020AC7E002079
:1063C000382200203A22002030220020AE7E002019
:1063D000B07E0020B27E0020A47E0020AA7E002095
:1063E000A87E0020012070470020704700207047E1
:1063F0000020704700207047002070479FED010A81
:10640000704700BF0000000070470000134A0260A0
:10641000134A426002F1BC0181601249C160124915
:10642000016102F67C41416102F62C01816102F5B5
:106430000361C16102F63401016202F63801416272
:1064400002F63C0102F50462C262084A0263A2F548
:1064500089624263064A816282637047C8500C08B1
:1064600070490020405F00206039002060640020F7
:1064700028280020152937D8DFE801F00F1317224C
:106480002636362A362E3636363636361E36360B13
:10649000321A00F5A9404C30704700F5AA40083088
:1064A000704700F5AA404430704700F5AB40704794
:1064B00000F5AE402430704700F5AC4034307047F2
:1064C00000F5AB403C30704700F5AB40783070478A
:1064D00000F5AC407030704700F5AD402C3070478F
:1064E00000F5AD40683070470020704700F5A040CF
:1064F000D0F8C80403685B681847000038B500F599
:10650000A0450446D5F8C80403685B699847094B61
:1065100004F50052187492F8B42ED5F8C804DA7055
:1065200003681B6A9847014604F59050BDE838405F
:106530003AF00ABBBD7F00202DE9F04700F5005975
:10654000064699F8B43E8B420F46924605D189F82B
:106550001C2201252846BDE8F087FFF78BFF044683
:1065600020B9304646F0E4F82546F3E703689B6817
:10657000984706F5325808F10808A8B1314804F0E8
:1065800095F9054680B923682046DB6998472E4A6D
:106590000346042140464BF009FA48F0FBF83A461E
:1065A0000A2147F0AFFED5E72648FBF733FA50B390
:1065B000236800211B68204698470546002839D0EB
:1065C00006F5804306F5964093F8C91B503056F007
:1065D00031F999F8B43E89F8B53E06F5A043524624
:1065E000C3F8C844394606F57F6089F8B47E89F857
:1065F0001CA247F097FA4046002152F0A9FE30460F
:10660000FFF77CFFA6E706F5A043D3F8C8040368AC
:10661000DB6898470028CBD023682046DB68984782
:1066200005460028C4D123682046DB699847074AFD
:106630000346AEE723682046DB699847044A0346D1
:10664000A7E700BF1027002050500C0879500C0815
:10665000A2500C080148FFF76FBF00BF10270020B1
:106660002DE9F04F07EE902A2DED048BF8EEE78A26
:1066700007EE901AB8EEE78A95B028EE080A4FF0B8
:10668000000BA8EEA80A0646884615461F46CDF818
:1066900008B0CDF80CB0CDF810B0CDF814B0CDF8EE
:1066A00018B0CDF81CB0A3F069FADFEDBB9AB4EED8
:1066B000E90AF1EE10FA10DDC9EE807A27EE888A39
:1066C00067EEA87ABDEEC88AFDEEE77A18EE103ABA
:1066D0000FFA83F817EE903A1DB2736807EE908AAE
:1066E00093ED2C7AB8EEE79AB5EEC07A07EE905AA1
:1066F000F1EE10FAF8EEE75A00F29A8093ED278A4D
:1067000028EE099A28EE258A736807EE907A93EDB1
:10671000280A93F9AC30F8EEE78A68EE808A002BFD
:1067200078D03369D3F8F8011DF0D2F89B4940F6D0
:10673000B83281461DF030F9434207EE903A736853
:10674000F8EEE77A93ED297A336967EE877AD3F822
:10675000FC01CDED027A1DF0BBF840F6B8328F494E
:1067600082461DF019F942427368CDF810B007EE69
:10677000102AD3ED2A6A93F9AC20B8EEC77A022A20
:1067800027EE267A8DED037A1ED1854AB2F95C4256
:106790004C457ADAA9EB040907EE909AD3ED295A11
:1067A000B8EEE76ADDED027AE5EEC67ACDED027A63
:1067B00054457BDAAAEB040407EE904AF8EEE77A38
:1067C000A6EEE77A8DED037AD6F834C00CF1840397
:1067D0000FCB10AC84E80F000DF1300908AC89E84C
:1067E0000F0084E80F0005AB02AA214660466FF057
:1067F0000DF9736893F9AC30022B5CD1DDED057AAD
:1068000039EE279ADDED067A38EE278ADDED077A34
:1068100078EEA78A229B83ED009A239B83ED008A62
:10682000249BC3ED008A15B0BDEC048BBDE8F08F4E
:10683000F7EE007AB4EEE77A89EE297A85EEA98A36
:10684000F1EE10FAC8BFC3ED2C7A7368D3ED2C6A51
:1068500093ED270A77EEE67A27EE076A27EE879A06
:1068600026EE076A28EE087A67EE887A27EE087A1D
:10687000A6EE869AE6EE877A29EE299A27EEA98A6D
:1068800029EE009A28EE008A3EE762424A458FDDF3
:10689000A14407EE909A9DED026AD3ED295AF8EED5
:1068A000E77AA5EEE76A8DED026A81E76342534518
:1068B0008ADD544480E7002D88EAE871B8BF6D4254
:1068C000A1EBE87189B2ADB2A9420191D4BF2146D2
:1068D00001A90895002FB8BF7F420B68DFED310A90
:1068E000BFB29F42A8BF49460C97D1ED007AF8EE9F
:1068F000E77AB7EE001A87EEA90A4FF4827031EEFC
:10690000400A1DF01BF83369D3ED937A05A820EEF9
:10691000270A1FF0CFFBF0EEC07A8DED071AB0EE1C
:10692000C91A31EE671A8DED050AB0EEC11A30EEC4
:10693000090ACDED060A4FF48670F1EE410A1CF00B
:10694000FDFFB0EE409A9DED060AB0EEC81AF0EEDB
:10695000C07A31EE671A30EE080AB0EEC11AF1EED5
:10696000410A40F211101CF0E9FFB0EE408A9DEDA3
:10697000070AB0EEE81AF0EEC07A31EE671A38EE88
:10698000800AB0EEC11A4FF48B70F1EE410A1CF090
:10699000D5FFF0EE408A3DE700A08C4548F4FFFFAC
:1069A00010470020000000000148FFF7C5BD00BFF0
:1069B000102700200048704798530020002070479F
:1069C0000120704701207047002070470048704741
:1069D00000510C080048704700510C0808B5036BC3
:1069E00003480022C3F85423FEF720FE012008BD0F
:1069F0001027002070B50446406990F8CB3088B06D
:106A000093B9012174F078FD606B62680368D2ED80
:106A1000020A5B6E9FED240A01219847606B08B063
:106A2000BDE870406FF0C0BB022174F065FD636A81
:106A3000E269A1691B6812680968B2F90820B1F916
:106A40000810B3F9083007A8029006A8019005A81D
:106A500000902046FFF704FE606B9DED071A036867
:106A6000DDED060A9DED050A9B6B9847656B2B686B
:106A70005E6E236A186853F0FFFB63680021D3ED54
:106A8000020A2846B047A36A6569186853F0F4FB08
:106A900085ED0E0AE36A6569186853F0EDFB85ED34
:106AA0000F0A08B070BD00BF000000000020704752
:106AB0000020704701207047002070470048704751
:106AC00048510C080048704754510C0870B50446F2
:106AD0002148FAF79FFF054600283AD01E48266B4A
:106AE000FBF71CFB6368B3F93020B3F92C3000EEE0
:106AF000903A434201EE102A00EE103AB8EEC11A65
:106B0000F8EEE00AB8EEC00A304670F077FC1248A2
:106B1000266BFBF703FB6368B3F93020B3F92C3025
:106B200000EE903A434201EE102A00EE103AB8EE21
:106B3000C11AF8EEE00AB8EEC00A304670F0D8FC90
:106B4000206B71F053FD2369D3F80022034BC3F887
:106B5000B424284670BD00BF102700201077002005
:106B600070B52DED028B8AB0044677F089FC06469D
:106B70007748256BFBF7D2FA6368B3F93020B3F995
:106B80002C3000EE903A434200EE103A01EE102A0B
:106B90002846B8EEC11AF8EEE00AB8EEC00A70F066
:106BA0002DFC60696B4D90F8CB30EBB9012174F08E
:106BB000A3FC606B62680368D2ED020A5B6E012180
:106BC000B6EE000A9847606B6FF0EEFA6069266BCC
:106BD00003681B699847304671F084FD2369D3F838
:106BE0000032C5F8B43496E0022174F085FCD5F883
:106BF000843441F28732F31A934237D805F28C433A
:106C000003A91B68069305F5926306A81B68079302
:106C100005F2944305F593651B6808932B68099367
:106C200004AA05AB1EF05EFC9FED4B7ADDED037A06
:106C3000DDED040A9DED051A606B9FED480A67EED5
:106C4000877A60EE870A21EE071ACDED040A8DEDF2
:106C5000051ACDED037A036821EE001A60EE800A72
:106C60001B6B27EE800A0121984754E0A369606BF3
:106C70001B68B3F9083008EE103AE3691B68B3F9F2
:106C8000083000EE903A0368F8EEE00A9B6ECDED16
:106C9000010A9847B8EEC88AB0EE401ADDED010A45
:106CA000B0EE480A04AA03A9A5F5A040FBF732F903
:106CB000636A1868438A828907EE903A284BF8EE97
:106CC000E77A93ED007A67EE877AFCEEE77A17EEC3
:106CD000903A99B253F066FA0146A5F5A040FBF749
:106CE00083F9DFED207A606BB0EEC07AB4EEE77A1C
:106CF000F1EE10FAB0EE401A11D40368DDED040A8B
:106D0000DB6A9DED030A98472369D3F80032C5F882
:106D1000B434C5F8B8640AB0BDEC028B70BDD5F8C8
:106D2000B83402689DED030ADDED040AFA33B3427C
:106D300004D9D36A9FED0C1A98474FE705F2B44384
:106D400093ED001A136BB8EE411A01218CE700BFD6
:106D50001027002010770020E02E65420000C84276
:106D6000FC5E0020000000340000000038B5836A9B
:106D700045690446186853F07FFA85ED0E0AE36A08
:106D80006569186853F078FA85ED0F0A38BD000080
:106D900030B52DED028B036A1B68B3F9083000EEA5
:106DA000103A83B00446B8EEC00A2F48FBF7C8F982
:106DB0002D488DED010AFBF7B1F963689DED010ADD
:106DC000B3F92C3001EE103A434200EE903AB8EE9F
:106DD000C11AF8EEE00A6C201CF0B0FDDFED237A5A
:106DE000B0EEC07AB4EEE77AF1EE10FAB0EE408A77
:106DF00019D51F4B256B93F8B02E93F9B03E002B9D
:106E00001EDA636895EDD57AD3ED2D7AF1EE046A3A
:106E100077EEE67AF4EE477AF1EE10FAC8BFF0EEBC
:106E2000477AC5EDD57A206BB0EE480A70F06CFB5E
:106E3000206B03B0BDEC028BBDE8304071F0C4BCE8
:106E40005306F0D5E06873F0ADFA236BF2EE047AE6
:106E500030EE270AD3EDD57AB4EE670AF1EE10FAD8
:106E6000C8BFF0EE407ADCE710270020CDCC4C3DC7
:106E70001047002010B50446FFF772FE2046FFF7CA
:106E800087FF2046BDE81040FFF770BF0120704724
:106E90000120704700207047012070470120704793
:106EA000004870479C510C08004870479C510C08E2
:106EB00030B5054685B0174803F0F8FC044620B30A
:106EC000154BB3F8802B012A22D903F5405203F564
:106ED0008053042193F8043882F86C17022B03D1F5
:106EE0000021284600F032FFDFED0C0A0C48B0EE1E
:106EF000601AF0EE601AB0EE600A72F09BFD284650
:106F000000F01AFF074822F03FF9204605B030BDD7
:106F10000024FAE71027002010470020000000009E
:106F2000746800205C52002070B5144C05460026A1
:106F3000A4F69C6084F86C6772F0E2FC60B92846A5
:106F4000FFF738FD0E4A04214AF030FDA4F5A040B9
:106F5000BDE87040FEF734B9A4F5005494F8043845
:106F6000022B09D03146284600F03CFE0146284657
:106F7000BDE8704000F0EABE70BD00BF1077002091
:106F8000A4510C08094B03F5A042022103F58043EC
:106F900082F86C1703F6A42203F6942192ED000AFE
:106FA00093F8C82AA1F11C0071F0B2BE102700208E
:106FB000F0B52DED028B0446B0EE408A4648DFED79
:106FC000478A8FB00E46174671F024FDF0EEC87A5E
:106FD000F4EEE87AF1EE10FA06D49FED410A3E484D
:106FE00028EE000A71F07CFD3E4D95ED000AA5F6F5
:106FF000A425B0EEC00A0FB1B1EE400A364871F0D8
:107000005FFD00233448079302AA07A90893099358
:1070100071F076FDDFED347A9DED027AB4EEE77A19
:10702000F1EE10FA54DD314F0123022207A90AA81C
:1070300087F86C370BF07EFB7168019130460BF0DE
:10704000B5F8019902460AA80BF086F80AA9A7F636
:107050009C6072F055FC18B9A7F5A040FEF7B0F897
:10706000E06873F09DF903A902684368204804931F
:1070700003921EF09DFC05A88DED050ACDED060AD4
:107080001EF064FD05F52A63D3ED007AF4EEE87A8C
:10709000F1EE10FABCBF05F68825D5ED007AF4EEC6
:1070A000C07AF1EE10FA4FF0000120460AD5DFED6C
:1070B000117AB4EEE70AF1EE10FA03DD00F092FD6A
:1070C0000146204600F042FE0FB0BDEC028BF0BD41
:1070D0002046FFF757FFF7E78871002000000034D3
:1070E0000000C842B47100200000964310770020D1
:1070F000A47100200000FA4337B59FED1A0A1A4D1B
:1071000004461A4871F09EFE01462846FDF780FDB0
:10711000694601AA284602F0C9FD6369009ADA634C
:107120006369019A9A63206B71F04EFBE369606BAF
:107130001B68B3F9083000EE903AA3691B68B3F9F5
:10714000083000EE103A036805F595451B6B95ED88
:107150000A1AF8EEE00AB8EEC00A0121984703B017
:1071600030BD00BF00000000102700208871002003
:10717000F0B52DED028B0446406B264D85B0F0EE48
:10718000408A6C309FED240AB0EE608A0E461746A6
:107190001EF090FFDFED217A8DED031AF7B928EE8E
:1071A000A70A1CF061FB9FED1E7ABDEEC00AF0EE4F
:1071B000C87A10EE103AF4EEC77AF1EE10FAC5F87C
:1071C0001C3818D53C2303212046A5F8203805B0EB
:1071D000BDEC028BBDE8F04000F0B8BD9DED030AA8
:1071E000BDEEC00A002EB8EEC00AB8BFF1EE688A44
:1071F000A8EEA70AD5E7DFED0B7AB4EEE78AF1EE49
:1072000010FA58BFB0EE678ABDEEC88A18EE103A81
:10721000D9E700BF105700209F0CB3450000C842BB
:107220000000003400007042DFED097A094BB4EE33
:10723000E70AF1EE10FA58BFB0EE670ABDEEC00AD9
:10724000072110EE102AA3F8202800F07FBD00BF10
:10725000000070421057002070B54B68164D06466E
:107260000C468BB98B687BB9C96869B900F0BAFC68
:107270000146304600F06AFD95F8C91B05F53560FA
:10728000BDE8704055F020BC95F8C91B0B4855F07F
:10729000C5FA40B90A4920460BF01AF918B1022183
:1072A000304600F053FD95F8C91B04482246BDE85E
:1072B000704055F0FDBB00BF1067002060720020D9
:1072C000185F002070B51921054624483EF016FDD0
:1072D000023802283FD8224C052384F86C3777F017
:1072E000CFF8C4F8BC041F481FF04CFBDFED1E0AAA
:1072F000A4F5BB60B0EE600A72F07AFDA4F5BB6045
:1073000072F054FE68692E6B03681B699847A4F5F8
:107310008054304671F0E6F994ED610A94ED651AF7
:10732000D4ED600A286BB0EEC00A70F067F894EDF7
:10733000610A94ED651AD4ED600A286BB0EEC00ABC
:1073400070F0D6F82846FFF735FB084A04214AF0CA
:107350002DFB012070BD0020FCE700BF5034002051
:10736000107700205C52002000000000D0510C0873
:10737000F0B52DED028B0446406990F8CB3085B016
:10738000FBB9012174F0B8F8606B62680368D2ED54
:10739000020A5B6E9FED680A01219847606B6EF0F0
:1073A00003FF664872F002FE6069256B03681B6983
:1073B0009847284605B0BDEC028BBDE8F04071F05F
:1073C00091B95F4819213EF099FC032864D0042844
:1073D0006BD002285B4D40F09F805B4B93ED608A41
:1073E00000232B60594D77F04BF8D5F8BC3403F5EA
:1073F0001C53103398420AD92046FFF7DBFA544A4F
:1074000002214AF0D3FAA5F5A040FDF7B1FE4B48A2
:10741000012172F05DFF694601AA4E4802F000FCAE
:107420006369009ADA636369019A9A63B0EE480A65
:10743000206B9FED418A70F067F8206B71F0C4F902
:1074400045488DED028AB0F95C328DED038A01EE7C
:10745000103AE3691B68B3F9083000EE903AA3696B
:107460001B68B3F9083000EE103AB8EEC11AF8EE16
:10747000E00AB8EEC00A03AA02A9A0F50050FAF784
:1074800049FD606BDDED030A03689DED020ADB6ACE
:10749000B0EE481A98474BE02B4B93ED618A294B8D
:1074A0000022B0EEC88A1A609CE72B4E96F8C83AC4
:1074B0009B072ED5234D2B6853B976F0E1FF28604A
:1074C0006069276B03681B699847384671F00AF9B1
:1074D00076F0D6FF2B6803F2DC53984219D9204688
:1074E000FFF768FA1D4A06214AF060FA194801219F
:1074F000FDF78EFB96F8D43E19486FF3C30386F868
:10750000D43E124B042283F86C2721F0CFFD0023D8
:107510002B609FED098A65E72046FFF74BFA114A79
:1075200002214AF043FA0B48FDF722FE00232B60AC
:1075300005B0BDEC028BF0BD0000000038710020EA
:1075400050340020BC7E00201067002010770020FF
:107550004D520C081027002010470020F4510C0851
:107560005C5200201A520C087FB505460F4803F004
:107570009DF90446B0B10E4E042386F86C3701A97C
:107580000023A6F69C6001930293039371F01EFE04
:1075900001A90022A6F69C6072F02CFB002128466F
:1075A00000F0D4FB204604B070BD00BF10270020BF
:1075B0001077002070B52DED028B0446406990F8DD
:1075C000CB3088B03BBB012173F096FF606B9FED21
:1075D000508A62680368D2ED020A5B6EB0EE480A18
:1075E00001219847606B6EF0DFFD4A488DED058AFA
:1075F000F0EE480AB0EE481AF0EE481AB0EE480A2B
:107600008DED068A8DED078A08B0BDEC028BBDE8D2
:10761000704072F00FBA404E96F8D41E11F001057A
:107620005DD1636A1B68A6F50050B3F90810FAF73C
:10763000DBFCDFED3A7AB0EEC07AB4EEE77AF1EE39
:1076400010FAB0EE408A03D42946204600F07EFBB3
:107650000221606973F050FF2E4872F0D1F80146A4
:107660002F48FDF7D5FA02A92D4803AA02F0D8FA4F
:107670006369029ADA636369039A9A63206B71F013
:10768000A3F8B6F95C32264801EE103AE3691B68AC
:10769000B3F9083000EE903AA3691B68B3F90830DB
:1076A00000EE103AB8EEC11AF8EEE00AB8EEC00AE1
:1076B00005AA04A9FAF72EFC1A4B656B93F8043857
:1076C00083B92B68DDED050ADB6A9DED040AB0EE97
:1076D000481A2846984708B0BDEC028B70BD9FED54
:1076E0000C8AB5E72B68DDED050A9DED048ACDED2A
:1076F000010A20461E6B00F0E9FDDDED010AB0EE47
:10770000401A0121B0EE480A2846B047E3E700BF1F
:1077100000000000746800201047002000000034C2
:10772000102700201057002030B52DED028B0446A5
:10773000406990F8CB3087B03BBB012173F0DCFE91
:10774000606B9FED3C8A62680368D2ED020A5B6E53
:10775000B0EE480A01219847606B6EF025FD36486F
:107760008DED038AF0EE480AB0EE481AF0EE481AA2
:10777000B0EE480A8DED048A8DED058A07B0BDECA8
:10778000028BBDE8304072F055B92C4D95F8D43ECF
:10779000DB074BD4636A1B68A5F50050B3F90810EA
:1077A000FAF722FCB0EE408A6069022173F0A4FE71
:1077B000214872F025F801462148FDF729FA69466B
:1077C00001AA1F4802F02CFA6369009ADA63636920
:1077D000019A9A63206B70F0F7FFB5F95C32184894
:1077E00001EE103AE3691B68B3F9083000EE903AF5
:1077F000A3691B68B3F9083000EE103A03AA02A986
:10780000B8EEC11AF8EEE00AB8EEC00AFAF782FB49
:10781000606BDDED030A03689DED020ADB6AB0EEE2
:10782000481A984707B0BDEC028B30BD9FED018A26
:10783000BAE700BF00000000746800201047002075
:107840001027002008B50748012101F0ABF8064BCE
:10785000032283F86C2703F2BC50BDE8084000F017
:10786000EBBF00BF087D00201077002010B5044654
:10787000134821F025FB134B93F86C37052B1DD8CB
:10788000DFE803F00303080D12172046BDE810409F
:10789000FFF790BE2046BDE81040FFF72DBCBDE8C5
:1078A0001040094801F052BA2046BDE81040FFF7E9
:1078B0003BBF2046BDE81040FFF75ABD10BD00BFDA
:1078C0005C52002010770020087D002001207047C6
:1078D0000020704701207047012070470048704722
:1078E000B0520C0800487047B8520C0870B52DED26
:1078F000028B614DDFED618AD5ED637ADFED600AC1
:1079000095ED5F0AF4EEE87AF1EE10FA0446A8BFAE
:10791000F0EE670A82B0006B6FF028FCA5F580409E
:10792000266BFAF7FBFB6368B3F93020B3F92C3010
:1079300000EE903A434200EE103A01EE102A304633
:10794000B8EEC11AF8EEE00AB8EEC00A6FF056FDC4
:10795000606990F8CB30C3B9012173F0CDFD606B45
:1079600062680368D2ED020A5B6E9FED460A012150
:107970009847606B6EF018FC05F6782002B0BDECFD
:10798000028BBDE8704071F0DFB9636A1B68A5F532
:107990008040B3F90810FAF727FBF0EEC07AF4EE56
:1079A000E87AF1EE10FAA5F580565CBF012386F85F
:1079B0001C32236A34481B68B3F90830B0EE408AA1
:1079C00000EE103AB8EEC00AFAF7BAFB022160697D
:1079D000F0EE408A73F090FD9FED2A0A2B4871F07B
:1079E00031FA01462848FDF713F9274801AA6946EC
:1079F00002F05CF96369009ADA636369019A9A6339
:107A000096F81C12606BD4E90632F1B112681B685B
:107A1000B2F90820B3F9083000EE902A00EE103ACF
:107A20000368F8EEE00ADB6AB8EEC00AB0EE481A66
:107A30009847206BB0EE680A6FF066FD206B70F01F
:107A4000C3FE02B0BDEC028B70BD12681B68B2F9B8
:107A50000820B3F9083000EE902A00EE103A0368CF
:107A600005F6A8251B6B95ED001AF8EEE00AB8EEB6
:107A7000C00A01219847DCE71067002000000034AD
:107A800000007A43000000001027002088710020C9
:107A9000F8B504462DED028B334802F007FF05468A
:107AA00000285CD0314EDFED328A9FED328A06F538
:107AB0008057D7ED630A97ED5F0A0023F4EEE80ADA
:107AC00086F81C32F1EE10FAB8BFF0EE480A206BCF
:107AD0006FF04CFBD7ED630A97ED5F0A206BF4EE75
:107AE000E80AF1EE10FAB8BFF0EE480A6FF0B6FB04
:107AF000A6F54050276BFAF711FB6368B3F9302005
:107B0000B3F92C3000EE903A434201EE102A00EE19
:107B1000103AB8EEC11AF8EEE00AB8EEC00A3846DC
:107B20006FF06CFCA6F54050276BFAF7F7FA636824
:107B3000B3F93020B3F92C3000EE903A434201EE15
:107B4000102A00EE103A3846B8EEC11AF8EEE00AF4
:107B5000B8EEC00A6FF0CCFC074871F0F5F8BDEC48
:107B6000028B2846F8BD00BF1027002010570020C8
:107B70000000003400007A43887100200120704723
:107B8000002070470120704701207047004870476F
:107B900000530C080048704708530C0890ED007A19
:107BA000DFED0F7AB0EEC77AB4EEE77AF1EE10FAB5
:107BB00014D590ED017AB0EEC77AB4EEE77AF1EE23
:107BC00010FA0BD590ED027AB0EEC77AB4EEE77AF0
:107BD000F1EE10FA4CBF01200020704700207047E2
:107BE00000000034436893F92930042B0BD8DFE8F8
:107BF00003F00C0A050308000420704781F001001F
:107C00007047062070470120704700207047000031
:107C100038B52DED048B0446406990F8CB30B3B9EC
:107C2000012173F069FC606B62680368D2ED020A9F
:107C30005B6E9FED3D0A01219847606B6EF0B4FAD0
:107C4000BDEC048B206BBDE8384070F0CFBC374DE5
:107C500095ED028AD5ED018A28EE080AA8EEA80A59
:107C6000A1F08CFF606B03689B6EB0EE409A984762
:107C70002F4BB3F95C3207EE903AF8EEE77AB4EEA8
:107C8000E70AF1EE10FA58BFB0EE670AB4EEC90A7F
:107C9000F1EE10FA48BFC0EE097A95ED030A44BF31
:107CA00028EE278A68EEA78A1BF0F4FD214BD3ED5E
:107CB000610A93ED601AF0EEE00AF1EE600AF0EE70
:107CC000409A4FF4307095ED040A1BF037FEB0EE89
:107CD000409A76F0D5FB2B68C01AB0F57A7F88BF42
:107CE0009FED118A60694FF0020184BFB0EE489A9F
:107CF000F0EE488A73F000FC606B0368B0EE691A1E
:107D00001B6BF0EE480AB0EE680A01219847206B21
:107D1000B0EE490A6FF0F8FBBDEC048B206BBDE8B8
:107D2000384070F051BD00BF00000000C47E00204C
:107D30001047002010670020034B00221A60002229
:107D40005A609A60DA607047F07E00200C4B93F81E
:107D500004288A420FD0022983F8041802D004298B
:107D60000AD0704703F614030269D2ED807AF8EE68
:107D7000E77AC3ED007A704703F62403F4E700BF07
:107D8000105700202DE9F0412DED048B82B088467C
:107D90001446F0EE608A0193B0EE408A074605F083
:107DA00057FB9FED279A90ED830A264D1BF09CFD13
:107DB00028EE098AF0EE409AB0EE480A1BF094FDD6
:107DC00030EE690A1BF0A6FDB5EEC00AF1EE10FA1E
:107DD0004CBF4FF0FF360126B8F1000F16D0019AC4
:107DE00071B26CB9DFED180A85F805481748B0EE96
:107DF000480A02B0BDEC048BBDE8F041FFF7B8B90A
:107E0000002368EE890A85F80538EFE764B128EEAB
:107E1000890A0E48012385F8053802B0BDEC048BB1
:107E2000BDE8F041FFF700BA2146384685F805481D
:107E300002B0BDEC048BBDE8F041FFF787BF00BF87
:107E40000AD7233C1057002000000000CC7C002003
:107E500070B5244D05F5A0430122044683F86D2733
:107E6000066B2846FAF75AF96368B3F93020B3F97C
:107E70002C3000EE903A434201EE102A00EE103A08
:107E8000B8EEC11AF8EEE00AB8EEC00A30466FF05C
:107E9000B5FA2846266BFAF741F96368B3F9302042
:107EA000B3F92C3000EE903A434201EE102A00EE76
:107EB000103AB8EEC11AF8EEE00AB8EEC00A304641
:107EC0006FF016FB206B70F091FB05F54055206BB1
:107ED00070F026F9002185F805182046BDE87040AD
:107EE000FFF734BF1027002038B50A4B93F86D37E1
:107EF000012B05460C4601D0FFF7AAFF76F0C0FA29
:107F0000054B186094E807002B6B03F5597383E861
:107F1000070038BD10770020C07E002030B50C4629
:107F200011461A46134B93F86D37012B85B0054661
:107F30000DD0CDED030A02928DED010A0091FFF7FD
:107F400087FFDDED030A029A9DED010A00999DF875
:107F500020302846FFF716FF76F092FA064B18609D
:107F600094E807002B6B03F5597383E8070005B00D
:107F700030BD00BF10770020C07E002070B5174EC6
:107F800006F5804506F5A043022295ED610A83F8C7
:107F90006D27044695ED651AD5ED600A006BB0EECD
:107FA000C00A6FF02BFA95ED610A95ED651AD5EDD3
:107FB000600A206BB0EEC00A6FF09AFA206B70F086
:107FC00015FB06F54056206B70F0AAF8002186F8E4
:107FD00005182046BDE87040FFF7B8BE1027002006
:107FE0002DE9F04F2DED028B89B00746154604A808
:107FF00002220C460AF09EFB284804A95DF056FDBB
:10800000814658B946F0C6FB0522162146F07AF99A
:10801000484609B0BDEC028BBDE8F08FDFF890A0B8
:108020009AF86D37022B02D03846FFF7A7FF76F09B
:1080300027FA1B4B1B4E216862681860A368B36067
:108040003160726095E80700DFF868809FED168A5E
:108050004FF0010B88E8070002AB386BCDF800B099
:10806000424631468DED028A8DED038A6FF0FEF8AF
:10807000B368386B029308F108025B4602A9B0EEC0
:10808000480A6FF0C1FF029BB3609AF86D1707486A
:108090002B462246FBF786FABAE700BF18480020B5
:1080A000C07E0020D87E00200000000010270020A5
:1080B00010770020E47E00202DE9F04F2DED028B9B
:1080C00089B00746154604A802220C461E46B0EEAB
:1080D000408AF0EE608A0AF02DFB2E4804A95DF07C
:1080E000E5FC814658B946F055FB0522162146F0BD
:1080F00009F9484609B0BDEC028BBDE8F08FDFF806
:10810000A8A09AF86D37022B02D03846FFF736FF49
:10811000F0EE680AB0EE480A9DF854309DF8502001
:10812000DFF888809FED1C8A31463846FFF72AFE2B
:1081300076F0A6F9194B1A4E216862681860A36898
:10814000B3603160726095E807004FF0010B88E87A
:10815000070002AB386BCDF800B0424631468DEDDA
:10816000028A8DED038A6FF081F8B368386B029351
:1081700008F108025B4602A9B0EE480A6FF044FF1E
:10818000029BB3609AF86D1706482B462246FBF710
:1081900009FAAEE71848002000000000C07E002069
:1081A000D87E00201027002010770020E47E0020D9
:1081B00070B5224E06F5804506F5A043032295EDE5
:1081C000610A83F86D27044695ED651AD5ED600ABE
:1081D000006BB0EEC00A6FF011F995ED610A95EDF4
:1081E000651AD5ED600A206BB0EEC00A6FF080F919
:1081F000206B70F0FBF976F043F92269104BD2ED59
:108200007E7A1860F8EEE77A06F54056C3ED017AFB
:10821000D2ED7F7AF8EEE77A0021C3ED027AD2ED53
:10822000807A86F80518F8EEE77A0022C3ED037A23
:108230001A612046BDE87040FFF788BD1027002076
:10824000C47E002038B52DED028B1C4B93F86D37A2
:10825000032B0D46B0EE408A01D0FFF7A9FF184C62
:10826000284604F10C0304F10802211D1DF03AF91F
:10827000DFED146AD4ED017A9FED137A94ED030AD1
:1082800067EEA67A20EE260A67EE877A20EE070AC6
:10829000C4ED017AD4ED027A67EEA67A67EE877AAA
:1082A000C4ED027A1BF0F6FA84ED048A84ED030A29
:1082B00076F0E6F8BDEC028B206038BD1077002028
:1082C000C47E0020E02E65420000C84230B52DED8E
:1082D000028B3C4A92F80438023B83B00446042BDC
:1082E0006AD8DFE803F0030B151D2000364803B001
:1082F000BDEC028BBDE83040F9F79ABE02F61C03D4
:1083000093ED000AB8EEC00A03B0BDEC028B30BD9D
:108310002D4803B0BDEC028BBDE83040F9F7ACBE90
:1083200092ED880AEEE72949DFED298AA1F10C00D8
:108330001BF0E8FC236BD3E9DC016D4685E8030004
:108340002846B0EE408A1DF001FC236B9FED217A98
:10835000D3EDC27A67EE877AB4EEE70AF1EE10FA4F
:1083600027DB28461DF0A8FBDFED1B7A20EE270A4D
:10837000F0EE487AD0EE287AB0EE670A1BF08AFA5F
:10838000636893F9283007EE903A5B4200EE903A2A
:10839000B8EEE71AF8EEE00A21EE281A60EEA80A15
:1083A0004FF44D701BF0CAFA38EE000A1BF05CFA6D
:1083B000AAE79FED0A0AE3E7094BD3F8743193ED7E
:1083C000D10AA1E7105700201027002008710020D3
:1083D0000000C842CDCCCC3DE02E6542000000003C
:1083E0001067002070B52DED028B0446406990F8AF
:1083F000CB3084B0D3B9012173F07EF8606B626832
:108400000368D2ED020A5B6E9FED6C0A012198476A
:10841000606B6DF0C9FE206B70F0E8F8206B04B063
:10842000BDEC028BBDE870406FF07ABE644890F8F6
:10843000D41E11F0010500F580566BD1636A1B68EC
:10844000A0F50050B3F90810F9F7CEFDDFED5D7A25
:10845000B0EEC07AB4EEE77AF1EE10FAB0EE408AF0
:1084600051D429462046FFF771FC6069022173F060
:1084700043F876F005F8544B1B68C01A40F6B83341
:1084800098420CD9256B05F55970FFF787FB30B979
:108490000023C5F86433C5F86833C5F86C33206B26
:1084A0006EF088FF206B6FF051FF206B90EDDB0AC0
:1084B0006FF02AF8206B70F087F903AA02A94348ED
:1084C00001F03AFC6369029ADA636369039A9A637A
:1084D00096F80438656BD4E90612F3B91368B3F95A
:1084E000083000EE903A0B68B3F9083000EE103A0D
:1084F0002B68F8EEE00ADB6AB8EEC00AB0EE481A64
:108500002846984735E096F805380BB10721A9E7CA
:108510000321A7E79FED298AA7E709681268B1F947
:108520000810B2F9082008EE101A00EE902A032B6A
:10853000B8EEC88AF8EEE00A1FD1B6F92038DFEDB0
:10854000247ACDED010A01EE903AF8EEE11A2046C8
:1085500061EEA71ACDED001AFFF7B8FEDDED001AA7
:10856000DDED010AB0EE401A2846B0EE480A6CF084
:1085700079FC04B0BDEC028B70BD072B2A680DD1CD
:10858000B6F920389FED121A07EE903AF8EEE77A26
:10859000D36A27EE811AB0EE480AB1E72046CDED46
:1085A000000A166BFFF792FEDDED000AB0EE401AEE
:1085B0000121B0EE480A2846B047DAE70000000083
:1085C0001047002000000034C07E0020102700204B
:1085D0000000C842F0B52DED028B0446406990F8CA
:1085E000CB308DB0D3B9012172F086FF606B626829
:1085F0000368D2ED020A5B6E9FED800A0121984765
:10860000606B6DF0D1FD206B6FF0F0FF206B0DB053
:10861000BDEC028BBDE8F0406FF082BD78489FED65
:10862000778A90F8D41E11F0010500F5805640F0CD
:108630009180636A1B68A0F50050B3F90810F9F740
:10864000D3FCDFED707AB0EEC07AB4EEE77AF1EEEB
:1086500010FAF0EE408A76D429462046FFF776FBE2
:108660006069022172F048FF75F00AFF664B1B68D3
:10867000C01A40F6B83398420AD9644D2846FFF72D
:108680008DFA28B985ED028A85ED018A85ED008A8B
:10869000236B5E4893EDBF0A5D4D1DF00BFD012776
:1086A00009A92846CDED070A8DED081ACDED0A0A75
:1086B0008DED0B1A8DED060A8DED090A1DF01AFDE0
:1086C0002946524A206B009709AB8DED098A8DED42
:1086D0000A8A6EF0CBFDAB689FED480A4D4A206BCD
:1086E000059305A93B466FF08FFC059B206BAB60A3
:1086F0006FF02CFE206B70F067F809AA06A94648B7
:1087000001F01AFB6369069ADA636369099A9A634E
:1087100096F80438656BD4E90612F3B91368B3F917
:10872000083000EE903A0B68B3F9083000EE103ACA
:108730002B68F8EEE00ADB6AB8EEC00AB0EE681A01
:108740002846984735E096F805380BB1072184E7AD
:10875000032182E7F0EE488A82E709681268B1F9DE
:108760000810B2F9082008EE101A00EE902A032B28
:10877000B8EEC88AF8EEE00A1FD1B6F92038DFED6E
:10878000277ACDED030A01EE903AF8EEE11A204681
:1087900061EEA71ACDED021AFFF798FDDDED021A82
:1087A000DDED030AB0EE401A2846B0EE480A6CF040
:1087B00059FB0DB0BDEC028BF0BD072B2A680DD123
:1087C000B6F920389FED151A07EE903AF8EEE77AE1
:1087D000D36A27EE811AB0EE480AB1E72046CDED04
:1087E000020A166BFFF772FDDDED020AB0EE401AC9
:1087F0003946B0EE480A2846B047DAE700000000E4
:108800001047002000000034C07E0020E47E0020DD
:10881000D87E0020EC7E0020102700200000C842F7
:10882000044B196083ED010AC3ED020A83ED031ABC
:10883000704700BFF07E002038B5054675F020FE79
:10884000054C2061E86871F0A9FD07C804F1140324
:1088500083E8070038BD00BFF07E002037B5284C04
:1088600023680546002B3FD1E86871F097FDD4EDF1
:10887000017A9FED247AF0EEE76AF4EEC76AF1EE32
:1088800010FA06D4D0ED026AF4EEE67AF1EE10FAB0
:1088900031DCD4ED027AF0EEE76AF4EEC76AF1EE6D
:1088A00010FA06D490ED027AF4EEC77AF1EE10FADF
:1088B00021D4D4ED037AF5EEC07AF1EE10FA1DDD85
:1088C00011491DF075F868468DED000ACDED010ADD
:1088D0001DF03CF9D4ED037AF4EEC07AF1EE10FA13
:1088E0004CBF0120002007E075F0CAFD2369226813
:1088F000C31A9342B8D3012003B030BD0020FBE778
:10890000F07E002000000034047F0020024B002293
:108910005A619A61DA617047F07E002070B51E4E90
:108920002DED028B9FED1D8A06F5A04384B0002536
:108930000446F0EE480AA3F69C60B0EE481AF0EE4A
:10894000481AB0EE480A83F86D578DED018A8DED17
:10895000028A8DED038A71F06DF801A910488DED42
:10896000018A8DED028A8DED038A06F5405670F07E
:108970002DFC2A4601A90A4871F03CF929462046F7
:1089800086F80558FFF72EF901462046FFF7DEF975
:1089900004B0BDEC028B70BD102700200000000069
:1089A0007468002038B5054605480C4601F07EFF86
:1089B00000B91CB12846FFF7B1FF0124204638BD9D
:1089C00010270020F0B5064687B01F480D465DF021
:1089D0006DF8044640B945F0DDFE0522162145F04C
:1089E00091FC204607B0F0BD184F97F86D3713B1D2
:1089F0003046FFF793FF1648294670F081FF044682
:108A000018B945F0C7FE0222E8E7D5ED027A97F8DB
:108A10006D171048F8EEE76AD5ED037ACDED006AE0
:108A2000B8EEE77AD5ED017A8DED017A0023F8EE04
:108A3000E77A0393049305936A4603ABCDED027A7C
:108A4000FAF7B0FDCDE700BF1848002010770020EE
:108A50007468002010270020F0B589B00222064675
:108A600004A80D4609F066FE134804A95DF01EF83F
:108A7000044640B945F08EFE0522162145F042FC21
:108A8000204609B0F0BD0D4F97F86D3713B1304651
:108A9000FFF744FF29460022094871F0ABF8002394
:108AA00001930293039397F86D17064801AB2A468A
:108AB000FAF778FDE4E700BF18480020107700209F
:108AC00074680020102700202DE9F0432DED028B63
:108AD00089B00646174604A802220D46B0EE408A29
:108AE0009846F0EE608A09F025FE1D4804A95CF066
:108AF000DDFF044658B945F04DFE0522162145F02C
:108B000001FC204609B0BDEC028BBDE8F083DFF824
:108B1000609099F86D3713B13046FFF7FFFE9DF86E
:108B20004830F0EE680A4246B0EE480A3946304610
:108B3000FFF728F975F0A4FC0A4B294618600022BB
:108B4000094871F057F8002301930293039399F8B1
:108B50006D17064801AB2A46FAF724FDD1E700BF9E
:108B600018480020C07E00207468002010270020D4
:108B70001077002070B52DED028B0446406990F807
:108B8000CB3086B03BBB012172F0B6FC606B9FED31
:108B9000698A62680368D2ED020A5B6EB0EE480A29
:108BA00001219847606B6DF0FFFA63488DED038AF1
:108BB000F0EE480AB0EE481AF0EE481AB0EE480A55
:108BC0008DED048A8DED058A06B0BDEC028BBDE803
:108BD000704070F02FBF594890F8D41E11F0010575
:108BE00000F5805651D1636A1B68A0F50050B3F9B7
:108BF0000810F9F7F9F9DFED527AB0EEC07AB4EE69
:108C0000E77AF1EE10FAB0EE408A37D429462046D2
:108C1000FFF79CF80221606972F06EFC464870F024
:108C2000EFFD01464748FBF7F3FF02A9454803AAB9
:108C300000F0F6FF6369029ADA636369039A9A6344
:108C4000206B6FF0C1FD96F80438656BD4E906120D
:108C5000F3B91368B3F9083000EE903A0B68B3F932
:108C6000083000EE103A2B68F8EEE00ADB6AB8EE46
:108C7000C00AB0EE481A2846984735E096F80538FD
:108C80000BB10721C3E70321C1E79FED2A8AC1E7A2
:108C900009681268B1F90810B2F9082008EE101A34
:108CA00000EE902A032BB8EEC88AF8EEE00A1FD136
:108CB000B6F92038DFED247ACDED010A01EE903AC5
:108CC000F8EEE11A204661EEA71ACDED001AFFF783
:108CD000FDFADDED001ADDED010AB0EE401A28467E
:108CE000B0EE480A6CF0BEF806B0BDEC028B70BD69
:108CF000072B2A680DD1B6F920389FED131A07EE1D
:108D0000903AF8EEE77AD36A27EE811AB0EE480A75
:108D1000B1E72046CDED000A166BFFF7D7FADDED7F
:108D2000000AB0EE401A0121B0EE480A2846B047CA
:108D3000DAE700BF00000000746800201047002040
:108D400000000034102700200000C842084B93F8B0
:108D50006D37032B0BD8DFE803F002040608FFF79A
:108D600009BFFFF73FBBFFF735BCFEF751BF7047A8
:108D700010770020002070470120704701207047C5
:108D8000002070470048704750530C080048704757
:108D900058530C0808B5036B03480022C3F854234A
:108DA000FCF744FC012008BD1027002038B52C4DED
:108DB00095F8A73F04469BB905F6DC60012172F0E7
:108DC0009BFB606B62680368D2ED020A5B6E9FEDED
:108DD000250A01219847606BBDE838406DF0E4B981
:108DE000022105F6DC6072F087FBA369186851F078
:108DF00043FA05F56F6383ED000AE369186851F0E3
:108E00003BFA05F6F86383ED000A636A186851F0CF
:108E100033FA6268D2ED287A20EE270AB0EE0B7A98
:108E2000C0EE077A05F57063C3ED007A236A18680F
:108E300051F022FA05F6087383ED000AA36A186858
:108E400051F01AFA05F6147383ED000AE36A186804
:108E500051F012FA05F6187585ED000A38BD00BF0D
:108E600010470020000000000020704700207047DD
:108E7000012070470120704700487047A0530C083C
:108E800000487047AC530C08044A00231370044A8E
:108E90001370044B01201880704700BF107F002022
:108EA0001E7F00201C7F0020F0B50446406990F82A
:108EB000CB508BB0B5B9012172F01EFB6069294619
:108EC000EEB272F035FA28B1606940F2DC523146F8
:108ED00072F02CFF01350C2DF0D19E4B00221A7040
:108EE0000BB0F0BD9B4D2B78042BF9D8DFE813F0C5
:108EF0000500110040005E002201974B01241C80F8
:108F0000964B00221A7075F0BBFA954B2C701860C6
:108F1000E6E7002660693146F7B272F009FA28B137
:108F2000606940F2DC52394672F000FF01360C2EC7
:108F3000F0D121698A4C01F5457108461DF036F9DA
:108F4000DFED887AB4EEE70AF1EE10FA02DD75F093
:108F500097FA206075F094FA236803F5FA73984243
:108F6000BED902232B7075F08BFA7F4B1860B7E7E0
:108F700075F086FA7C4B1B6803F5FA73984212D29F
:108F8000754B60691A88754B02EB8202C2EB0212C4
:108F9000920002F2DC52197812B272F0C7FE002879
:108FA0009ED1042300E003232B7099E72369DFEDB2
:108FB0006F5AD3EDC57ADFED6E6A674F93EDC66ADF
:108FC00093EDC77AB7F90010644EF4EEE57AF1EE4E
:108FD00010FAF4EEE67ACCBF01220022F1EE10FA8C
:108FE0004CBF01230023D21AB4EEE56A4A43F1EEE6
:108FF00010FAB4EEE66A07EE902ACCBF01220022F6
:10900000F1EE10FA4CBF01230023D21AF8EEE77AF2
:109010004A43CDED017A07EE902AF8EEE77ACDEDDE
:10902000027AF6EE007AB4EEE77AFEEE007AF1EE1E
:1090300010FAB4EEE77ACCBF01230023F1EE10FA68
:109040004CBF012200229B1A4B4307EE903AF8EEE8
:10905000E77A3178CDED037A72F050F907A901A8CB
:109060008DED070ACDED080A8DED091A1CF0ACFF55
:10907000F8B12046FDF79EFC33783E4A01330621C5
:1090800048F094FC3178606901231944C9B22B700F
:1090900031703B8072F04CF900287FF421AF042638
:1090A00020462E70FDF786FC334A314648F07EFCA0
:1090B00016E701A81CF0C2FF317860698DED040A43
:1090C000CDED050A8DED061A72F018F907A904A86E
:1090D0008DED070ACDED080A8DED091A1CF074FF1D
:1090E00070B12046FDF766FC3378244A013306212F
:1090F00048F05CFC31786069012272F021F9C1E727
:109100002046FDF757FC1E4A062148F04FFCB7F9F0
:109110000030013309D12046FDF74CFC3378194A61
:109120000133042148F042FC3BE74FF6FF733B80DC
:10913000012339E7144B082293F8B51E2046FDF7AA
:1091400033FC1248012216210BB0BDE8F040F8F7BD
:10915000FBBA00BF1E7F00201C7F0020107F002074
:10916000147F00200AD7233C187F0020CDCCCC3EB2
:10917000CDCCCCBEB4530C084E540C08C7530C08CD
:10918000EB530C081C540C0810470020B85E00205C
:109190000020704700207047012070470120704771
:1091A00000487047B8540C0800487047C0540C0879
:1091B00070B52DED028B84B0044675F061F906465A
:1091C00060696E4D90F8CB3003BB012172F094F9C9
:1091D000606B62680368D2ED020A5B6E0121B6EE35
:1091E000000A9847606B6CF0DFFF206B6FF030F87F
:1091F000206BB6EE000A6FF075FA2369D3F80032DF
:10920000C5F8B43404B0BDEC028B70BD022172F01D
:1092100073F9E36A186851F02FF8A36A1868B0EE82
:10922000408A51F029F80023A5F5A040F0EE408ACD
:109230000093019301F03AFB00287CD09FED507A17
:10924000F0EEC87AF4EEC77AF1EE10FA06DCF0EE32
:10925000E87AF4EEC77AF1EE10FA02DD206B6EF0D8
:10926000F7FF484801AA694600F066FD206B6FF0E1
:109270006DF89DED010A636970EE288A9DED000A84
:10928000C3ED0E8A30EE088A636983ED0F8A636A44
:109290001868438A828907EE903A3B4BF8EEE77AEA
:1092A00093ED007A67EE877AFCEEE77A17EE903A54
:1092B00099B250F077FF01463248F8F795FE334BEC
:1092C0003048B3F95C3201EE103AE3691B68B3F938
:1092D000083000EE903AA3691B68B3F90830B0EE8D
:1092E000408A00EE103AB8EEC11AF8EEE00AB8EE85
:1092F000C00A03AA02A9F8F70DFEDFED257A606B1C
:10930000B0EEC87AB4EEE77AF1EE10FA17D403683B
:10931000DDED030ADB6A9DED020AB0EE481A9847BC
:109320002369D3F80032C5F8B434C5F8B8642046D0
:10933000FDF72EFD66E7206B6EF08AFF99E7D5F802
:10934000B83402689DED020ADDED030AFA33B34238
:1093500009D9D36A9FED0F1A98472369D3F80032D1
:10936000C5F8B434E3E705F2B44393ED001A136B88
:10937000B8EE411A01219847D9E700BF10770020C5
:10938000CDCCCC3D10270020FC5E002010470020F3
:109390000000003400000000F8B504462DED028BFB
:1093A0003E4801F083FA0646002873D03C4DDFEDBD
:1093B0003D8AD5ED630A9FED3C8A95ED5F0A206BEF
:1093C000F4EEE80AF1EE10FAB8BFF0EE480A6DF0DC
:1093D000CDFED5ED630A95ED5F0A206BF4EEE80A49
:1093E000F1EE10FAB8BFF0EE480A6DF037FFA5F5C0
:1093F0008040276BF8F792FE6368B3F93020B3F929
:109400002C3000EE903A434201EE102A00EE103A62
:10941000B8EEC11AF8EEE00AB8EEC00A38466DF0B0
:10942000EDFFA5F58040276BF8F778FE6368B3F988
:109430003020B3F92C3000EE903A434201EE102A6E
:1094400000EE103AB8EEC11AF8EEE00AB8EEC00A23
:1094500038466EF04DF8206B6EF0FAFE206B6FF020
:10946000C5F8606B62680368D2ED020A5B6E012189
:10947000B6EE000A9847606B6CF096FE206BB6EE75
:10948000000A6FF02FF9236905F58055D3F80032F3
:10949000C5F8B434BDEC028B3046F8BD102700206F
:1094A000106700200000003400007A43002070475D
:1094B0000120704701207047002070470048704726
:1094C00008550C080048704714550C08036B00221F
:1094D000C3F854230369D3F80022024B0120C3F8D8
:1094E000B42470471077002073B5044674F0C8FFA9
:1094F00006466069544D90F8CB30B3B9012171F044
:10950000FBFF606B62680368D2ED020A5B6E9FED41
:109510004F0A01219847606B6CF046FE2369D3F82F
:109520000032C5F8B43402B070BD022171F0E4FF1E
:10953000A5F5405301AAB3F95C3201EE103AE36994
:109540001B68B3F9083000EE903AA3691B68B3F9C1
:10955000083000EE103AB8EEC11AF8EEE00AB8EEA4
:10956000C00A6946A5F5A040F8F7D4FC636A1868FC
:10957000438A828907EE903AA5F5C05313ED057A28
:10958000F8EEE77A67EE877AFCEEE77A17EE903A24
:1095900099B250F007FE0146A5F5A040F8F724FD6A
:1095A000DFED2B7A606BB0EEC07AB4EEE77AF1EEC5
:1095B00010FAB0EE401A29D40368DDED010ADB6A27
:1095C0009DED000A98472369D3F80032C5F8B434FA
:1095D000C5F8B864656B2B685E6E236A186850F036
:1095E0004BFE63680021D3ED020A2846B047A36A08
:1095F0006569186850F040FE85ED0E0AE36A6569FA
:10960000186850F039FE85ED0F0A8CE7D5F8B834AC
:1096100002689DED000ADDED010AFA33B34209D973
:10962000D36A9FED0A1A98472369D3F80032C5F828
:10963000B434CFE705F2B44393ED001A136BB8EEE0
:10964000411A01219847C5E710770020000000006B
:10965000000000340120704700207047012070474F
:1096600001207047004870475C550C08004870475F
:1096700064550C0837B5436993F8CB200446D2B93A
:109680001A681846926A90476069012171F034FFA8
:10969000606B62680368D2ED020A5B6E9FED360A6A
:1096A00001219847606B6CF07FFD206B03B0BDE833
:1096B00030406EF09BBF314D95F9B03E002B03DA80
:1096C0001B220221FDF770F9B5F95C322C482D4DB3
:1096D00001EE103AE3691B68B3F9083000EE903AE6
:1096E000A3691B68B3F9083000EE103A01AAB8EE7E
:1096F000C11AF8EEE00A6946B8EEC00AF8F70AFCAB
:10970000636A1F481B68B3F90810F8F76DFC606BBB
:10971000DDED010A0368B0EE401ADB6A9DED000A38
:109720009847236B95ED600A93EDC31AF7EE000A94
:109730003320B0EEC00A1AF001F9FDEEC07AA5F5AB
:10974000805517EE903AA5F82432206B6DF0DCFEC0
:10975000206B6FF039F8A36A6569186850F08CFDCA
:1097600085ED0E0AE36A6569186850F085FD85EDA0
:109770000F0A03B030BD00BF0000000010470020FA
:10978000102700201067002070B504461D48F8F728
:1097900041F90546A0B31B48266BF8F7BFFC636888
:1097A000B3F93020B3F92C3000EE903A434201EE89
:1097B000102A00EE103AB8EEC11AF8EEE00AB8EE40
:1097C000C00A30466DF01AFE0E48266BF8F7A6FC6C
:1097D0006368B3F93020B3F92C3000EE903A43427D
:1097E00001EE102A00EE103A3046B8EEC11AF8EE3B
:1097F000E00AB8EEC00A6DF07BFE206B6EF0F6FE5C
:10980000284670BD1027002000487047AC550C0852
:1098100000487047B8550C0810B50446FCF7F6FD33
:10982000054B2360054BE363002384F8403000239D
:109830006364204610BD00BFE0560C08000080BFE6
:10984000034BC3639FED030A03486DF083BF00BF62
:10985000000080BF000000006064002037B50546AE
:10986000FDF734F9044660B12846FFF7E9FF1548D3
:1098700000F086FD054638B9134A1448062148F021
:1098800095F8204603B030BD1148124C70F08AFDA7
:10989000D4ED9C7AB4EEE70AF1EE10FA0FDB9FEDFF
:1098A0000E7A67EE877A17EE900AF6F72DFE0B4ACE
:1098B000CDE90001042104F6884048F077F82C46F1
:1098C000DFE700BF10270020C0550C089853002088
:1098D000405F0020104700200AD7233CE2550C08C7
:1098E00030B5364C2DED028B94F8B43E152B83B079
:1098F0000546B0EE408A06D0314A042104F688407D
:1099000048F054F819E02F4870F04CFDD4ED9C7AE3
:10991000B4EEE70AF1EE10FA14DB9FED2B7A67EE56
:10992000877A17EE900AF6F7EFFD284ACDE9000195
:10993000042104F6884048F039F82846FFF780FFF4
:10994000002034E0B4F9CC3A07EE903AF8EEE77A2A
:10995000F4EEC87AF1EE10FA01DD1D4ACDE7B4F954
:10996000CE3A07EE903AF8EEE77AF4EEC87AF1EEE6
:1099700010FA20D4DFED147A85ED0F8A68EE277A8D
:1099800017EE900AF6F7C0FD124ACDE90001062154
:1099900004F6884048F00AF80A4870F003FDD5ED57
:1099A0000F7A0D4830EE670A6DF0D4FE012003B047
:1099B000BDEC028B30BD094A9FE700BF1047002075
:1099C00008560C08405F00200AD7233C2F560C088D
:1099D00061560C088B560C0860640020AD560C08CC
:1099E00038B504462DED028B1C4800F0C9FC90B33D
:1099F000D4ED0F7A1A4DF5EEC07A05F6D823F1EEC4
:109A000010FA93ED008A0FDC05F6D42393ED000ADB
:109A1000D5ED9C7AB4EEE70AF1EE10FA04D530EEFB
:109A2000480A2046FFF75CFFD4ED0F7AF5EEC07AC6
:109A3000F1EE10FA0FDD78EE277A95ED9C7A094B5E
:109A4000F4EEC77AF1EE10FAA4BF77EE677A38EE3B
:109A5000278A83ED3D8ABDEC028B38BD102700209C
:109A6000104700201067002030B52DED028B036AEF
:109A70001B68B3F9083000EE103A83B00446B8EE24
:109A8000C00A4848F8F75CFB46488DED010AF8F734
:109A900045FB63689DED010AB3F92C3001EE103AE5
:109AA000434200EE903AB8EEC11AF8EEE00A6B209D
:109AB00019F044FFDFED3C7AB0EEC07AB4EEE77AFD
:109AC000F1EE10FAB0EE408A58D594F8403083B1E8
:109AD000E068D4ED0F8A70F065FCD4ED117A38EEB1
:109AE000800A204630EE670AFFF7FAFE002384F86A
:109AF00040302E4B93F8B02E93F9B03E002B22DA73
:109B00006268236BD2ED2D7A93EDD57AF1EE046A7B
:109B100077EEE67AF4EE477AF1EE10FAC8BFF0EE8F
:109B2000477AC3EDD57A2046FFF78AFE206BB0EE68
:109B3000480A6DF0E9FC206B03B0BDEC028BBDE878
:109B400030406EF041BE530614D5E068256B70F0CE
:109B500029FC236BF2EE047A30EE270AD3EDD57A96
:109B6000B4EE670AF1EE10FAC8BFF0EE407AC5ED28
:109B7000D57AD8E72046FFF733FFD7E7D4ED0F7A41
:109B8000F5EEC07AF1EE10FAD0DD94F84030002BFB
:109B9000CCD1E06870F006FC012384ED110A84F852
:109BA0004030C3E710270020CDCC4C3D10470020AB
:109BB00010B50446FCF7D4FF2046FFF755FF2046BA
:109BC000BDE81040FDF7D2B838B5044604F5A0450D
:109BD00074F056FCD5F8C43403F5FA7398421BD9D7
:109BE00004F5325004F500540C4A0621083047F0C1
:109BF000DDFE94F8B03E6FF3C30384F8B03E6AF024
:109C000081FC036801229B680321984774F038FCAB
:109C1000C5F8C004002038BD0120FCE718570C0827
:109C200070B52DED028B00F5804300F50054D3F89C
:109C30007431D3EDCF7AD3EDD08AFDEEE77A1546B5
:109C4000B4F95C2217EE903A0E46F1EE688A514262
:109C5000FDEEE88A09B218B219F0AEFEB4F95C2242
:109C600018EE903A514208EE100A09B218B219F0F3
:109C7000A3FEB4F95C3207EE903AB8EEC88AF8EE6B
:109C8000E77A88EE277ABDEC028B07EE900A86ED24
:109C9000007AB4F95C32B8EEE77A07EE903AF8EE63
:109CA000E77AC7EE276AC5ED006A70BD70B52DED85
:109CB000028B00F5804300F50054D3F8843AD3EDCD
:109CC000CF7AD3EDD08AFDEEE77A1546B4F95C225F
:109CD00017EE903A0E46F1EE688A5142FDEEE88AA0
:109CE00009B218B219F068FEB4F95C2218EE903A85
:109CF000514208EE100A09B218B219F05DFEB4F92B
:109D00005C3207EE903AB8EEC88AF8EEE77A88EE51
:109D1000277ABDEC028B07EE900A86ED007AB4F943
:109D20005C32B8EEE77A07EE903AF8EEE77AC7EEE3
:109D3000276AC5ED006A70BD70B52DED028B00F588
:109D40007553D3EDD37AD3EDD48A00F50054FDEEEC
:109D5000E77A1546B4F95C2217EE903A0E46F1EE1A
:109D6000688A5142FDEEE88A09B218B219F024FE61
:109D7000B4F95C2218EE903A514208EE100A09B28A
:109D800018B219F019FEB4F95C3207EE903AB8EE49
:109D9000C88AF8EEE77A88EE277ABDEC028B07EEE8
:109DA000900A86ED007AB4F95C32B8EEE77A07EEF5
:109DB000903AF8EEE77AC7EE276AC5ED006A70BD03
:109DC00000F53B501C3070F027BC000070B5044615
:109DD00074F056FB04F5A043D3F8C02402F51C53DD
:109DE000103383420AD94AB1164A04F5325002218F
:109DF000083047F0DBFD0025284670BD124B1B687C
:109E0000D86A0368DB699847012801D10F4AECE75B
:109E100004F5005696F8A75F3DB904F532500C4A98
:109E20000421083047F0C2FDE6E704F53B501C3042
:109E300070F0F2FB96F8B03E43F0080386F8B03EAF
:109E4000DAE700BF30570C08082700205D570C08E0
:109E500092570C0884B070B52DED048B84B0044685
:109E60000DA880E80E0074F00BFB04F5A04304F588
:109E70000055C3F8C40495F8B03E1B071DD44A4EE4
:109E800074F0FEFA336803F5FA6398420DD9204660
:109E9000FFF79CFF88B904F53250444A042108308A
:109EA00047F084FD74F0ECFA3060002004B0BDECA3
:109EB000048BBDE8704004B07047129802280CD0A3
:109EC000F6F700FBCDE9000104F53254384A0834B6
:109ED0000421204647F06AFDE7E79DED0E0A9DED5F
:109EE0000D8A8DED030AF0EE000ADDED0F8A19F000
:109EF00023FC9DED030A50B110EE100AF6F704FBA7
:109F000004F53254CDE900012A4A0834E0E7F7EEBF
:109F1000000A8DED030A19F00FFC9DED030AA8B1AC
:109F2000FDEEE88AFCEEC87A18EE903ACDED037AA1
:109F300004F53B509DF80C101AB21C3004B0BDEC77
:109F4000048BBDE8704004B071F0F0BEDFED1A0A7A
:109F500019F0F2FB0028A8D09FED189ADFED160A41
:109F60008120B0EE491AB0EE680A19F0E7FCC0EEA5
:109F7000096AD5F8942AB2F90A30B2F90E20D21A39
:109F800007EE902AB8EEE77A07EE903AF8EEE77A15
:109F9000E6EE877ABCEEC87AFDEEE77A8DED037ABD
:109FA00017EE903AC4E700BF207F0020B4570C089A
:109FB000D6570C08EA570C08000000000000C84201
:109FC00038B500F50053044693F8B42E142A1DD07A
:109FD00093F8B02E120703D5BDE83840FFF7F4BD63
:109FE000012283F8A82F51F0D1FD054651F064FD00
:109FF00051F0F8FC51F0EEF804F53B501C3072F0D3
:10A0000041FE2846BDE8384051F05EBD38BD000035
:10A0100010B504460020FBF77FF904F50054C4F89E
:10A02000900A0120FBF778F9C4F88C0A0220FBF7AC
:10A0300073F9C4F8940A0320FBF76EF9C4F8980A80
:10A040000420FBF769F9C4F89C0A0520FBF764F9C2
:10A0500041F29411C4F8A00AD4F88C0A50F076F8B2
:10A06000D4F8900A41F2941150F070F8D4F8980A9C
:10A0700041F2941150F06AF8D4F8940A4FF47A71CE
:10A0800050F060F8D4F89C0A41F2941150F05EF858
:10A09000D4F8A00A41F2941150F058F8D4F88C0A80
:10A0A0001E2150F057F8D4F8900A1E2150F052F8B3
:10A0B000D4F8940A1E2150F04DF8D4F8980A2821BB
:10A0C00050F048F8D4F89C0A1E2150F043F8D4F818
:10A0D000A00A1E2150F03EF80024E0B2002240F217
:10A0E000DC5101344FF034FF062CF6D1204600221B
:10A0F00040F2DC514FF02CFF002240F2DC510720EF
:10A100004FF026FF0820FBF707F90022B0F90A10EC
:10A1100008204FF01DFF0920FBF7FEF80022B0F9E0
:10A120000A1009204FF014FFBDE81040002240F251
:10A130004C410A204FF00CBF37B5044604F50055DA
:10A1400000F53B501C30B5F8A212019071F0C2FA34
:10A1500095F818130198002271F0A8FAD5F8943AEE
:10A160000198B3F90A10B3F90E2072F0B1FD01980D
:10A1700072F0B0FB04F55E5001212830F7F7D4F9F6
:10A1800010B12046FFF71CFE03B0BDE8304051F08F
:10A1900083B9000013B5044600F58C60019005F00A
:10A1A00041FA94F871340198242202FB0303D3EDA1
:10A1B0000B7AF5EEC07AF1EE10FA02DD05F0F6F951
:10A1C000019804F5005494F8B13EDB0709D594F8E2
:10A1D000D91E05F0DBF994F8D83E60F3000384F84B
:10A1E000D83E02B010BD000037B5102300F554650D
:10A1F0000446C0F8EC3F192128463CF0CBF904F5A1
:10A200002B504FF07A5301A91C30019304F50054F0
:10A2100047F00CF8192128463BF07AFD94F8C83A2B
:10A2200060F3000384F8C83A03B030BDF0B52DEDFB
:10A23000028B00F5546683B0054630463BF022FEA3
:10A24000192130463BF08AFD1921074630463BF084
:10A2500055FD042805F5005473D0002094F8C83A41
:10A2600060F3410384F8C83A192130463BF066FD9B
:10A27000A4F8CA0A05F56050303070F093F804F67F
:10A28000D42383ED000A192130463BF07DFD1921CE
:10A29000A4F8CC0A30463BF06DFD94F8C83AA4F817
:10A2A000CE0A9B0728D574F0EBF8D4F8D03A0646CE
:10A2B000F31AB3F57A7FB4F9CA3A07EE903A05F586
:10A2C0002B50F8EEE77A00F11C004BD901A9CDED37
:10A2D000017A46F01BFF2848C4F8D06A03460830CC
:10A2E00093ED008A46F010FFD0ED007A78EE677AA1
:10A2F00004F6D823C3ED007A94F8C83A04F6D824BB
:10A3000005F58040226800F62424C3F30006C3F359
:10A31000400113F0010380F81E6A80F8201A2260C1
:10A3200004D090F91F3A003B18BF012380F8C93AC6
:10A3300080F8CA1A00F67820426503B0BDEC028BA3
:10A34000F0BD192130463BF03BFD022885D97A1C2F
:10A3500006D094F96C32BB42CCBF002001207DE7CF
:10A3600001207BE7054BCDED007A01AA69460193F8
:10A3700046F060FFAFE700BFE4510020CDCC4C3D7C
:10A3800010B5044674F07CF804F5005393F8C82A1D
:10A3900012F001010BD0C2F34001920707D5D3F8A8
:10A3A000D03AC01AB0F57A7F2CBF002101210846AF
:10A3B00010BD000008B500F5005090F8B03EB1EBBC
:10A3C000D31F13D061F3C713094A80F8B03E0021B0
:10A3D0001B06116006D544F0DDF9A321BDE8084055
:10A3E00043F070BF44F0D6F9A421F7E708BD00BFE1
:10A3F000287F002008B500F5005090F8B03EC3F368
:10A4000080128A4213D061F38613094A80F8B03E65
:10A4100000215B06116006D544F0BCF9A521BDE81A
:10A42000084043F04FBF44F0B5F9A621F7E708BD57
:10A43000247F002070B500F5005586B095F8A71F61
:10A44000044649B90191FFF7B5FF0199204606B0CE
:10A45000BDE87040FFF7CEBF00F59250002303A97E
:10A46000103003930493059302F0F0FDDDED057ABF
:10A470009FED3F7AF4EEC77AF1EE10FA49DD9FEDD9
:10A480003D7AF4EEC77AF1EE10FA4CBF01260026B1
:10A4900095F8B13EDA0746D595F8D83EDB0742D5A8
:10A4A00094F8712495EDC56ADFED336A04F58C6389
:10A4B000242101FB023393ED0B7A95F9B03E002B7A
:10A4C000C6EE267A27DADFED2B6A77EEE67AF4EE2F
:10A4D000C77AF1EE10FA4CBF012100212046FFF7A8
:10A4E00069FF95F8E33E002B3FD0002E3DD0234A74
:10A4F000136807EE903AB8EE677ADFED217AB4EE92
:10A50000E77AF1EE10FA1FD401212046FFF772FF1F
:10A5100021E00026BCE7B4EEE77AF1EE10FACCBFFA
:10A5200001210021DAE7E6B195F8E43EABB1154A26
:10A53000136807EE903AB8EE677ADFED117AB4EE61
:10A54000E77AF1EE10FA02D50133136003E001213E
:10A550002046FFF72FFF06B070BD95F8E33E002BB5
:10A56000C5D100212046FFF725FF0021CDE700BF20
:10A57000CDCC4CBDCDCC4C3D0000C842247F00204A
:10A580000000C843287F0020F9F73CB80148FAF7DB
:10A590005BBB00BF1027002038B500F59255103581
:10A5A0000446284601F008FC04F58053042283F891
:10A5B0006424002283F85925B4F9A43004F6C800B5
:10A5C0001BB9B4F8A230A4F8A430B4F8A41018F061
:10A5D00021FD2846BDE8384001F0E8BC2DE9FF41E7
:10A5E000044600F5905036F07BFA04F5485004F527
:10A5F0008C66343005F0D4FC304605F04BFBB7EEEA
:10A60000000A7D483AF084FC94F8FD347B4800EE63
:10A61000103AB8EE400A3AF07BFC04F532500830AC
:10A620004BF0FAFB4FF04AFD9922292150F012FD20
:10A630004FF044FD4FF0EAFC2046FFF7E9FC2046CE
:10A64000FFF77AFD2046FAF777FF04F58E500C30BD
:10A6500056F012FB6A4B6B491B68986A03684FF40B
:10A660007A72DB6A98470423C4F8A43104F5907029
:10A6700010F04EF808F030FE4FF40053036308F07A
:10A680002BFE09F0EFFE04F50053802504F5315050
:10A69000C3F888504FF40061043037F075FC04F5BE
:10A6A00096405030019004F5804852F041FD9FEDF6
:10A6B000561A98F8C91B0198F0EE410AB0EE410A0B
:10A6C000002252F0D9F8032298F8C91B019852F0E1
:10A6D000BFF804F59540503006F0C6FE0021304624
:10A6E000C4F8745405F0AAF8304604F09BFF94F8BF
:10A6F00070C404F58057002304F2744024225FFAEA
:10A7000083F8C44520D903FB02215D1C415C01296B
:10A710006CD104F5005502A904F2FC408DF8083014
:10A720003AF0E0FE95F8B13E85F8D98E43F001038A
:10A7300085F8B13E4146304604F028FF95F8D83EF2
:10A7400060F3000385F8D83E04F5005504F59256F1
:10A7500095F8B13E13F0010306F110060DF108085B
:10A7600046D1414604F2FC408DF808303AF0BAFE7A
:10A77000B2EE040A304602F005FC04F52A502430FB
:10A780006FF050FE04F5A043D7F85024C3F8B4246A
:10A790002046FFF729FD04F52B50283051F090FB9F
:10A7A00004F52D500C301DF031FD4FF48073C5F8C9
:10A7B000403C164B0293164B039398E8060004F5B1
:10A7C0007F6042F0C7FF2046FFF7E6FE2046FAF71B
:10A7D00021F94FF40023C4F8E03B95F8B03E43F074
:10A7E000100385F8B03E04B0BDE8F0812B4686E743
:10A7F0009FED080ABEE700BF04580C0811580C086A
:10A80000082700208DA50108000000001027002067
:10A8100089A50108CDCCCC3D13B5044600F5925076
:10A82000103001F0DBFC90B104F56050303004F5DD
:10A8300000546FF0A9FD94F8A72F0190C3B2C0F3A4
:10A84000001032B918B99DF80500C0F3400002B0FD
:10A8500010BD0028FBD083F08000C009F7E700009E
:10A8600037B5044600F59250103001F0B7FC88B1BE
:10A8700004F5005595F9490C60B104F5605030308D
:10A880006FF082FD95F8A73F01902BB99DF8050068
:10A8900000F0010003B030BD9DF804301A07C3F387
:10A8A000C00044BF83F08000C009F3E710B500F595
:10A8B0000053044693F8D43E5B0707D4FFF7ACFF80
:10A8C00028B92046BDE81040FFF7CABF002010BDE0
:10A8D00037B500F57F65044604F50054284601911C
:10A8E00043F080F894F8B03E019960F341032846A4
:10A8F00084F8B03E03B0BDE8304043F071BD0000C5
:10A90000002070470020704737B500F5974568353F
:10A910000446284641F018FB012201A9284641F0CF
:10A9200093FA20B104F55464019BC4F89C3203B03F
:10A9300030BD000010B504210446FFF7C9FF30B157
:10A9400004F597406830BDE8104041F04BBB10BDA6
:10A9500000F5A253D3ED077A9FED237AF5EEC07A86
:10A96000F1EE10FA03F11C0304DBF4EEC77AF1EE0A
:10A9700010FA17D4F4EEC77AF1EE10FA14DC9FED5A
:10A980001B7AF4EEC77AF1EE10FA4CBF02230323D0
:10A9900000F5405090F8E827032A0ED8DFE802F0CF
:10A9A00006161B1F0023F3E70123F1E7012B07D154
:10A9B000D0F8E4270132C0F8E42780F8E837704780
:10A9C000032BFAD1D0F8E427013AF4E7022BEFD0B9
:10A9D000002BF7D0F1E7032BEAD0012BF1E7002B96
:10A9E000E6D0022BEDE700BFDB0FC93FDB0FC9BF8D
:10A9F00013B50446143000F0C1FD04F12C0000F042
:10AA0000BDFD04F1740075F06FFB04F1F40075F006
:10AA10006BFB4FF0FF331549C4F85031204639F035
:10AA2000CFFE00230DF1070104F128008DF8073057
:10AA30003AF02AFD01230DF1070104F129008DF8F8
:10AA400007303AF021FD0F230DF1070104F1250035
:10AA50008DF807303AF018FD054B1A6812B1054819
:10AA600073F0DCFC20461C6002B010BDCC590C0811
:10AA70002C7F00201C580C082DE9F0478CB003A94E
:10AA800038F0D0FF60B300210D2208A807AF1C4C9E
:10AA9000DFF87080DFF8709007910B26A1F01EF9A7
:10AAA0000697237ADFF864A08DF81430002554F857
:10AAB00025300493D8F80000E368B5B90093C06A64
:10AAC00053461122394615F075FC0021B7EE000AF5
:10AAD00003A839F0ABF935B1013E04F11004E0D11F
:10AAE0000CB0BDE8F0870125E1E701930223009354
:10AAF00011224B463946C06A15F05CFCE5E700BF01
:10AB00006C5A0C080827002079580C0870580C085B
:10AB10002DE9F04F2DED028BD0F8543183B004466F
:10AB200093BB9FED7E8ADFF800A2074600F1740810
:10AB300000F5AA750126721ED2B297ED070A01929E
:10AB4000404675F0F1FAFB69C8F83C304FF07E538F
:10AB5000C8F8483097F92830019A013B5FFA86FB24
:10AB60000E2B22D8DFE803F015414D5A636C7D218E
:10AB70008B959FAA21C5B500D4F8543103B9636100
:10AB8000D4F8583103B9E36203B0BDEC028BBDE8E1
:10AB9000F08F4820019207F027FE814618B1019AF4
:10ABA000214674F09DF9C5F80090286898B10368B3
:10ABB0009B689847002840F0AA804DF0ABFD584AAA
:10ABC0003346032146F0F2FE286810B103685B6843
:10ABD000984700232B60022E07F1180708F1800820
:10ABE00005F10405C8D00226A5E72820019207F048
:10ABF000FBFD81460028D6D0019A214675F05CFA0B
:10AC0000D1E76820019207F0EFFD81460028CAD005
:10AC1000FF23019A214674F005FCC4E768200192E5
:10AC200007F0E2FD81460028BDD00023F1E768204F
:10AC3000019207F0D9FD81460028B4D00123E8E74E
:10AC40004420019207F0D0FD81460028ABD0019A44
:10AC5000214673F093FDC9F800A00023C9F84030E5
:10AC6000A1E74820019207F0BFFD814600289AD055
:10AC7000B1EE040A019A214673F01EFE93E74820C4
:10AC8000019207F0B1FD814600288CD0B2EE040A93
:10AC9000F0E74820019207F0A7FD8146002882D006
:10ACA000B3EE040AE6E74820019207F09DFD8146D5
:10ACB00000283FF478AFB3EE0E0ADBE7482001929C
:10ACC00007F092FD814600283FF46DAFB0EE480AD0
:10ACD000D0E74420019207F087FD814600283FF429
:10ACE00062AF019A214673F049FD0E4BC9F800305E
:10ACF000B3E73420019207F077FD814600283FF446
:10AD000052AF019A0023214674F066FE4BE72B6890
:10AD1000002B3FF460AF84F84FB15CE70000704255
:10AD200056580C0848AA0D08CCAC0D0813B50446BB
:10AD3000FFF7A2FE204638F0CBFF68B994F928301F
:10AD400013B994F940303BB101230DF107012046BE
:10AD50008DF807303AF0C6FB94F90030002B08DD7F
:10AD600094F928302BB1204602B0BDE81040FFF71F
:10AD7000CFBE02B010BD00000346406C012807D0D2
:10AD8000032805D0986C012802D0032818BF0220A0
:10AD90007047000070B590F90030002B04460D4656
:10ADA00011DD0B78012B0ED8D0F8540110B10368D7
:10ADB000DB699847D4F8580128B103682946DB6954
:10ADC000BDE87040184770BD90F90030002B0ADDD7
:10ADD000012908D8182303FB010090F92800003846
:10ADE00018BF0120704700207047000037B50446A7
:10ADF000FFF7EAFF9FED0B0A0D4680B104EB8103DC
:10AE00008DED010AD3F8540138B1036801A9DB685C
:10AE1000984704EBC51484F865009DED010A03B062
:10AE200030BD00BF0000000070B50446FFF7CCFF46
:10AE300050B104EB8104D4F8540128B10368BDE893
:10AE400070401B6911461847002070BD2DE9F04F76
:10AE50002DED028B90F90030002B83B00646894619
:10AE600053DD2C4B1B68D86A03685B68984704461F
:10AE700050B14DF04FFC284A062103B0BDEC028BC7
:10AE8000BDE8F04F46F092BD9FED248ADFF890A018
:10AE9000DFF890B0354606F14407B046214630460B
:10AEA000FFF792FF20B195F8643043B188ED068A30
:10AEB0008035043708F118083CBB0124EEE7B9F1EE
:10AEC000000F03D098F92630002BF1D1D7F81021CC
:10AED000631C01933AB94DF01DFC019B5A460321B6
:10AEE00046F064FDE4E773F0CBFA0022A5F8702089
:10AEF000A5F872200122A86685ED1B8A3A604DF004
:10AF000009FC019B52460621EAE703B0BDEC028B27
:10AF1000BDE8F08F0827002084580C0800000000CE
:10AF2000C2580C089B580C082DE9F0432DED028BFC
:10AF300085B004460D46B0EE408AFFF745FF98B352
:10AF400004EBC119CF01D9F868306BB373F098FAEC
:10AF5000D9F86830C01AB0F57A7F03D3B9F87230E7
:10AF60000F2B0CD8E31993F86520002A40F08C8051
:10AF70003C44B4F872300133A4F8723014E0B9F8EC
:10AF8000703005F1010805F1100693B94DF0C2FBD0
:10AF900004EB86064346454A042146F007FD032399
:10AFA00073603C440023A36605B0BDEC028BBDE892
:10AFB000F08307EE903AD9ED1B6AD4F85C21F8EEE5
:10AFC000E77A86EEA77A8DED037ACAB394F9023058
:10AFD000002B35DD07EE903AB2F90C209FED345A84
:10AFE000F8EEE75AF7EE007AE5EE857A182101FBD4
:10AFF000054506EE902AF8EEE66A95ED066A67EEDC
:10B00000A67A37EE467A67EEA77AB0EEC77AE6EE12
:10B01000E67AF6EE006A67EEA67AF4EEC77AF1EE0B
:10B0200010FA0DD5B0EEC66AB5EEC06AF1EE10FAB0
:10B0300006DD4DF06FFB1F4A4346042146F0B6FC87
:10B04000182003A900FB084004EB86063AF0E0F95B
:10B05000022373606368DB060ED54DF05BFB05468B
:10B060000398F5F751FA144ACDE900014346062149
:10B07000284646F09BFC94E74DF04CFB0F4A4346B4
:10B08000062146F093FC8CE7B3F87220052A7FF680
:10B090006FAFD3ED1B7AB3F8702037EE880A013218
:10B0A00083ED1B0AA3F8702062E700BFE4580C0888
:10B0B0000AD7233CFA580C0827590C084E590C089B
:10B0C00010B590F90030002B02460C461CDD90F8BC
:10B0D0004D31CBB9FFF778FEA8B1182101FB04224E
:10B0E00092F9243093B1022B0DD1462050F06CF927
:10B0F000DFED077AB0EEC00AB4EEE70AF1EE10FA1F
:10B100004CBF0120002010BD0020FCE71846FAE7E4
:10B11000000000342DE9F8432DED028B04460E4665
:10B12000FFF752FEE8B104EB81090DB2D9F85431B2
:10B13000BBB173F0A5F904EBC6174FEAC618386621
:10B14000D9F8540103685B69984770B1D9F8540184
:10B15000036839469B69503198473B6D87F8650015
:10B16000FB64BDEC028BBDE8F8833146204697F8BE
:10B170006590FFF73BFE182303FB064393ED068A19
:10B18000BB6E30EE488A87ED178A1BB131462046E8
:10B19000FFF7CAFEB9F1000F43D0DFED447A9FED0F
:10B1A000447A04EB080368EE277AD3ED166AE6EEDC
:10B1B000877A182104EB080701FB0646C7ED167ACB
:10B1C00096F9273083B3012B53D1DFED3A8AF1EEA4
:10B1D000487A05EB4505B4EEE88AC7ED157A04EB2D
:10B1E000C505F1EE10FA95ED070A58BFF0EE687A42
:10B1F00027EE800A9EF0C2FC87ED130A97ED160A2F
:10B20000B4EEE80AF1EE10FA48BFF1EE408A95ED8F
:10B21000070A28EE800A9EF0B1FC444484ED140A2B
:10B220009FE7F0EE487AC4E7B5EEC08A05EB450526
:10B23000F1EE10FA87ED158A04EBC505D8BF9FED36
:10B240001D8A95ED070A28EE000A9EF097FC04EB94
:10B250000803D3ED167A83ED130AF5EEC07AF1EE0A
:10B2600010FAD8BFDFED137A95ED070A27EE800AB2
:10B27000D1E7B0EEC88A05EB450587ED158A04EBEA
:10B28000C50494ED070A28EE000A9EF077FCD7ED7E
:10B29000167A87ED130A94ED070AF0EEE77A27EEA7
:10B2A000800A9EF06BFC87ED140A5AE79A99993E42
:10B2B0003333333F0000000038B50A460446FFF739
:10B2C00083FD10B304EBC113CD0193F8653033B1A6
:10B2D00004EB8103D3F85431003B18BF012318213C
:10B2E00001FB0242D2ED067AF0EEE77AF5EEC07A83
:10B2F000F1EE10FA08DC2C4494F8640020B992F9BD
:10B300002600003818BF0120184038BD10B50021B4
:10B310000446FFF759FD18B12046FFF7CDFF50B1A5
:10B3200001212046FFF750FD30B12046FFF7C4FF52
:10B33000003818BF012010BD0846FCE710B50246D2
:10B34000FFF742FD20B102EBC11292ED140A10BDCD
:10B35000BFEE000AFBE7000010B50246FFF734FD20
:10B3600020B102EBC11292ED130A10BDBFEE000A2C
:10B37000FBE7000010B50246FFF726FD20B102EB07
:10B38000C11292ED150A10BD9FED010AFBE700BF47
:10B390000000000010B50246FFF716FD20B102EBD9
:10B3A000C11292ED170A10BD9FED010AFBE700BF25
:10B3B000000000002DE9F04F2DED028B8DB004460A
:10B3C00073F066F89FED3C8ADFED3C8A8046894643
:10B3D000274625464FF0000B04F5AA7A5FFA8BF654
:10B3E00031462046FFF7F0FC002858D05AF82B30A1
:10B3F000002B54D06A462046FFF716FD08B9CDED64
:10B40000008A1D22002104A8A0F068FCA3238DF867
:10B410000430952331468DF80530204672238DF88F
:10B420000630CDF80780CDF80B908DF80F60FFF750
:10B4300093FF20468DED040AFFF79CFFDDED007AB7
:10B440008DED050A67EE887A2046FDEEE77A17EE65
:10B45000903AADF81830FFF79DFF10EE103A2046F5
:10B46000CDF81A30BB69CDF81E30FFF729FE314602
:10B470008DF822002046FFF71FFFD5F8BC30099356
:10B48000D5F8C0300A9394F84E318DF823008DF82A
:10B490002C3043F07FF9292201A942F083F91837B3
:10B4A0008035BBF1000F04D00DB0BDEC028BBDE8C0
:10B4B000F08F4FF0010B91E70000C8420000000040
:10B4C000F8B590F90030002B04464DDD0021FFF760
:10B4D00021FE01212046FFF71DFE94F90030002BCC
:10B4E0000DDD94F9403053B14DF014F901210546BA
:10B4F0002046FFF723FF1D49284646F0E3FC667807
:10B5000094F84E7131462046FFF7D6FE054668B9DD
:10B5100001462046FFF7D0FE28B901212046FFF75B
:10B52000CBFE28B1012584F84E5101E084F84E612C
:10B53000204673F075FC94F84E31BB4204D043F0C2
:10B5400029F95A2142F0BEFED4F8503101330BD014
:10B5500043F020F9D4F8501142F042FF20B12046C8
:10B56000BDE8F840FFF726BFF8BD00BF68590C08DA
:10B57000014B1868704700BF2C7F002010B50349AD
:10B58000044639F01DF9204610BD00BF1C5B0C08B5
:10B59000F0B52DED048B91B004466D46284606F0BB
:10B5A000D5FD94F8BC33002B72D004F57A730FCB21
:10B5B00085E80F0094F8F833D4EDEC8A94EDED8A29
:10B5C00094EDEE9A002B63D094F8D033002B5FD02B
:10B5D0002D22002104A8D4F8C073D4F8C463D4F891
:10B5E000C853D4F8CC43A0F079FBA3238DF81030D6
:10B5F00095238DF8113046238DF8123072F048FFF4
:10B600009FED250A9FED257ACDF8171068EE807A18
:10B61000CDF8130067EE877AFDEEE77A17EE903AE1
:10B6200068EE007A29EE000A67EE877AADF81B30E3
:10B63000FDEEE77A20EE070A17EE903AADF81D30DE
:10B6400018F012F9DDED017A9FED157ACDF82D7025
:10B65000BCEEC00AF8EEE77A10EE103A67EE877A91
:10B66000ADF81F3017EE903ACDF82130029BCDF89F
:10B670002530039BCDF82930CDF83160CDF8355019
:10B68000CDF8394043F086F82D2204A942F08AF81B
:10B6900011B0BDEC048BF0BDE02E65420000C84245
:10B6A0000AD7233C30B52DED028B8BB00446242203
:10B6B0000D4601A80021A0F011FBA3238DF8043052
:10B6C00095238DF8053048239FED1F8A8DF80630AD
:10B6D00072F0DEFED4ED817A2B68CDF80F3067EE84
:10B6E000887A95ED020ACDF80B1017EE903AD4ED5A
:10B6F000827ACDF8133067EE887A6B68CDF8173010
:10B7000017EE903ACDF80700CDF81B3018F082F80C
:10B7100010EE103A94ED830ACDF81F3020EE080A9F
:10B7200018F078F810EE103ACDF8233094F80C3376
:10B730008DF8273043F02EF8242201A942F032F888
:10B740000BB0BDEC028B30BDE02E654230B587B04A
:10B7500014460D46182200216846A0F0BFFAA32324
:10B760008DF8003095238DF8013049238DF8023093
:10B7700072F08EFEA3680393E36804936368CDF8C8
:10B7800007100593CDF803008DF80B5043F002F835
:10B790001822694642F006F807B030BD10B58EB0E9
:10B7A000044602A806F0D2FC02A9204601F0FEFBE6
:10B7B000002845D001F04CFE694601F085FA1F22B1
:10B7C000002106A8A0F08AFAA3238DF8183095234B
:10B7D0008DF819304A238DF81A3072F059FEDDEDDC
:10B7E000037A9FED1B7A049BCDF82330F8EEE77ABD
:10B7F000059BCDF8273067EE877ACDF81B0017EE52
:10B80000903ADDED007ACDF82B30F1EE677A17EE45
:10B81000903ACDF81F10204601A9CDF82F3000F046
:10B8200047FD78B1DDED017AF1EE677A17EE903AD7
:10B83000CDF8333042F0AEFF1F2206A941F0B2FF2F
:10B840000EB010BD42F0A6FFDFED027AEEE700BFBA
:10B850000AD7233C5241C07F7047000010B5044610
:10B8600006F0CAFF204610BD0023036043608360DA
:10B87000C360036143618361C36103627047000079
:10B880002DE9F041076A07F54876044600F16C059A
:10B890000FCE0FC50FCE0FC533682B6007F545736C
:10B8A00093E8070004F1900888E8070094ED2E7AE9
:10B8B000D4ED2D7A77EE877A9FED367AF0EEE77A3F
:10B8C000F4EEC77AF1EE10FA8EB004F16C0718D4DA
:10B8D00004F14802394604A804AD18F039FB0FCD35
:10B8E0003E460FC60FCD0FC62B683360414604F1AC
:10B8F000240018F0AFFA84ED240AC4ED250A84ED83
:10B90000261A04F10C0304F10802211D384618F030
:10B91000CDFC9FED216AD4ED037A94ED017ADFED41
:10B920001F6A206A67EE867A27EE067A67EEA67AA5
:10B9300027EE267AFDEEE77ABDEEC77A17EE903A4B
:10B9400084ED047A94ED027A002BB8BF03F50C4322
:10B9500027EE067AB8BFA03327EE267AA36104F15A
:10B96000B003039304F1AC03BDEEC77A029304F174
:10B97000A803019304F1A403009384ED057A04F174
:10B98000A00304F19C02394601F022FE0EB0BDE88E
:10B99000F08100BF00000034E02E65420000C84284
:10B9A00010B504468AB0006A01F0A0FD04A904F1B4
:10B9B00024008DED040ACDED050A8DED061A18F070
:10B9C00049FA0AB010BD000030B58BB001460446FC
:10B9D0006D46684618F02CFB0FCD0FC40FCD0FC479
:10B9E0002B6823600BB030BDF8B50446244B0360D0
:10B9F00000F124050162027704F148072846FFF7A9
:10BA000033FF3846FFF730FF04F16C00FFF72CFFDF
:10BA1000217F00231829C4F89030C4F89430C4F86A
:10BA2000983026D0192926D039BBC4F8B430D4EDCB
:10BA30002D7A84ED2E0A30EE270A17F0EBFE9FEDEB
:10BA4000111ADFED110A284660EE200AB0EE410A15
:10BA500018F0CCFB0FCD3E460FC60FCD0FC62B689E
:10BA600033603846FFF7B0FF2046FFF709FF204656
:10BA7000F8BD064BD9E7064BD7E7064872F0CEFC77
:10BA8000005C0C080000000035FA8E3C0000B44257
:10BA900000008743DC5B0C08002303604360836085
:10BAA000C360036143618361C36103627047000047
:10BAB00090F8F432B02202FB030390F8382393F895
:10BAC000D13012B1012B28BF012318467047000066
:10BAD0002DE9F04F04468BB04FF0000A0D461EF0E2
:10BAE0005FFC84F814A204F506704FF07E5771F0E5
:10BAF000F3FB4FF47A73A4F8623284F86852C4F806
:10BB00004872C4F84C72C4F8507204F51B700025DA
:10BB100006F01CFB04F52B790323C4F8803204F5EE
:10BB20003476C4F89452C4F89852C4F89C52C4F8BD
:10BB3000A052C4F8A452C4F8A8524846FFF7ACFF7C
:10BB400004F5487B3046FFF7A7FFC4F81453C4F848
:10BB50001853C4F81C535846FFF79EFFC4F84453CB
:10BB6000C4F84853C4F84C53C4F85053C4F8545361
:10BB7000C4F85853C4F85C53C4F86053C4F8645311
:10BB8000C4F86853C4F86C53C4F87053C4F88C53A9
:10BB9000C4F89053C4F89453C4F8A853C4F8A453F9
:10BBA000C4F8A053C4F8B053C4F8B453C4F8B8539D
:10BBB000C4F8CC53C4F8C853C4F8C453C4F89C7335
:10BBC000C4F8C07304F5757006F0C0FA04F57A7015
:10BBD00006F0BCFA04F58063C4F8FC531D6004F55C
:10BBE000816304F583601D605D609D6006F0AEFAC0
:10BBF00004F22C4304F264481D605D609D606B4B51
:10BC0000C4F83C3404F50D73C4F8403404F50E73E5
:10BC1000C4F8443404F50F73C4F8483404F51073C1
:10BC2000C4F84C3404F24523C4F8503404F51173BD
:10BC3000C4F8543404F58B6340461D605D609D601C
:10BC4000FFF72AFF04F59160FFF726FF04F59763DD
:10BC500004F23C421D605D609D6004F2C44304F246
:10BC6000A4501D605D609D6004F59A631D605D6079
:10BC70009D6004F2DC431D605D609D6004F2EC4356
:10BC80001D605D609D6004F2FC431D605D609D6011
:10BC900004F5A463C2F8D470C2F8D8701D605D606A
:10BCA0009D6004F22C531D605D609D6004F5A963E6
:10BCB0001F605D6004F26C531D605D609D6004F563
:10BCC000AF631D605D609D6004F5B2631D605D60E3
:10BCD0009D6006F03BFA04F2B45324221D605D60BF
:10BCE00004F2BC5351461D605D6004F2C4534046EB
:10BCF0001D605D609FF0F2FF04F2E450C8F8207010
:10BD0000C8F81070C8F80070FFF7C6FE04F5C163EC
:10BD100004F5C7601D605D609D6004F214631D60E2
:10BD20005D609D6004F5C4631D605D609D6004F20C
:10BD30002C631D605D609D6006F008FA1C4B1D4978
:10BD40001C60204638F03CFD94F8683243F0010353
:10BD500084F868325146242258469FF0BFFFC4F849
:10BD60004073C4F83073C4F8207304F5257207CA11
:10BD700004F5287383E80700484694EDAA1AD4ED29
:10BD8000A90A94EDA80A18F031FA354649466846E2
:10BD90006E4618F04DF90FCE0FC50FCE0FC53368A4
:10BDA0002B6020460BB0BDE8F08F00BF545E0C083E
:10BDB000307F0020105D0C0810B5044688B001F0FB
:10BDC000E5FB94F93232012B02D1274804F00CFE36
:10BDD000022B0AD1032384F8323204A9012304F18F
:10BDE00011008DF8103039F03FFB94F8323284F8AE
:10BDF000903204F23C4001F06BFB94F93132642B39
:10BE000030D1652304A904F231208DF8103039F0C7
:10BE100069FB04A9204637F03DFE18B304238DF8D2
:10BE200018300023CDE9013303930F2305936946AE
:10BE300004A837F0AFFF059B28B108AA02EB8302E4
:10BE4000009942F8581C0133112B0593EFD967F084
:10BE5000D3F89DED031ADDED020A9DED010A65217F
:10BE600067F088F808B010BD085C0C0870B500F5E4
:10BE7000257600F528758CB00446314628461AF020
:10BE8000A3F8E0B996E8070085E8070004F52B71F0
:10BE900094EDAA1AD4EDA90A94EDA80A01910846D6
:10BEA00018F0A4F902AD019902A818F0C1F80FCD5D
:10BEB00004F534740FC40FCD0FC42B6823600CB08D
:10BEC00070BD000013B540F2411200F50671044642
:10BED00001A814F091F804F23C4001F0F5FC204672
:10BEE0001EF0B6FC01A814F0A9F802B010BD0000C5
:10BEF000F8B50B68C0F804324B68C0F808328B689C
:10BF0000C0F80C3201F10C0607460C4600F54875E6
:10BF10000FCE0FC50FCE0FC533682B6004F1300272
:10BF200007CA07F5457383E8070004F13C0207CA16
:10BF300007F5517383E8070004F1480207CA07F5C3
:10BF4000547383E80700543494E8070007F55773E7
:10BF500083E80700384601F02DFC3846BDE8F8407C
:10BF600001F010BC13B5044600F23C40019003F010
:10BF70008BF804F5BB610198009102F0D9FB0099A0
:10BF8000204602B0BDE81040FFF7B2BF4A78064B2A
:10BF9000C2F340121A754A78C2F380125A750A78B1
:10BFA000C2F300129A757047BD7F002013B540F2AE
:10BFB000F522044600F5067101A814F01DF80021D1
:10BFC00004F23C4001F0D0FE94F8603223B12046E8
:10BFD0001EF086FE84F8600201A814F02FF802B06B
:10BFE00010BD000038B590F80C3305460C462BB157
:10BFF000032B0BD095F86832DB070CD405F5C7632B
:10C000000FCB84E80F0095F8480603E01EF096FC7D
:10C010000028EFD038BD0020FCE7000000F23C40D3
:10C0200090ED350A7047000000F23C4090ED360A72
:10C030007047000010B490F80C230C462AB1032A74
:10C040000AD000205DF8044B704700F5B26007C8C5
:10C0500084E807000120F5E75DF8044B1EF02CBCD6
:10C0600090F88403431E58425841704738B590F801
:10C070000C330D468BB900F23C4001F097FC0446AE
:10C0800010B90024204638BD01F0E4FBD5ED007A5C
:10C0900027EE800A85ED000AF4E7D0EDE07AC1EDE5
:10C0A000007A90F87C43002CEBD090EDDE7ADFED47
:10C0B000086AB4EEE67AF1EE10FAF7EE006AB8BF5D
:10C0C000B0EE667A67EE877AC1ED007ADAE700BFF4
:10C0D0000000003490F80C33032B01D11EF066BB36
:10C0E0000020704710B490F80C43032C03D15DF886
:10C0F000044B1EF067BB00205DF8044B7047000046
:10C1000090F80C23032A01D11EF0CEBC00F23C4073
:10C1100002F08CB830B590F80C3385B004460D466B
:10C120008BB1032B18D004F5257019F087FF284632
:10C1300001A98DED010ACDED020A8DED031A19F06A
:10C140003BFB012006E000F23C4001F0D9FB002857
:10C15000E9D1002005B030BD90F86032002BF8D056
:10C160001EF08AFCDFE700007FB590F80C2332B1A7
:10C17000032A4FF0000309D0039304930CE000F26C
:10C180003C4007B05DF804EB01F072BC03A90393D7
:10C19000049305931EF000FB9DED030ADDED040AF8
:10C1A00007B05DF804FB000007B590F80C3333B11D
:10C1B00000F57F7003B05DF804EB19F0C7BC00F226
:10C1C0003C4001F055FC68468DED000ACDED010ABA
:10C1D00019F0BCFC03B05DF804FB000090F80C0300
:10C1E000003818BF0120704708B590F80C23032AC7
:10C1F00005D0BDE8084000F23C4001F021BC1EF033
:10C20000CBFA012008BD000010B590F80C230C46B5
:10C210001AB1032A07D0002010BDBDE8104000F27B
:10C220003C4001F0D5BB1EF0DDFA012084ED000A90
:10C23000F2E7000090F80C33032B01D11EF0DCBBB9
:10C240000020704730B590F80C3385B005460C4699
:10C2500023B1032B09D0002005B030BD00F23C40D3
:10C2600005B0BDE8304002F093BA002302A9029362
:10C2700003931EF079FA0028EDD001A928461EF09C
:10C280007FFA0028E7D0029B2360039B6360019B39
:10C29000A360E1E790F80C231AB1032A05D000202F
:10C2A000704700F23C4002F0A7BA1EF05DBA0000F1
:10C2B00090F80C231AB1032A05D00020704700F231
:10C2C0003C4002F08BBA1EF05BBA000090F93232AB
:10C2D0003BB990F8683213F0010F14BF032000201F
:10C2E0007047032070470000F7B50446FFF7EEFFE4
:10C2F0000546002862D0032839D194F860326BB328
:10C3000094F86832D8072BD501A920461EF012FEFA
:10C31000BDF80430002B18BF002594F8146206F015
:10C32000FD06012E4AD10023032D019307D101A957
:10C3300020461EF00BFE20461EF0CEFB064604F201
:10C340003C4002F0D7FA08B994F809039DF804308C
:10C35000D90703D55A0701D59F0632D400252DE011
:10C3600020461EF071F9002808BF0025D5E70025FA
:10C37000D3E713F0020F2EE094F9443223B99DF86D
:10C380000430DB092FD0E9E7002EF8D00FF008FDCC
:10C39000FFF78EFB022807D99DF805309806DDD5FA
:10C3A0009DF80430D906D9D5FB6A93F89C30002B50
:10C3B000E5D118E0DA0601D41B0718D5284603B0EA
:10C3C000F0BD0028FAD094F80923B4F94C36002ABD
:10C3D000CFD013F0010FF1D1154B1F68FB6A93F812
:10C3E0009C30002BC8D19DF804309C07E2D406F0A5
:10C3F00073FF06F06FFE0028B0D10FF0D1FCFFF7FD
:10C4000057FB0228AAD90FF0CBFC90F8F432B022E7
:10C4100002FB030090ED3B7AF0EE007AB4EEE77A8F
:10C42000F1EE10FA9AD59DF80530DB09C6D195E7F3
:10C43000082700202DE9F04790F8603292B00446BA
:10C44000002B00F0948020461EF040FF2046FFF7AE
:10C450004BFF03287BD104F548780027414620464E
:10C460000097019702971EF0DDFA694620461EF0FC
:10C47000CFFA009BC4F80432019BC4F80832029B37
:10C48000C4F80C32204601F095F9204601F07AF903
:10C4900016F04EFD054620461EF058F90028A8BFAC
:10C4A000C6B203AA4FF0FF312046BCBF95F81293E5
:10C4B00095F813630397A8BFB146049705971EF03C
:10C4C0009FF903A819F0BAFD4FF00C0A0AFB0950B6
:10C4D00084EDD10AC4EDD20A84EDD31A04F551716A
:10C4E00000F5117019F0BAFD04F557770AFB0655EF
:10C4F00084EDC50AC4EDC60A84EDC71A3A464FF06A
:10C50000FF31204605F5C4751EF08EF995E8070049
:10C5100006AE86E807003946304619F005FE04F5F8
:10C520002B72414609A817F013FD314609A817F0F0
:10C5300091FC09A9204684EDD40AC4EDD50A84ED06
:10C54000D61A1EF003FD09A92046FFF71FFD94F837
:10C550004E36002B3AD109A805F0F8FD09A920466E
:10C560001EF0F8F990B3012384F84E362EE0D0F88F
:10C5700064321BB971F084FFC4F86402154B1B6868
:10C58000D86A03685B68984788B171F079FFD4F87E
:10C590006432C01AB4F86232984204D920461EF0C0
:10C5A0009FFB84F8600294F860327BB14BE771F036
:10C5B00067FFD4F86432C01A41F287339842E4D856
:10C5C00042F0E8F841F028FF0028DED112B0BDE8C3
:10C5D000F08700BF0827002090F80C3323B1032B0D
:10C5E0004FF0000007D0704790F93222032A04D19F
:10C5F0000A70012070470870FBE71846704700007A
:10C6000073B50D460DF107010446FFF7E5FF064639
:10C6100028B19DF807302BB1032B09D000263046F6
:10C6200002B070BD04F5C7630FCB85E80F00F6E7D5
:10C63000294620461EF082F994F86062EFE7000078
:10C640007FB50E460DF103010446FFF7C5FF054611
:10C6500018B90025284604B070BD9DF8033083B199
:10C66000032B16D004F5257019F0E8FC01A930461B
:10C670008DED010ACDED020A8DED031A19F09CF83B
:10C68000E8E7314604F23C4001F03AF90028E9D1EC
:10C69000DFE794F86032002BDBD0314620461EF0F5
:10C6A000EBF9DFE737B50D460DF107010446FFF75B
:10C6B00093FF28B19DF8073023B1032B0FD0002042
:10C6C00003B030BD04F5BB631B682B6004F2DC5380
:10C6D00004F5BC641B686B602368AB60F0E7204620
:10C6E00029461EF095F994F86002E9E710B5044672
:10C6F000FFF7ECFD18B1032807D0002010BD04F2AD
:10C700003C40BDE8104001F025B994F86032002BA0
:10C71000F3D020461DF098FF0028EED094F8143294
:10C7200003F0FD03012BE9D194F80C03C31E58421A
:10C730005841E3E710B50446FFF7C8FD80B1032870
:10C7400010D194F8600250B171F09AFED4F86432BE
:10C75000C01A44F62063984294BF0020012010BD07
:10C760000120FCE70020FAE708B50246FFF7AEFD1E
:10C77000032804D110461EF0E9FB012008BD00206B
:10C78000FCE7000030B585B004460191FEF7F0FEED
:10C790000199054610B9002005B030BD0191FEF7A2
:10C7A0008FFC01990028F6D02846FEF785FD002869
:10C7B000F1D0B4F84C365907EED494F80933002B75
:10C7C000EAD00B4A1268D26A92F89C506DB103A964
:10C7D0002046FFF7C9FF30B19DF80E309A07DBD530
:10C7E000C3F38000D8E72846D6E71846D4E700BF51
:10C7F000082700201EF07EB91EF0B2B910B490F8E0
:10C800000C4324B1032C08D05DF8044B70475DF84D
:10C81000044B00F23C4001F069B85DF8044B1EF097
:10C8200031B8000090F80C33F5EE007A002BB7EE2B
:10C83000000A08BFB0EE670A7047000010B5044652
:10C84000FFF744FD032804D12046BDE810401EF048
:10C850004BB8002010BD00002DE9F04190F80C33DA
:10C860008CB00027032B06460C461546009701970F
:10C87000029719D11DF06AFF6A4680464FF0FF31DA
:10C8800030461DF0D1FFB8F1FF3FA7606760276019
:10C890000DD116F04DFB2B4690F81313224615F0E0
:10C8A000D5FB0CB0BDE8F0814FF0FF38EBE716F098
:10C8B0003FFB2B4622465FFA88F115F0C7FB95ED4A
:10C8C000000A684619F0F6FB03A920468DED051A0B
:10C8D0008DED030ACDED040A19F026FC06F52B7246
:10C8E00006F5487103A817F033FB214603A817F09B
:10C8F000B1FA84ED021A84ED000AC4ED010A95ED47
:10C90000007ADFED037AA7EE271A84ED021AC8E752
:10C910000AE81C411FB5DFED0B7A20EE270A0C4612
:10C920001946094BCDE90042BDEEC00A18688DEDED
:10C93000020A064B9DF81820C06A13F03BFD04B0B4
:10C9400010BD00BFE02E6542082700201C5C0C08CB
:10C950002DE9F0472DED028B92B0002504460F46DD
:10C960004FF07E5A00F5487106A89046CDF818A001
:10C9700009950895079518F025FB06F0ADFC06F023
:10C98000A9FB81462046FFF7A1FC032803D094F8B9
:10C990000C33032B4FD19FED558ADFED558A0026CE
:10C9A0002379F2B2934247D90AAA71B22046CDF850
:10C9B00028A00D950C950B951EF03EF80AA906A827
:10C9C00018F06CFFB4EEC80AF1EE10FA0DDD494A1A
:10C9D000CDF800803B4648492046FFF79BFF0020EA
:10C9E00012B0BDEC028BBDE8F0870AA906A803953A
:10C9F0000495059518F03CFF03A90EA88DED0E0ACD
:10CA0000CDED0F0A8DED101ACDED111A18F060FC66
:10CA1000B9F1000F0DD09DED050AB0EEC00AB4EEDD
:10CA2000E80AF1EE10FA04DD344ACDF800803B4606
:10CA3000D1E70136B4E7002394F8686216F00100EC
:10CA400001D0012BCCD104F2E4510AA8CDF828A0E2
:10CA50000D950C950B9518F0B5FA0AA906A818F0D3
:10CA60001DFFDFED227AB4EEE70AF1EE10FA05DDE4
:10CA7000204ACDF800803B462149ADE72046FFF72C
:10CA800025FC03282DD120461EF01AF894F86832B0
:10CA9000DB0728D438BB0AA906A803950495059599
:10CAA00018F0E6FE03A90EA88DED0E0ACDED0F0AD3
:10CAB0008DED101ACDED111A18F00AFCB9F1000F26
:10CAC00011D09DED050ADFED0A7AB0EEC00AB4EE92
:10CAD000E70AF1EE10FA06DD084ACDF800803B4681
:10CAE000CAE70020D2E701207AE700BFC2B8323E91
:10CAF000C2B8B23E485C0C08535C0C086F970D0836
:10CB0000585C0C082DE9F743144605468846019306
:10CB1000FFF7ECFD019A074638B92448244B00681A
:10CB20002146C06A13F046FC019A0192214628462C
:10CB3000FFF70EFF064630B32846FFF7C7FB95F810
:10CB40000C33019A83420DD006F0C6FB06F0C2FA00
:10CB5000019A38B1174B154800682146C06A13F096
:10CB600029FC10E02846FFF7B1FB18B103280FD0CD
:10CB7000114BF0E713464146224605F23C4000F0D7
:10CB8000FDFE00B107B90026304603B0BDE8F083D2
:10CB900095F86092B9F1000F01D1084BDBE713461D
:10CBA0004146224628461DF05FFDEAE7082700209F
:10CBB0005C5C0C08685C0C08985C0C08875C0C08D2
:10CBC00090F80C33032B01D11EF0D6B9002070472A
:10CBD00090F80C33032B01D11EF00EBA00207047E1
:10CBE00090F80C33032B01D11EF04ABA0020704795
:10CBF00008B50246FFF76AFB10B1032806D008BD4E
:10CC0000BDE8084002F23C4000F06EBEBDE80840BE
:10CC100010461EF0A7B900000B4610B411462BB108
:10CC2000032B09D000205DF8044B70475DF8044BDE
:10CC300000F23C4000F06EBE5DF8044B1DF08ABE71
:10CC400013B50446FFF742FB0A460146204601920F
:10CC5000FFF7E2FF70B9084B019A1B68DB6A93F893
:10CC60009C0038B194F80C13204602B0BDE8104087
:10CC7000FFF7D2BF02B010BD0827002037B5044629
:10CC80000D4640F2B25200F5067101A813F0B4F956
:10CC9000294620461DF07CFE94F80C33032B0546F4
:10CCA00010D148B104F583612046FFF7C9FF84F82D
:10CCB0002804204600F0AEFD01A813F0BFF9284675
:10CCC00003B030BD0025F7E770B590F87C32DB0784
:10CCD00086B004460D460CD402F0FCFE437C2422B0
:10CCE00002FB0300D0ED0B7AF1EE677AC5ED007A16
:10CCF0003BE002A805F02AFA01A92046FFF7D8FA7E
:10CD0000E8B90FF04DF894F94432022B0646E3D10E
:10CD1000FEF7CEFE0228DFD996F8F4029FED147AD2
:10CD2000B02303FB0066D4F87032D6F8E0209B1ADB
:10CD300007EE903AF8EEE77A67EE877AD6E702A92F
:10CD40002046FFF77DFF0028DBD0D4F87022039B3C
:10CD5000DFED076A9DED017A9B1A07EE903AF8EE37
:10CD6000E77AA7EEE67A85ED007A06B070BD00BFDF
:10CD70000AD7233CF0B50C4687B000F5067106468D
:10CD800040F6863201A813F037F9A36853B9E36877
:10CD900043B9636833B9002701A813F04FF9384647
:10CDA00007B0F0BD204605F0D9FA0028F3D094E88A
:10CDB0000F0002AD85E80F000021284605F090FA2B
:10CDC00007460028E7D096F87C32DB0704D441F010
:10CDD000E1FC192141F076FA95E80F0006F51B7C7D
:10CDE0008CE80F0096F87C3243F0010386F87C3221
:10CDF000304600F00FFD4BF08DFC46214CF0A8FAB8
:10CE00004BF088FC45214CF0A3FA054BA2681B6847
:10CE1000DB6A1A61E2685A6162689A61BCE700BF26
:10CE20000827002038B5144B1B68DD6A2B680446C0
:10CE30005B6828469847F0B12B690BB96A69D2B193
:10CE4000C4F874326B69C4F87832A969002204F519
:10CE50001B7005F081F994F87C3223F0030343F052
:10CE6000030384F87C324BF055FCBDE83840034A9C
:10CE7000062144F09BBD38BD08270020AC5C0C089F
:10CE800010B588B004460593FFF720FA0328059BE8
:10CE90004FF000000AD10690079006A802900B9868
:10CEA00001900A98009020461DF0F0FD08B010BDDA
:10CEB00038B50446FEF75CFB0546D0B194F80C3358
:10CEC000032B03D095F84E41204638BD20461DF077
:10CED000FFFCFF280446F5D001462846FEF7ECF992
:10CEE0000028EFD021462846FEF7EAF80028E9D0CE
:10CEF000EAE70446E8E7000008B590F80C33032B96
:10CF000005D016F015F890F91203C0B208BD1DF057
:10CF10001DFC431CF9D1F4E708B590F80C3383B13C
:10CF2000032B03D1BDE808401DF008BC3FF050FEC4
:10CF300040F6ED424FF480113FF002FE4FF0FF301B
:10CF400008BD1846FCE7000090F80C33032B01D114
:10CF50001EF008BB7047000090F80C33032B01D182
:10CF60001DF0D0BA704700001DF056BB10B5044646
:10CF700020F084FB2046FEF70BFB2046BDE8104066
:10CF8000FEF70CBC07B5203001A98DED010A38F081
:10CF90003FFA03B05DF804FB90F80C330BB1032BA0
:10CFA00001D11EF05BBB00207047000030B500F5DA
:10CFB000757304460D460FCB85E80F0094F8E40323
:10CFC00030BD00007FB5054668460E4605F0BEF848
:10CFD00095F87C32DB0703D40024204604B070BDF2
:10CFE00069462846FFF7E2FF04460028F4D0694668
:10CFF00005F51B7005F0C2FA86ED000AC6ED010AC0
:10D00000EBE70000D0F880330B6090F87C037047AA
:10D01000D0F888330B6090F88503704730B500F581
:10D02000677304460D460FCB85E80F0094F8AC03F8
:10D0300030BD000030B500F5836304460D460FCBCC
:10D0400085E80F0094F8280430BD000010B500F208
:10D050002C4203460C4607CA84E8070093F83804BC
:10D0600010BD00002DE9F0432DED028B8BB005467D
:10D070000E461746FFF71CFF014680462846FFF77D
:10D0800081FB0446002848D0FEF772FA4146FEF7BD
:10D0900055F986ED000A95F93032002B3ADD0EF095
:10D0A0007FFEFEF705FD012834D90EF079FE90F8D9
:10D0B000F432D5EDDE7ADFED5D8A96ED000AB0221E
:10D0C00002FB030095F93032D0ED3B0A07EE103A2F
:10D0D000F4EEE87AB8EEC77AF1EE10FAB7EE008A0D
:10D0E000B8BFF0EE487A37EE201A20EE270A70EE2D
:10D0F000C70A40F2B63016F021FCD5EDDE7AF4EE28
:10D10000E87AF1EE10FAB8BFF0EE487A80EE277AAE
:10D1100086ED007A01233B7003E095F8083333B9BC
:10D12000387020460BB0BDEC028BBDE8F08395F85B
:10D130000C334FF00009CDF80490CDF80890CDF8ED
:10D140000C9043B1032B10D0CDF81090CDF8149073
:10D15000CDF818907CB902233B703246414605F267
:10D160003C4001F08BFB0446DBE701A928461DF09B
:10D17000A3FB0446E8E795F80C33002BEBD004A999
:10D180002846FFF763FF04460028E4D001A904A85D
:10D1900018F07AFF07A8CDED080A8DED091A8DED7C
:10D1A000070A19F085FB04A8B0EE408A19F080FB4D
:10D1B00095F93032002B30DD07EE903AF8EEE77A41
:10D1C0004FF47F7070EE670A37EE801AF5EEC00AF2
:10D1D000F1EE10FA48BFDFED160AF4EE410AF1EE67
:10D1E00010FAB0EE480AC8BFB0EE601A16F0A6FBFF
:10D1F000B0EE408AD5EDDE7A9FED0C7AF4EEC77A78
:10D20000F1EE10FAB7EE007AB8BFF0EE477A88EE8A
:10D21000277A032386ED007A7DE7B5EEC08AF1EE2A
:10D2200010FA48BF9FED028AE4E700BF0000003417
:10D230000000000010B50446FFF75EFE84F80D0301
:10D240002046FFF759FE84F80E032046FFF754FEF0
:10D2500084F80F032046FFF75FFE04F55A7184F847
:10D2600010032046FEF7E6FE84F8740300F0F2FA9D
:10D2700004F5617284EDDE0A04F560712046FFF763
:10D28000F1FE04F5627184F87C032046FEF7EEFEA1
:10D2900004F5637184F885032046FEF71BFF04F54F
:10D2A000677184F898032046FEF734FF04F56C712B
:10D2B00084F8AC032046FFF7F5F904F5707184F8A3
:10D2C000BC032046FFF7BCF904F5757184F8D00360
:10D2D0002046FEF787FE04F57A7184F8E4032046C1
:10D2E000FFF78EF984F8F8032046FEF73DFF04F5BA
:10D2F000806384EDFF0A2046C3ED000AFEF754FF69
:10D3000004F2044383ED000A04F2144204F581613F
:10D310002046FFF7A1FA04F583612046FFF790FC51
:10D3200004F22C4184F828042046FEF75DFF84F8BF
:10D33000380410BD37B50D46044600F027F91DB975
:10D3400015F0F6FD14F0B2FD4FF4BE7204F506714F
:10D3500001A812F051FE94F869322BB92046FFF76C
:10D3600061FD012384F86932224B1D68A86A0368B5
:10D370009B6998472046FEF779FD2046FEF7F2FDAF
:10D38000204600F079FA2046FFF754F8286B30B1B8
:10D390000368D4EDD20ADB6894EDD10A9847D4F83B
:10D3A000100208B1FEF76CFA204600F091F8204612
:10D3B000FEF79AFF94F8903284F80C0383420ED063
:10D3C00084F8900298B10C4D0C4B032808BF1D4601
:10D3D0004BF0A0F90A4A2B46062144F0E7FA204612
:10D3E000FFF728FF01A812F029FE03B030BD054D5C
:10D3F000EEE700BF08270020A71A0C08535C0C08B2
:10D40000C45C0C08585C0C08D0EDDE7A9FED057A00
:10D41000F4EEC77AF1EE10FAB7EE000AA8BFB0EE4C
:10D42000670A704700000034D0EDDE7A9FED077A7E
:10D43000F4EEC77AB7EE000AF1EE10FAB8BFF0EEDC
:10D44000407A67EEA77A80EE270A70470000003422
:10D45000014B1868704700BF307F00204FF0FF304D
:10D46000704700000120704770470000002070479F
:10D470000020704770470000704700000020704790
:10D480000020704700207047002070470020704740
:10D490000020704700207047012070470368D3F8D0
:10D4A00094301847002070470020704700207047D4
:10D4B0000020704700207047002070470020704710
:10D4C0000020704700207047002070477047000020
:10D4D0007047000008B515F02BFD90F8130308BD48
:10D4E00008B515F025FD90F8120308BD30B585B0DC
:10D4F00090F80E53044615F01BFD0C2303FB0500AA
:10D5000004F5517100F5117005B0BDE8304018F018
:10D51000A5BD000030B52DED028B9FED1A1ADFED91
:10D520001A0A91ED000A87B005462D200C468DEDB4
:10D53000011ACDED000A16F001FA9DED011ADDED9C
:10D54000000AF0EE408A2E2094ED010A16F0F6F95A
:10D550009DED011ADDED000AB0EE408A2F2094ED1A
:10D56000020A16F0EBF903A905F52570CDED038A43
:10D570008DED048A8DED050A38F098F807B0BDEC02
:10D58000028B30BDC2B8323EC2B832BE10B50446BE
:10D5900070F076FFD4F8F4321BB1C21AB2F57A7F7C
:10D5A00012D30A4A1268D26A92F89C2002B15BB97F
:10D5B000C4F8F40294F8314215F0BAFC80F80D4337
:10D5C00005F08AFE80F8254010BD00BF0827002026
:10D5D0002DE9F0432DED028B91ED007AD1ED037A28
:10D5E00087B08DED047AB0EEC77AB5EEC07AF1EE71
:10D5F00010FADDE91087DDF84C90CDED057A0C4688
:10D6000015461E4606DCF0EEE77AF5EEC07AF1EE3E
:10D6100010FA02DD04A818F017FB6B20B7EE001A11
:10D62000FFEE000A9DED050A16F088F96C2089EDE1
:10D63000000AB7EE001AFFEE000A9DED040A16F08C
:10D640007DF904A888ED000A18F05AFAB7EE008AAE
:10D65000002852D00023C9F8003088ED008AD4EDAC
:10D66000067A67EEA77AF4EEC87AF1EE10FA4ADB92
:10D670000023336085ED008ADFED3F0A96ED000A56
:10D680007C20B7EE001A16F059F986ED000A95EDE8
:10D69000000A7D20B7EE001AFFEE000A16F04EF9E0
:10D6A00085ED000AD4ED067A129BDFED346AF1EEC7
:10D6B000677AC3ED007A96ED007AF0EEC77AF4EE61
:10D6C000E67AF1EE10FA2BD503AB02AA01A92046A7
:10D6D00016F0ECFD9DED018AB0EE480A9BF0E2FEEB
:10D6E00085ED000AB0EE480A9CF032F887ED000A9A
:10D6F00007B0BDEC028BBDE8F08304A818F0ECF98C
:10D700000028A7D1ABE738EE670A16F049F886ED96
:10D71000000A94ED087AC7EE007AC5ED007AABE70F
:10D7200094ED076AC6EE077AC7ED007A96ED007AA7
:10D73000B0EEC77AB4EEE67AF1EE10FAC4D495ED05
:10D74000007ADFED0F6AB0EEC76AB4EE666AF1EEFA
:10D7500010FAB9DCB4EE477AF1EE10FAB4D6B0EEB6
:10D76000E77AB4EE667AF1EE10FAADDCF4EE677AA1
:10D77000F1EE10FABCD7A7E700000000000000346B
:10D78000FFFF7F7F1FB500F51773039300F5167336
:10D79000029300F51573019300F51473009300F5DF
:10D7A000127200F5137300F54871FFF711FF05B011
:10D7B0005DF804FB9FED156A90ED817ADFED146A48
:10D7C000D0ED837A27EE067A67EE867A27EE267A00
:10D7D00067EEA67ABDEEC77AFDEEE77A80ED7E7A37
:10D7E00090ED827A27EE067A17EE903A27EE267AA7
:10D7F000002BB8BF03F50C43BDEEC77AB8BFA0330A
:10D8000080ED7F7AC0F80032704700BFE02E65429D
:10D810000000C8421FB50E4B1B680446B3B16846F2
:10D8200004F094FC69462046FFF704FC20B16A46E8
:10D8300000212046FDF78AFF94F87C32DB0705D5EE
:10D8400004F51B7201212046FDF780FF04B010BDD6
:10D850001482002008B502F03DF9BDE8084001F04F
:10D8600059BD000010B580F8F812044670F008FEAB
:10D87000C4F8FC0210BD000010B590F8F832044660
:10D8800053B170F0FDFDD4F8FC32C01AB0F57A7FC8
:10D8900084BF002384F8F83294F8003353B170F059
:10D8A000EFFDD4F80433C01AB0F57A7F84BF0023AB
:10D8B00084F8003310BD000000F5AA700B4607C8BD
:10D8C00083E80700012070470023C0F89C30C0F8AF
:10D8D0009830C0F89430C0F8A830C0F8A430C0F830
:10D8E000A030C0F8AC30704770470000024B0B60AE
:10D8F0004FF07C53136070470000484270470000AF
:10D9000008B50B4600F12801184617F05BFB012013
:10D9100008BD000010B500F5B4700C460FC884E8CF
:10D920000F00204604F002FC30B1FFF791FD00F536
:10D930001B700FC884E80F00204604F0F7FB80F04E
:10D940000100C0B210BD000010B5044604F054FF41
:10D95000204610BD10B5D0F8603104465BB170F0C0
:10D960008FFDD4F86031C01A41F28833984294BFD9
:10D970000020012010BD0120FCE7000013B500933A
:10D9800003680192D3F890309847DDE900210446FE
:10D9900028B90448044B0068C06A12F00BFD204609
:10D9A00002B010BD082700205C5C0C0813B50446CB
:10D9B0000191FDF7DDFD2368019A1B6D014608B159
:10D9C00090F84E11204602B0BDE810401847000004
:10D9D00030B585B0002301930293039303680D468D
:10D9E000DB6D01A99847044620B1039B2B602046BC
:10D9F00005B030BD02F06EF8417C01F0C7FD044671
:10DA00000028F4D002F066F801F026FDB1EE400ADD
:10DA100085ED000AEBE7000010B5FDF7A9FD04460F
:10DA200058B190F84E11FDF74BFB30B194F84E1100
:10DA30002046BDE81040FDF73FBC002010BD0000AF
:10DA400038B50D460EF0ACF90446FEF731F8022861
:10DA500081BF94F8F402B02303FB004000F582700C
:10DA600089BF07C8002085E80700012038BD0000F5
:10DA70002DE9F0432DED028B8FB003680025DB6CA0
:10DA80000395049505950695029502A904469847C5
:10DA9000064638B1FFF7DEFEDDED027A27EE800A9A
:10DAA0008DED020A0EF07CF9FEF702F80746002E13
:10DAB00050D0DDED027AD4ED646A94ED657A236886
:10DAC0000B9527EE877A67EEA67A8DED097ACDED74
:10DAD0000A7A0C950D959B6C0BA9204609AD9847C9
:10DAE0000BA9284617F054FF012F8DED030ACDED49
:10DAF000040A40F2B3800EF053F990F8F432DFEDEF
:10DB00005B7AB02505FB030090ED3C8A28EE278A5E
:10DB1000B0EE480A9BF0C6FCF0EE408AB0EE480A30
:10DB20009BF016FECDED0B8A8DED0C0A0EF038F948
:10DB300090F8F43205FB030090ED3B0A0BA817F0B8
:10DB400047FF09AD8DED050ACDED060A05A896BB88
:10DB500003C885E00128CED89DED020AB5EEC00AC3
:10DB6000F1EE10FA7FDD07AED4F89421D4F89031AD
:10DB700007923046089317F067FF23680B950C95C2
:10DB80000D959B6C0BA920469847DDED077A9DED1E
:10DB90000B7A77EE877A9DED0C7ACDED077ADDED85
:10DBA000087A77EE877A09ABCDED087A96E803001C
:10DBB00083E8030049E0236993ED000AB7EE008A89
:10DBC00038EE408A17F004FF04F5BC798DED090AA0
:10DBD0004846B0EE480ACDED0A0A17F0F9FE0BA947
:10DBE0002846CDED0C0A8DED0B0A17F0D1FE04F599
:10DBF000C47603AFC4ED5F0A314684ED5E0A384651
:10DC000017F0D6FE04F5C0788DED090A4046B0EE57
:10DC1000480ACDED0A0A17F0DBFE0BA928468DED68
:10DC20000B0ACDED0C0A17F0B3FE97E8030084ED64
:10DC3000600AC4ED610A86E803004946404617F0D1
:10DC4000A7FE8DED090ACDED0A0A9DED090ADDED6D
:10DC50000A0A0FB0BDEC028BBDE8F083DDE90301D9
:10DC600085E80300F1E709950A95EEE735FA8E3C61
:10DC700010B590F84213044604F058FF7C23C0B25C
:10DC800003FB0044D4F8A00010BD0000044B026F59
:10DC90001B68DB6A5A60426F9A60826FDA60704775
:10DCA00008270020F0B58FB0044615F041F9002395
:10DCB00002930393049390F8121301AB02AA054652
:10DCC00014F06AF904F19407D8B39DED010AB5EE9A
:10DCD000C00AF1EE10FA34DD02A818F0FBF904F1E5
:10DCE000B00684ED2C0AC4ED2D0A84ED2E1A3946B7
:10DCF000304618F0FFF904F17C01304618F0AEF917
:10DD000004F1880105A88DED050ACDED060A8DED1B
:10DD1000071A18F0A3F908A88DED080A9DED010A6D
:10DD2000CDED090A8DED0A1A18F0C4F90BA904F11A
:10DD300028008DED0B0ACDED0C0A8DED0D1A16F0B5
:10DD400061FB95F812030C2303FB0050394600F5E4
:10DD5000117018F083F984ED2C0AC4ED2D0A84EDBE
:10DD60002E1A0FB0F0BD00002DE9F047824B0025C0
:10DD70001F682DED028BC0F89C50C0F89850C0F879
:10DD80009450C0F88450C0F88050C567C0F89050D7
:10DD9000C0F88C50C0F88850C0F8B850C0F8B450E3
:10DDA000C0F8B0500446F86A03688AB05B680E4653
:10DDB000984704F12809002854D070F061FB42F222
:10DDC0000F7398424ED8FB6A9FED6C8A93ED010A5F
:10DDD00084ED1C0AD3ED020AC4ED1D0A93ED031A6B
:10DDE000484684ED1E1A16F001FA4AF093FCD4ED71
:10DDF0001E7A67EE887A054617EE900AF2F784FBE2
:10DE0000D4ED1D7A67EE887ACDE9040117EE900A09
:10DE1000F2F77AFBD4ED1C7A67EE887ACDE902013D
:10DE200017EE900AF2F770FB554ACDE90001062182
:10DE3000284643F0BBFD94ED1E8AB0EE480A9BF0E5
:10DE400031FB84ED650AB0EE480A9BF081FC84ED5D
:10DE5000640A70F015FBC4F864010AB0BDEC028BD3
:10DE6000BDE8F087A6B194ED1C0AB4EE400AF1EECD
:10DE700010FA0DD6D4ED1D0AF4EE600AF1EE10FA98
:10DE800006D694ED1E1AB4EE411AF1EE10FA52D7EE
:10DE900015F04EF890F813334FF00C0A0AFB030309
:10DEA00003F5C473074693E8070007AE86E807004A
:10DEB0004FF01508B2EE028AF2EE068A304618F0EC
:10DEC000F7FCB4EEC80AF1EE10FA38D508F1FF38C5
:10DED00018F0FF083CD1304618F0EAFCF1EE047A65
:10DEE000B4EEE70AF1EE10FA43DD9DED090ADDED2F
:10DEF000087A9DED078A20EE000AA7EEA70A9BF09C
:10DF00003DFEF0EE400AB0EE480A9BF0EDFCDDED80
:10DF1000090A84ED1D0A9DED080AF1EE600AB1EED2
:10DF2000400A9BF0E1FC84ED1C0A9FED161AD4ED2B
:10DF30001D0A94ED1C0A484616F058F97BE7304656
:10DF400018F0B6FCB4EEE80AF1EE10FABEDCC2E757
:10DF5000384613F0E3FE384613F0A8FF97F8133362
:10DF60000AFB037303F5C47393E8070086E8070010
:10DF7000A4E725676567D8E708270020E02E6542FB
:10DF8000D05D0C08000000000021FFF7EDBE00008E
:10DF900037B5044608461546019118F089FCB7EEDE
:10DFA000007AC7EE007AB4F8D03001980133A4F8B3
:10DFB000D03094ED337A37EE277A84ED337AB0EEB1
:10DFC000007AF4EEC77AF1EE10FA06D5B6EE007AD2
:10DFD000F4EEC77AF1EE10FA0DDC9FED0E7AF4EE56
:10DFE000C77AF1EE10FA13D59FED0B7AF4EEC77AEB
:10DFF000F1EE10FA0CDDB0EE670A18F05BF80120C4
:10E0000085ED000AC5ED010A85ED021A03B030BDA9
:10E010000020FBE700247449BD37863570B52DED2F
:10E02000028B00F1280600F134058AB02946044627
:10E03000304618F0BBF8B6EE008A20EE088A284673
:10E04000B0EE480A18F036F807A93046CDED080AB8
:10E050008DED091A8DED070A18F016F830468DED92
:10E06000010AB0EE480ACDED020A8DED031A18F050
:10E0700021F807A928468DED070ACDED080A8DED98
:10E08000091A18F001F804A901A88DED040ACDEDD4
:10E09000050A8DED061A18F09DF8324601A92046B2
:10E0A0008DED070ACDED080A8DED091AFFF770FF17
:10E0B00058B970F0E5F90121C4F860012046FFF776
:10E0C00053FE0AB0BDEC028B70BD2A4604A920465F
:10E0D000FFF75EFF0028ECD004F1400207A92046BC
:10E0E000FFF756FF0028E4D0EBE7000030B52DED38
:10E0F000028B0D4683B091F842130446284604F083
:10E1000015FDC1B27C2000FB0151903104F12800C3
:10E1100015F0FCFE68468DED000ACDED010A17F002
:10E1200015FDDFED1C7AB4EEE70AF1EE10FA05D525
:10E130009FED190A03B0BDEC028B30BD684617F0A5
:10E1400083FD684617F0DCFC0028F1D1284694EDE9
:10E15000428A04F04FFEF0EE400AB0EE480A15F095
:10E16000EBFA80B9284604F045FE84ED420AB0EE91
:10E17000408A9BF097F984ED430AB0EE480A9BF081
:10E18000E7FA84ED440A04F58671684617F086FCC8
:10E19000D0E700BF00000034000000009FED0C7AC3
:10E1A000B4EEC70AF1EE10FA0BD4DFED0A7AB4EE42
:10E1B000E70AF1EE10FA07DCC0EE077AB0EE670A64
:10E1C0007047F7EE007AF9E7F2EE047AF6E700BF5F
:10E1D000F3665F3F58A00B4108B51C3017F0B6FC42
:10E1E000F1EE007AB4EEE70AF1EE10FA9DBFF1EE1F
:10E1F000027A37EEC00ADFED047A9FED040A98BF79
:10E2000020EE270A08BD00BFCDCC4C3ECDCCCC3D86
:10E2100008B5836993F9000038B10DF0C1FDFDF731
:10E2200047FC012894BF0020012008BDF8B52DED62
:10E23000028B054605F050F804F04CFF0446B8B3D5
:10E24000FFF706F990F8093393B32846FFF7E0FF8C
:10E25000064668B30DF0A4FD90F8F432B02707FB32
:10E26000030090ED3B7AF0EE087AB4EEE77AF1EE37
:10E2700010FA1DD495ED1E8A0DF092FD90F8F4323F
:10E28000DFED1E7A07FB030090ED3C0A98EE270AAB
:10E2900015F0D6FADFED1A7AB0EEC00AB4EEE70A4E
:10E2A000F1EE10FA08DC70F0EBF83446C5F85001D6
:10E2B000BDEC028B2046F8BD05F5AA7018F0F8FAFF
:10E2C000B0EE408A0DF06CFD90F8F4329FED0D7ABF
:10E2D00007FB0303D3ED3B7A67EE877AB4EEE78A58
:10E2E000F1EE10FADFD570F0CBF8D5F85041001BF5
:10E2F000B0F5FA6F8CBF00240124D9E7E02E654207
:10E3000000003442CDCC4C3F10B50A4B1B68DB6A91
:10E3100093F89C3004465BB970F0B2F8D4F86431DD
:10E32000C01A44F61F6398428CBF0020012010BD24
:10E330000020FCE708270020F8B52DED068B0446E9
:10E340000DF02EFD054604F0C7FF064607F0FEFC63
:10E35000002840F0AB802046FFF768FF002800F05F
:10E36000A8803046FFF784FCD4F8DC30984200F0F7
:10E370001A813046FFF77CFCD4F8DC30DFED8F7A71
:10E38000C31A08EE903AF8EE688A304668EEA78A1B
:10E39000FFF76EFC94F8BC30C4F8DC00F3B93046EB
:10E3A00004F0AAFED0B104F1280796F842233946BA
:10E3B000304604F023FDD4ED1D0AB0EE401A384675
:10E3C00094ED1C0A15F012FF0023C4F89030C4F835
:10E3D0008C30C4F88830012384F8BC3020463146A4
